:020000040000FA
:040000006FD00400B9
:101000006F009044000000000000000090200020CD
:10101000A4220020A9BDF9F55C23002000000000F7
:10102000000000005C230020902000200000000051
:101030000000000090200020000000009020002010
:101040000000000090200020902000209020002030
:101050009020002090200020B82B0020902000201D
:10106000000000009020002090200020EC230020B1
:1010700090200020C22300209020002090200020FB
:101080009020002090200020902000209020002020
:101090009020002001A04111B7170040985F3AC688
:1010A000945F3247E39CE6FE3245410182800111A4
:1010B00013078008F337078093F787083EC20100C3
:1010C0000100B7170040930570052380B70413068D
:1010D00080FA2380C7040100010083C6B70493F699
:1010E000F60DA385D704238007049246F3A6068055
:1010F0000100010093760502D5CEF336078093F602
:10110000860836C4010001002380B7042380C70489
:1011100001000100B70614007D89558D88C70100C4
:1011200001000100010023800704A246F3A6068007
:101130000100010073370780137787083AC6010062
:1011400001002380B7042380C704010001000100CF
:1011500001003727004093061005A303D7802380A2
:101160000704B247F3A70780010001009307800836
:10117000F3B7078093F787083ECE01000100B71749
:101180000040130770052380E704130780FA2380CB
:10119000E7040100010003C7B70413670708A3852C
:1011A000E70423800704F247F3A70780010001004A
:1011B0000561828093760504BDC6F336078093F6F9
:1011C000860836C8010001002380B7042380C704C5
:1011D00001000100B7061400938606047D89558D31
:1011E00088C7010001000100010023800704C246F6
:1011F000F3A6068001000100733707801377870884
:101200003ACA010001002380B7042380C70401000B
:1012100001003727004093062005A303D7802380D1
:101220000704D24781B773370780137787083ACC12
:10123000010001002380B7042380C70401000100DE
:1012400098471367070C98C723800704E24719BF24
:101250000111814601468145114506CE6D24930753
:101260008008F3B7078093F787083EC601000100A6
:10127000B7170040130770052380E704130780FAAF
:101280002380E7040100010003C767041367170008
:101290002383E70423800704B247F3A707800100F4
:1012A0000100F2400561828041118146014681457D
:1012B0001145912C13078008F337078093F78708AF
:1012C0003EC401000100B7170040130670052380DB
:1012D000C704930680FA2380D70401000100FD555E
:1012E0002396B70223800704A245F3A505800100D9
:1012F000010073370780137787083AC601000100A1
:101300002380C7042380D7040100010003C76704BA
:10131000136717002383E70423800704B247F3A76A
:1013200007800100010001A0BD473305F50201005F
:101330007D1575FD8280411122C426C206C6AA848D
:10134000014463179400B2402244924441018280D8
:1013500005041305803E4204C13F4180DDB7000013
:101360009305000273A04580824573901534924026
:101370002242B2424243D2436244F2440255925561
:101380002256B2564257D2576258F25806499649E9
:10139000264AB64A464BD64B664CF64C065D965DE1
:1013A000265EB65E465FD65F09617300203041114C
:1013B000B7170040985F3AC6945F3247E39CE6FE59
:1013C000324541018280B71700401307000323888C
:1013D000E7028547171700002326F7F47300203033
:1013E000411122C406C6370400201C408297F5BF75
:1013F00037370040834747009146BD8B6389D7004C
:1014000099466394D700834757407300203097165E
:10141000000083C6F6F39387160017160000A30991
:10142000F6F203478700973700009387E7FCB697EB
:101430002380E700B7E70400BC4F0946894517152C
:1014400000000345C5E98297C9B723030480154707
:101450002303E48001002302A48082808307648048
:10146000E3CE07FE23030480828083076480E3CEFB
:1014700007FE03454480828083076480E3CE07FE35
:101480002302A4808280411126C44AC24EC006C6EF
:101490001377F50BAD47AA892E8995446306F700AB
:1014A00019456537653F8D444E854537FD59FD1417
:1014B00063983401B240A2441249824941018280BA
:1014C000135509011375F50F453F2209CDB70111D9
:1014D00026CC06CEB704080051371545BD37713705
:1014E00069372AC6A53F32459377150089EB136506
:1014F00015001375F50FF240E24405618280FD147A
:10150000E9FC0145CDBF397126DC4ADA4ED852D606
:1015100056D45AD25ED006DE62CE66CCB7E700E083
:101520007D5783AA070022C603AA470023A0E71815
:1015300023A2E718B7170040130770052380E704BC
:10154000130780FA2380E70483C74704930B75FFD2
:10155000B684E20793FBFB0F8546AA892E8B32895E
:1015600037240040E187015763FA76016308D5000C
:101570008946130700026313D5000157D98F93F7EB
:10158000F70FB71C00402382FC0411472303E480BB
:101590001305F00F5D3D094CD135636D7C11B70526
:1015A0000700DA9537870700795563F2E504B387BA
:1015B0009500636EF702370B0800A94733EB65010E
:1015C0006399F90689E48144513D26850DA0DA85A9
:1015D0000945553D05090345F9FFFD14050B693D16
:1015E00081C49377FB0FFDF7DD3569FD7D55B71796
:1015F0000040130770052380E704130780FA238057
:10160000E70403C74704418B2382E704F250B7E79E
:1016100000E023A0571123A24711E254324452594B
:10162000C259325AA25A125B825B724CE24C21615F
:101630008280A5476395F90685691309F00FB30603
:101640009900B3742B01B6941349F9FFB374990050
:10165000856B33796901416B9387F9FFB3F72701F4
:1016600099E363FC340193D94900C147E3E637FFAE
:1016700099BF0569C1697D19D9B71305800D6388C4
:101680006901130500026384790113051008CA85F6
:10169000DD3B353D21DD4E99B3843441D9B7DA8540
:1016A0002D45D533CA94E30099F205097D3BA30F7C
:1016B000A9FED5BF9387F9FF93F7F70F6361FC0C81
:1016C00083C71C0413073008631FF704370708009B
:1016D000636BEB04B3079B00B706100063F5D704F8
:1016E000334BEB0089476393F9068980D549E38C36
:1016F00004ECDA850945413B11090327C9FF9147ED
:101700002320E48003076480E34E07FE2303348133
:10171000FD17EDFBFD14110B81C49377FB0FE9FF5F
:101720007D3371F5E1B5B717004003C75704B7071C
:1017300008001377070219E3B78707007955E378A4
:10174000FBEA33079B00E3FFE7F855B58547E382E3
:10175000F9F2DA852D45053B9389F4FFE38504E62C
:10176000293393F7390091EB83260480032709007E
:1017700093074900E39AE6E43E89CE84F1BFB5477A
:101780006396F9001305900BC93135BDB1471305B8
:10179000B00AE38BF9FE99476391F904B705080095
:1017A000B365BB002D45C53181448D4BA1497539C9
:1017B00063967401832704802320F9008504E3984D
:1017C00034FF8327048013172B016355070023126E
:1017D000F900D5BB2322F900FDB39D476399F902B7
:1017E00081451305B0044531BD442320090023225F
:1017F0000900FD599D3993F77400CA9703C7070084
:10180000FD14398D2380A700E39634FF6DBBA147FB
:101810006392F9046D398144630D0B008D47930485
:10182000C0036308FB009304000563048B01930469
:1018300040041375C507E30895D81945393139397E
:101840000545213126850D3909453D314931E31CD6
:1018500005D669BB91476399F90013056006F53613
:10186000F53E130590090DB7E38F09D4F154A9BBD8
:10187000BD660147173600001306C6E4938606A628
:1018800085458347060093F7F70F91C382800507CC
:10189000E3F9E6FE973700002386B7E2DDB77D1651
:1018A0006206618693178601E18763D407000145CC
:1018B0008280931726003307F500AE9718439C43A8
:1018C00063E7E7007D16E37FF7FC7D5582800545E1
:1018D0008280FD15E205E18513978501618793F705
:1018E000F50F63480700FD15139725002A97584305
:1018F00065D7138517006205618582803308B502BC
:101900001C4283A80600B335B502C29733B5070160
:10191000AE98469585486367B5006394A50063E378
:10192000070181480C43C6950CC388C21CC2828043
:1019300081471397870161876343B70082801397BC
:1019400027002A97232007008507E5B7814701472D
:1019500093968701E18663C5B60013351700828030
:1019600093962700AA9694428507558FD5B793D7AB
:1019700055408A07AA979C4305453315B5007D8DD0
:10198000828017F3FFDFE702C33B2A84993705C53E
:10199000931725003E940327C4FF814711EB7D1563
:1019A00016053E954205418517F3FFDF6700A33B0F
:1019B00005838507E5B70145C5BF814713978701B3
:1019C00061876343C700828013972700B386E500D1
:1019D00094422A97850714C3D5B77D16620661869F
:1019E000014793178601E18763D507001335170078
:1019F000828093172600B306F500AE9794429C436D
:101A00007D16B58F5D8FF1BF8A05AA950147636387
:101A1000B500828083A6C5FFF11593D71600D98F34
:101A20009CC11397F601E5B72A8301480147014598
:101A30006343D7008280B387050183A80700B307FB
:101A400006019C43C697AA976384F80033B5170133
:101A50000507B3080301620723A0F8006187110896
:101A6000C1BF2A8301478147014563C3D7008280F4
:101A70003388E50083280800330EE600032E0E00AD
:101A80003388A8403308C8416384080133B508018E
:101A90008507B308E300E20723A00801E1871107E7
:101AA000E9B717F3FFDFE702C3290111B286B28459
:101AB0002E86AA850A8575372A84A6850A857935F2
:101AC00033348000060413351500018D056117F3CA
:101AD000FFDF6700432917F3FFDFE702032441110B
:101AE000AA89AE8A328BB68402C202C402C60144FD
:101AF000131C8401135C8C4163499C02939B14006A
:101B0000FD1B0549138CF4FFF15C33048901620469
:101B10006184634D740592478E04CE9423AEF4FE27
:101B2000410117F3FFDF6700C32213192400B30B31
:101B30002B01014A93172A00D69783A50B008843EF
:101B40007800340050005D3B050A93178A01E18755
:101B5000F11BE351FCFE92474E9905042320F90046
:101B6000A2473EC2B24702C63EC459B7131A890102
:101B7000135A8A41131D240093178A01E18763CF0A
:101B8000970092470A044E941CC0A2470509137996
:101B9000F90F3EC2B24702C63EC485BFB3079A03DF
:101BA00013152A0056950841780034005000050AA4
:101BB000EA97DA978C439933C1B70000197106C2CE
:101BC00012C416C61AC81ECA22CC26CE2AD02ED2BD
:101BD00032D436D63AD83EDA42DC46DECAC0CEC26D
:101BE000D2C4D6C6DAC8DECAE2CCE6CEEAD0EED29D
:101BF000F2D4F6D6FAD8FEDA97050000938505727E
:101C00008841E700050092402242B2424243D2435B
:101C10006244F244025592552256B2564257D25768
:101C20006258F25806499649264AB64A464BD64B60
:101C3000664CF64C065D965D265EB65E465FD65FE8
:101C40000961730020300000972100209381813BBF
:101C500017510020130101BB17F5FFFF1305C53A0B
:101C6000970500209385053A171600201306C6FD38
:101C700063FAC5008322050023A0550011059105D4
:101C8000E3EAC5FE17A50100130545559715002089
:101C90009385C5FB171600201306C66563FAC500B9
:101CA0008322050023A0550011059105E3EAC5FE36
:101CB000171500201305056497450020938585ECD2
:101CC0006377B500232005001105E36DB5FEFD42E5
:101CD000739002BC8D4273904280B72200009382C1
:101CE000828873900230970200209382A23193E29F
:101CF00032007390523097420000938202F5739045
:101D000012346FC0E42F73002030397101436EC666
:101D100019A0397141536AC866CA62CC5ECE19A057
:101D2000397101535AD056D252D44ED64AD826DAF7
:101D300022DC06DE33016140828241114AC026C2A4
:101D400022C406C68282B24D4101024D924C224C01
:101D5000B24B4101024B924A224AB2494101024927
:101D600092442244B240410182803D432A876373FA
:101D7000C3029377F700BDEFADE5937606FF3D8A8A
:101D8000BA960CC34CC30CC74CC74107E36BD7FED4
:101D900011E28280B306C3408A069702000096963D
:101DA0006780A6002307B700A306B7002306B70085
:101DB000A305B7002305B700A304B7002304B700A9
:101DC000A303B7002303B700A302B7002302B700A1
:101DD000A301B7002301B700A300B7002300B70099
:101DE000828093F5F50F93968500D58D9396050126
:101DF000D58D61B79396270097020000969686824C
:101E0000E78086FA9680C1171D8F3E96E374C3F86B
:101E1000A5B73367B500FD530D8B79E7B7877F7F93
:101E20009387F7F710419441B372F6003363F600DD
:101E3000BE92B3E262006397720C6318D6065041FB
:101E4000D441B372F6003363F600BE92B3E262008F
:101E50006398720A631BD60410459445B372F6006A
:101E60003363F600BE92B3E262006391720A631EAE
:101E7000D6025045D445B372F6003363F600BE92E5
:101E8000B3E26200639A72086311D6021049944962
:101E9000B372F6003363F600BE92B3E2620063935E
:101EA00072085105D105E30FD6F613170601939773
:101EB0000601631CF7001357060193D7060133058B
:101EC000F7409375F50F91E982804183C183330513
:101ED000F7409375F50F91E182801377F70F93F731
:101EE000F70F3305F74082800346050083C60500DF
:101EF000050585056313D60065FA3305D640828053
:101F000011059105E312D6FE014582802105A10548
:101F1000E31CD6FC014582803105B105E316D6FCF1
:101F2000014582804105C105E310D6FC0145828050
:101F3000B717004003C777051377E70FA38BE704B4
:101F4000130700F8A38DE7043D47238CE70413072C
:101F50005003A38CE70403C7A7051377D70F238D7E
:101F6000E7048280B717004003C7E7020D894111DB
:101F70001377C70F498F93068008F3B6068093F650
:101F8000860836C601000100930670052380D70439
:101F9000930680FA2380D704010001002387E7021B
:101FA00023800704B247F3A7078001000100410125
:101FB000828041112A83014E930E407E130F001937
:101FC000930F400663E56E12930800191303400651
:101FD000B3781503854E0D4FA14F337365020D89FC
:101FE0001335150063EFBE121308F6FF7946729899
:101FF0004208135808013307C70213D61700BE075B
:1020000032976146B3F6C60213068070B386C602E5
:102010003697A166F58F42075D8FB716004083C7DC
:10202000F60293F70708A303F1000346710083C784
:10203000F60293F70708E394C7FE83477100B716CB
:10204000004093F7F70F6388071293078008F3B7F0
:10205000078093F787083EC401000100B7170040CE
:10206000930670052380D704930680FA2380D70453
:102070000100010023AA070383C6170393E606089D
:10208000A388D70223800704A247F3A70780010093
:1020900001001166B71700407D16D45BC85F9385B9
:1020A0004703A98EF18EF5FA93068008F3B60680F1
:1020B00093F6860836C6010001009306700523805A
:1020C000D704930680FA2380D7040100010098C149
:1020D00003C7170313670704A388E70223800704D5
:1020E000B247F3A7078001000100410182807D1300
:1020F0003368E3039308E016630E08003368F303C4
:102100009308D016630808009378330093B818003A
:102110009388D81633081E01131E0801135E0E01A2
:1021200055B56393E50305486386080001486303DA
:1021300003002A8871087298FD15131E0801C20554
:10214000135E0E01C18179BD13F8150063F4BF0061
:102150007908D5B713381800E5BF83C7F60293F79F
:102160000708A303F1000346710083C7F60293F743
:102170000708E394C7FE8347710093F7F70FF1DF79
:10218000E9B531714AD966CB06DF22DD26DB4ED7B1
:1021900052D556D35AD15ECF62CD6AC96EC7AA8CCA
:1021A00002D8EF00901C2A8993078008F3B70780B4
:1021B00093F787083EDA01000100B71700401307C4
:1021C00070052380E704130780FA2380E7040100E9
:1021D000010003C7F7021377770FA387E70203C74E
:1021E000F70213678700A387E70223800704D2570B
:1021F000F3A70780010001000545AD33130780C137
:102200003347E902116A93070AE893065002BD6951
:10221000930BA004814A014B1304800893047005BA
:102220007D1AB347F9023307D7023EC0FD873ECC83
:10223000938709A69309803E3347F7023AC27D8708
:102240003AC4334739038549B399990193D9394041
:10225000B306D702B30B7703B3C6F602B3CBFB02C8
:1022600036C6FD8636C893D6FB4136CEB7460F003C
:10227000938606243349D9028566938606FAB39677
:102280009601B389E902130760553309D902930611
:102290000010B389E9023349D902B3C9F902931690
:1022A000390036CA37190040FD8636D0930D09042F
:1022B00093D7F9413ED2F336048093F6860836DC94
:1022C00001000100930770052380FD00930680FA4A
:1022D0002380DD00010001008346390593F6860F57
:1022E000A309D9048346390593E61600A309D90446
:1022F00023800D00E256F3A6068001000100130CB6
:1023000080FA116DF336048093F6860836DE0100FC
:102310000100930770052380FD0023808D010100DB
:10232000010083463905216693E60602A309D90414
:1023300083560905B3E6A6012318D9048356090577
:10234000D18E2318D90423800D00F256F3A60680FF
:10235000010001008346390593F60602638A0618D8
:1023600003463905218A6DDE0818EF001004733624
:10237000048013768608B2C20100010023809D000C
:1023800023808D0101000100B717004003C6370507
:102390001376F60DA389C70403C637051366060234
:1023A000A389C704835609052166B3E6A60123184D
:1023B000D90483560905D18E2318D90423800D0032
:1023C0009646F3A60680010001008346390593F680
:1023D00006026386061483463905A18AEDFE97003E
:1023E0000020E78040CBAA8636D497000020E78003
:1023F00080CAA256E30AD5FE835609054255B3E6C4
:10240000A6012318D904C12783463905A18AEDDE28
:10241000035609058346290582473376CA00B30669
:10242000DA0293D5F641B296B388F640E24733B864
:10243000C6002E983308F840A247B3B616013308F9
:10244000D84063C70701631DF800924763FA17017C
:10245000C247634DF80E63950701B24763E8F80E73
:10246000894663E7660FF2469315180013D3F80107
:102470005E8613951800B365B30042D646D4EF606C
:10248000213C3258050B137BFB0F6347000163129D
:102490000838A258638F083613081500B336A80011
:1024A000B69513D6F5013298B336C800AE961358D8
:1024B0001800FE06B3E6060173360480137686081C
:1024C000B2C60100010023809D0023808D01010020
:1024D00001000356C902B296C206C1822316D90270
:1024E00023800D00B646F3A606800100010019BD49
:1024F000F336048093F68608B6C0010001002380FD
:102500009D0023808D01010001008346390593E67B
:102510000602A309D90423800D00864605BDF336C3
:10252000048093F68608B6C40100010023809D0054
:1025300023808D01010001008346390593E60602E0
:10254000A309D90423800D00A646A5BDE30D0BF019
:10255000F336048093F68608B6C80100010093069E
:1025600080FA23809D002380DD0001000100834666
:10257000390593F5FC0F93F6860FA309D90483461A
:102580003905CD8EA309D90423800D00C646F3A6D4
:10259000068001000100130580FA03463905930601
:1025A00039051D8A631496297336048013768608CC
:1025B000B2CC01000100130680FA23809D00238025
:1025C000CD000100010003C606001376F60D23803E
:1025D000C60003C60600136606022380C6008356A3
:1025E00009051166D18E2318D90483560905216681
:1025F000D18E2318D90423800D00E646F3A6068069
:1026000001000100130680FA8346390593F606029D
:102610006388062483463905130C3905A18AFDDA3F
:1026200008186123F336048093F68608B6D00100BB
:102630000100930680FA23809D002380DD000100C5
:10264000010083460C00116693F6F60D2300DC00B2
:1026500083460C0093E606022300DC00835609053E
:10266000D18E2318D904835609052166D18E2318EB
:10267000D90423800D008656F3A6068001000100D0
:10268000130680FA8346390593F606026385062011
:1026900083463905A18AEDFE97000020E780A09FC0
:1026A0002A8C97000020E780009FE30C85FF83566B
:1026B000090511664255D18E2318D9042923834672
:1026C000390513063905A18AFDDAF336048093F63D
:1026D0008608B6D401000100930680FA23809D008D
:1026E0002380DD00010001008346060093F6F60D0D
:1026F0002300D60023800D00A656F3A60680010015
:1027000001008356090503462905D247B376DA004E
:102710003306CA021305800C9355F6413696330DE5
:10272000F6408257333CD6002E9C3336A601330C3C
:10273000FC40330CCC403308850392564E86B335AB
:10274000A5033305A503C295EF60810F63468001A1
:10275000631E0C16630C0D16130615003335A60008
:102760002E959356F5013696B335D600AA959396D5
:10277000F50105828585D18E6346B000639D051AFB
:10278000638B061A0356C90215823305D600333609
:10279000C500B2956348B000639105241306F00F9D
:1027A000637DA622894663F3561593078008F3B725
:1027B000078093F78708BED6010001003717004055
:1027C000930770052300F704930780FA2300F704AA
:1027D000010001008356C70289678117D58FC207A0
:1027E000C1832316F70223000704B657F3A7078017
:1027F00001000100FA506A54DA544A59BA592A5A67
:102800009A5A0A5BFA4B6A4CDA4C4A4DBA4D296126
:1028100082801308F5FF3335A800FD152E95135659
:10282000F5013298B336C800AA9651B1F336048048
:1028300093F68608B6CA0100010023809D0023801C
:10284000AD000100010083463905CD8EA309D904EE
:1028500023800D00D646F3A606800100010035BB9B
:10286000F336048093F68608B6CE0100010023807B
:102870009D002380CD00010001008346390593E6C9
:102880000602A309D90423800D00F646F3A60680AC
:102890000100010095BBF336048093F68608B6D29A
:1028A0000100010023809D002380CD000100010074
:1028B0008346390593E60602A309D90423800D0057
:1028C0009656F3A60680010001006DBB9306F5FF46
:1028D00033B5A600FD152E959355F501AE96B3B50B
:1028E000B600AA951396F501858269B5F336048082
:1028F00093F68608B6D801000100930680FA23807B
:102900009D002380DD00010001008356C902056699
:10291000011693F6F60FD18EC206C1822316D90294
:1029200023800D00C656F3A6068001000100850A2B
:1029300093FAFA0F49B233E6B60045C20356C9020C
:102940003305D0403338A000B305B040B38505410E
:1029500015826345B000D1E16371A608894663F032
:10296000560593078008F3B7078093F78708BEDA08
:1029700001000100B7170040130770052380E7042A
:10298000130780FA2380E7040100010003D7C70280
:102990007D8B2396E70223800704D65781BDF3364B
:1029A000048093F68608B6DC01000100930680FAE5
:1029B00023809D002380DD00010001008356C902B1
:1029C0000566011693F6F60FD18EC206C182231654
:1029D000D90223800D00E656B9B793078008F3B7F4
:1029E000078093F78708BEDE01000100371700401B
:1029F000930770052300F704930780FA2300F70478
:102A0000010001000356C70293975600B297C20710
:102A1000C1832316F70223000704F657C1BB914771
:102A200063EEB70217870100130707B28A05BA954C
:102A30009C41BA978287B717004003A7470B1345FD
:102A4000F5FF698F23AAE70A03A7070B698F23A85D
:102A5000E70A03A7070A798D23A0A70A8280B71780
:102A6000004083A6470B1347F5FFF98E23AAD70A28
:102A700083A6070B558D23A8A70A83A6070A758F7F
:102A800023A0E70A8280B717004003A7470B498FAE
:102A900023AAE70A03A7070B1345F5FF45BFB7179E
:102AA000004083A6470B1347F5FF758F23AAE70A5B
:102AB00003A7070A598D4DB7B717004003A7470B67
:102AC000498FEDB7914763EEB702178701001307EF
:102AD000E7A88A05BA959C41BA978287B717004044
:102AE00003A7470D1345F5FF698F23AAE70C03A73A
:102AF000070D698F23A8E70C03A7070C798D23A086
:102B0000A70C8280B717004083A6470D1347F5FF37
:102B1000F98E23AAD70C83A6070D558D23A8A70CE1
:102B200083A6070C758F23A0E70C8280B71700409F
:102B300003A7470D498F23AAE70C03A7070D1345E9
:102B4000F5FF45BFB717004083A6470D1347F5FFB4
:102B5000758F23AAE70C03A7070C598D4DB7B7173C
:102B6000004003A7470D498FEDB7B71700408847CE
:102B7000420541819377050491EB9377F501375531
:102B8000E801130505803345F50282809377050C33
:102B9000130700046397E7009377F50137459C1C02
:102BA000CDB72165130505D0828037E700E01C43CF
:102BB0005443A183E206D58F1CC1FD572320F7188B
:102BC0002322F718828013178500B7E700E023A0BF
:102BD000E710618123A2A7108280B7F700E0884741
:102BE000CC478280814737370040A14663C4C70085
:102BF000328582800345B740E38EA6FE3385F5001B
:102C00000345050085072304A740CDB7970700209B
:102C10009387476A9C43173700201307A7F63E9512
:102C2000636EE500174700201307C79D6368A70080
:102C3000170700202320A7683E858280FD57EDBF3F
:102C4000411122C406C62A840D372947B307E5027D
:102C5000B2408D83B3D7870222449507B3D7E702EA
:102C600037370040C207C1832316F7004101828035
:102C7000716541111305052006C6D937B7370040E5
:102C8000130770F82381E7000D47A381E7001307BE
:102C90000004A380E70005472387E700B240410115
:102CA000828037370040834727001A0593F7F703E0
:102CB000C98F93F7F70F2301F7008280B7370040E1
:102CC00003C7170019C9D98DA380B70003C7070030
:102CD000136787002380E700828093C5F5FFF98D95
:102CE000A380B7008280AE872A87B736004021468E
:102CF0003738004099E36F30200F83C8B600E30BEC
:102D000016FF05078348F7FFFD17C20723041801C4
:102D1000C183CDB7411122C406C62A84B9352947DB
:102D2000B307E502B2408D83B3D7870222449507EB
:102D3000B3D7E70237370040C207C1832316F740F5
:102D400041018280716541111305052006C6D937FE
:102D5000B7370040130770F82381E7400D47A38180
:102D6000E74013070004A380E74005472387E740B7
:102D7000B24041018280CC41411106C6328503C672
:102D8000150083C5050022064D8E42068D654186DD
:102D9000138875A2630C0611634BC804138845A2FF
:102DA0006300060D634AC800938535A26301B60827
:102DB0002390060029464DA0138855A26305060DF1
:102DC000938565A2E316B6FE8D451D4663E6E508CC
:102DD0001146198E63F3C7003E86B7E704002390BF
:102DE000C600FC4797950100938545399DA013883F
:102DF00095A263030611634E060D1388A5A2630016
:102E00000613938505A5E315B6FA99451D4663E5B6
:102E1000E504198E63F3C7003E86B7E704002390EC
:102E2000C600FC4797050020938545491DA09D4598
:102E30001D4663E3E5022146198E63F3C7003E8613
:102E4000B7E70400FC472390C60097050020938550
:102E5000654ABA9582970146B24032854101828027
:102E6000AD451D46E3EAE5FE3146198E63F3C70022
:102E70003E86B7E704002390C600FC479775010023
:102E80009385C570F9B7B1451D46E3E7E5FC3546C6
:102E9000198E63F3C7003E86B7E704002390C6008F
:102EA000FC47977501009385656F65B78D451D4695
:102EB000E3E4E5FA1146198E63F3C7003E86B7E7EF
:102EC00004002390C600FC47979501009385C52B0D
:102ED00049B78D451D46E3E1E5F81146198E63F3C8
:102EE000C7003E86B7E704002390C600FC479795CD
:102EF00001009385252BB1BFA5451D46E3EEE5F402
:102F00002946198E63F3C7003E86B7E70400239075
:102F1000C600FC4797750100938585661DBFB545C2
:102F20001D46E3EBE5F23946198E63F3C7003E8692
:102F3000B7E704002390C600FC479775010093850E
:102F4000256301BFB7E7040003A30713970600201A
:102F50009386C6D84146A54517050020130505CF21
:102F600002832D4559EF03C5050009476317E5089E
:102F700003A84500411106C60347180032850346E1
:102F8000080022074168518F930828FE6308170341
:102F900063E9E80005186303070523900600294547
:102FA0001DA8130648FE630BC7021518E31707FF99
:102FB00015463E87637BF602154705A83E8691C3FA
:102FC0000546B7E70400FC472390C6004206CC45FF
:102FD000418282970145B240410182801306700F01
:102FE0003E876374F6001307700FB7E70400239061
:102FF000E600FC4713160701D9BF239006000545DC
:1030000082808280416779176304E504411122C4FC
:1030100006C685472A84639FF500B7E7040022852A
:103020002244B24003A38713970500209385452DC2
:103030004101028389476399F500B7E7040083A73C
:10304000070B8545829771D9B240224441018280A5
:103050008280797122D452CC2E842A8A97750100FD
:1030600093850556177501001305455706D63AC6D0
:1030700026D24AD0B68432894ECEEF50B147A685CB
:103080001775010013058556EF50D1462945EF50BD
:10309000B14A8347840093F70702E1E783490400BC
:1030A0008947054532476396F908544083C716009F
:1030B00083C60600A207D58FC166138616FE638CF1
:1030C000C7028D16638FD7068D6693862690294595
:1030D0006391D706B7E70400A285225403A34714DF
:1030E000B250F249A6864A86925402595285624AE3
:1030F0008547456102832D450DEF9307700F3545D8
:1031000063E99702B7E70400FC4748441306700FD1
:10311000CA8582978149970700209387271F9C4380
:10312000014581CB9C4391C74E852686CA858297EF
:103130000145B250225492540259F249624A456103
:1031400082802D457DF79307700F3545E3E397FEA9
:10315000B7E70400FC4748441306700FCA858297FE
:103160005DBF2145F9B7411122C437E4040083272C
:10317000841326C2AA84416506C69705002093855C
:1031800025187D1582978327C40A170500001305AB
:10319000A5E78588829795C0032304132244B24093
:1031A000924497060020938626C54146C5451705DB
:1031B0000020130565B341010283B24022449244CA
:1031C00001454101828019C59707002023A0A7145B
:1031D00001458280454582801147636AA70A977638
:1031E00001009386A63C0A0536951841411106C692
:1031F0003697AE87B28502871307700F6145639DCE
:10320000E700B7E70400FC471306700F170500201E
:103210001305851682970145B2404101828005471A
:103220006145E39BE7FEB7E70400FC470546170549
:1032300000201305A50CF9BF1307700F6145E39D2E
:10324000E7FCB7E70400FC471306700F17050020E2
:1032500013050522C1B71307700F6145E39EE7FA16
:10326000B7E70400FC471306700F1705002013058D
:10327000A52F4DB715476145E390E7FAB7E704007E
:10328000FC471546170500201305C50761B709451A
:103290008280411126C2B7E4040083A7C41322C46C
:1032A0004AC006C62E8497050020938565052A89A5
:1032B0008297058905C5970700209387E7A283D7E2
:1032C000A70BA28503A3440D2310F4002244B240AF
:1032D00092444A850249014641010283B240224498
:1032E0009244024949454101828097070020238189
:1032F00007029707002023AF0700B717004003A776
:10330000070CB706C0FFFD16758F23A0E70C03A7B7
:10331000070DB7064000558F23A8E70C03A7070C3D
:103320003D9B23A0E70C03A7070D1367070123A804
:10333000E70C8280B717004003A5470C83A7470C12
:10334000598113451500C18B058999E31365250043
:103350009707002083C7C7FB6380A7029707002059
:103360002388A7FA11C9970700209387A7FA03A318
:103370000700630303000283828011456FE07FE052
:10338000411193962500AA852D4506C697F0FF1F8B
:10339000E7806017B240014541018280011122CCD3
:1033A00006CE3714004026CA4AC84EC652C48344CB
:1033B0007405034AB4058349840503499405EFE085
:1033C0003FB78347A40593F4F40F137AFA0F93E7FA
:1033D0001700230DF40493F9F90F1379F90FB717B8
:1033E000004003C7A705058B6DFF03D5C705A38D57
:1033F0004705238C3705A38C2705A38B9704F24040
:103400006244D2444249B249224A05618280411154
:103410009397050122C406C626C2C1872E8463DCA9
:103420000700B7E40400FC54829719C1BC5482978A
:103430002165218D3DA093F7150013C5150095E377
:1034400093F7250085C7FD35B7E70400BC4F130689
:10345000000A894517050020034545EC829713456E
:103460002400B24022449244410182809397250176
:1034700063D50702B7E4040083A7C41E8297F53D15
:10348000BC4C37F60200130606E0896517050020DC
:103490000345C5E88297096569BF93971501014502
:1034A000E3D107FC177501001305051BEF505119F7
:1034B000B7E70400BC4F13060064916517050020B0
:1034C0000345C5E582971165ADB72D71232A91108B
:1034D000FD74E98C232C811023282111232631111E
:1034E0002A84AE893289930600100A86A6852D4566
:1034F000232E111097F0FF1FE780E0001315440101
:10350000B7E70400FC4751810A0513962900CA85D4
:103510000A958297A68585660146254597F0FF1F87
:10352000E78060FE0A86A68593060010294597F07D
:10353000FF1FE78040FD8320C111032481118324F4
:103540004111032901118329C11015618280B7F748
:10355000070003C70701411106C622C426C24AC09C
:10356000A547631AF7009537B240224492440249B6
:1035700001454101828013942500AA843289A286E4
:10358000AA850146254597F0FF1FE780C0F7A28670
:103590004A86A685294597F0FF1FE780C0F6E9B760
:1035A0001D71A2CC37E404005C5C485886CE4946C5
:1035B000977501009385C505829701E9177501008C
:1035C00013054506EF50D10701A0B7F600E0795783
:1035D00098CAFD57DCCA0567B7E700E023A0E710EB
:1035E0001306F00290C223A0E7180100010037077C
:1035F000002018471306000481459706002023ADDC
:10360000E6D04157A38AE7403C44080882979717C1
:1036100000209387279E3EC8856713870740231A9B
:10362000E1001D673ACC37070105130707103ACEB2
:103630009387B7D31307B00F2310E1022312F102CF
:10364000054797F7FFFF938787592301E1023ED88B
:1036500017070000130707D397070000938747D485
:10366000B7F50700BAC23EDC17070000130767EE84
:10367000970700009387A7D081463000E1051945E0
:10368000BAC43EDE97F0FF1FE780E0E718088147E5
:10369000994630003E960346060085070507A30BB2
:1036A000C700E398D7FEC24791C70357410185671A
:1036B0006373F70001A0B7E7040083A7470A08086F
:1036C0008297AA8501C9177501001305E5F6EF5029
:1036D000616201A0F640664425618280411126C2E4
:1036E000B7E4040083A7040806C622C41705000037
:1036F000130525D2829717040020130424C2230047
:10370000A4003128DD3603450400224403A38405C8
:10371000B2409244130600328965410102837971F7
:1037200006D622D413078008F337078093F787085B
:103730003EC201000100B7170040930570052380C9
:10374000B704130680FA2380C7040100010083C672
:10375000F70293F6A60FA387D702238007049246A9
:10376000F3A60680010001007337078013778708EE
:103770003AC4010001002380B7042380C70401007C
:10378000010003C7F70213672700A387E70223801E
:103790000704A247F3A70780010001000545EFE0F9
:1037A0006FFCE13E0147814681470546854513058B
:1037B000407EEFE01F8037E404003C44680051463F
:1037C00081458297B707C0A83EC8B787E8039387AB
:1037D00007D03ECA97F7FF1F938767BD3EC67C5848
:1037E00068008297B25022544561828041119775DA
:1037F00001009385A54C17750100130525DE06C64B
:10380000EF50414F1775010013050564EF50814ECD
:10381000B240294541016F50215241119775010075
:103820009385054B17750100130545DB06C6EF5060
:10383000614C177501001305E55FEF50A14BB240D5
:10384000294541016F50414F411122C406C68347AB
:1038500005002A849DC3977501009385254D177532
:1038600001001305A5D7EF50E1484C401775010042
:103870001305C571EF5001481DA058411DE797750C
:1038800001009385A54A17750100130525D5EF5052
:103890006146177501001305E570EF50A1452244FC
:1038A000B240294541016F502149A1679386D70352
:1038B0006311D7029775010093854547177501007D
:1038C0001305C5D1EF500143177501001305856E2F
:1038D000E9B7ED0797750100938545451775010018
:1038E0001305C5CF6319F700EF50C14017750100EC
:1038F0001305856D5DB7EF50E13F4C401775010032
:103900001305856E85BF4111977501009385853D2F
:1039100017750100130585CC06C6EF50A13DB240D6
:10392000294541016F504141797122D426D24AD0B4
:103930002E842A898145B2844800714606D6EFE07C
:10394000CFC297F7FF1F9387A76ADC4783D707008B
:10395000231421012313F100EF20B0079547A3059D
:10396000F1009307401F3EC6FD572305A100230A1F
:10397000F100EF2050182686A2854800EF2050085D
:10398000B250225492540259456182809707002018
:10399000239F079A97070020238A079AB7E7040016
:1039A000BC47411106C641468145138501EE829709
:1039B000EF10D06AEF1050480145EF30401A03C7AE
:1039C000C1EF9307F00A631DF7009307F0F88945EC
:1039D0001385C1EF238EF1EEA38E01EEEF30A044EC
:1039E000EF3080548145370504009707002023AB52
:1039F00007949707002023950794970700202382B8
:103A0000079497070020239A079297070020239591
:103A10000792970700202394079297070020239589
:103A20000792EF20803C0145EF30A04697750100DA
:103A30009385C52D17750100130545BAEF50812BED
:103A40001775010013058560EF50C12AB240294562
:103A500041016F50612E411122C406C626C293F760
:103A600015002E84638D070C814617F6FF1F130681
:103A7000A6558545170500200355C58BEF80500FCF
:103A800005C5977501009385252917750100130554
:103A9000E5B4EF502126177501001305A5CAEF50B4
:103AA00061252945EF504129977501009385C52669
:103AB00017750100130585B2EF50C123177501007A
:103AC000130585C9EF5001232945EF50E12617F56D
:103AD000FF1F1305E5515C4505472390E700EFF014
:103AE000801F977501009385252317750100130525
:103AF000E5AEEF50212017750100130525C7EF50E3
:103B0000611F2945EF504123930710F8238EF1EEF2
:103B10009707002083D7C781A38EF1EE1385C1EFED
:103B2000A1839145238FF1EEA38F01EEEF30A02FFB
:103B300013451400B240224492444101828093F71D
:103B40002500D1CB17F7FF1F0357877F51C397F687
:103B5000FF1F9386267F9442977701009387075132
:103B600017F6FF1F0346E67D8145138501EEEF4002
:103B7000700DAA8431CD977501009385A520177526
:103B800001001305A5A5EF50E116A68517750100E4
:103B9000130545BFEF5001162945EF50E11997F77E
:103BA000FF1F239F0778930710F8238EF1EE97F7F6
:103BB000FF1F83D7E777A38EF1EEA183238FF1EE6A
:103BC00091458D471385C1EFA38FF1EEEF30A0250E
:103BD0001345240085B793F74500B1CF97750100D1
:103BE0009385451A177501001305459FEF50811005
:103BF000177501001305C5BAEF50C10F2945EF50E5
:103C0000A113930720F8238EF1EE97F7FF1F83D7B8
:103C1000C772A38EF1EEA183238FF1EE8547A38FA8
:103C2000F1EEEF20406D1385C1EF9145EF30A01FFD
:103C30001345440001B793F785008DCF97750100B8
:103C4000938545141775010013054599EF50810AB6
:103C500017750100130505B6EF50C1092945EF504E
:103C6000A10D97F7FF1F239D076CEF40900A1345A6
:103C70008400C9B593F70501A5C3854517F5FF1F56
:103C80000355A56BEF005154977501009385850F7F
:103C90001775010013058594EF50C10517750100D4
:103CA000130585B2EF5001052945EF50E108930750
:103CB00030F8238EF1EE97F7FF1F83D70768A38EA6
:103CC000F1EE1385C1EFA1838D45238FF1EEEF3027
:103CD000801513450401B9BD93F70502B5C3977567
:103CE00001009385250A177501001305258FEF50F4
:103CF000610017750100130565AFEF40B17F2945DD
:103D0000EF508103930740F8238EF1EE97F7FF1FE2
:103D100083D78762A38EF1EEA183238FF1EE8547CF
:103D2000A38FF1EE97F7FF1F23980760EF20A05CA9
:103D30001385C1EF9145EF30000F13450402DDBB41
:103D400093F70504CDC7977501009385A5031775F3
:103D500001001305A588EF40F179177501001305DF
:103D600065AAEF4031792945EF40117D83C7C1EF46
:103D70001307700A6388E7041307800A6386E7065F
:103D80001307600A6397E702930760F8238EF1EE4A
:103D900097F7FF1F83D7A75AA38EF1EEA183238F36
:103DA000F1EE8547A383F1F0B1451385C1EFEF3004
:103DB0008007EF2040541345040497F7FF1F23901A
:103DC00007588DBB930770F8238EF1EE97F7FF1F0E
:103DD00083D7E756A38EF1EEA183238FF1EE8547BB
:103DE000A380F1F09945D1B7930780F8F1BF93F71D
:103DF00005080145E38007D497750100938585F890
:103E0000176501001305857DEF40D16E1775010020
:103E10001305C5A0EF40116E2945EF40F1719307DE
:103E2000A0F8238EF1EE97F7FF1F83D7E751A38EFB
:103E3000F1EEA183238FF1EE8547A38FF1EE97F783
:103E4000FF1F23930750EF20004B1385C1EF9145CF
:103E5000EF20707D13450408F1B9411122C4977514
:103E600001009385E5ED2A841765010013050577A8
:103E700006C6EF4031684C40177501001305850EEA
:103E8000EF4051672945EF40316B0347040093072A
:103E9000F00F6319F70297750100938565EA1765BE
:103EA00001001305A573EF40F1644C401775010044
:103EB0001305450CEF4011642244B24029454101ED
:103EC0006F409167B24022444101828085CD41110B
:103ED00022C417650100130565702E8497750100D3
:103EE000938505E106C6EF40F160A28517750100D4
:103EF00013058513EF4011602244B240294541016A
:103F00006F4091638280411122C426C22E84AA840C
:103F100097750100938585DE176501001305056C13
:103F200006C6EF40315D177501001305A510EF407F
:103F3000715C2945EF40516097750100938505DC60
:103F400097F7FF1F2398973E176501001305056932
:103F5000854497F7FF1F239D873C97F7FF1F239A00
:103F6000973C97F7FF1F2394873EEF40B15897F592
:103F7000FF1F83D5C53D177501001305250CEF40C4
:103F800071572945EF40515B97F7FF1F2380973CFE
:103F9000EF10806A2285EF20903C0545EF20706F7E
:103FA00097F7FF1F9387C704DC4703D70700C16754
:103FB000FD176312F7022244B7E70400B2409244AF
:103FC00003A3870517F5FF1F0345C5351306000A30
:103FD000854541010283B2402244924441018280DE
:103FE000011122CC37E404005C5C06CE26CA3546BB
:103FF00097750100938585E6177501001305057E09
:10400000829701E9176501001305C561EF4051630F
:1040100001A097F7FF1F9387A7643EC4B7F5070079
:10402000856793870780814617F6FF1F1306C62F03
:10403000E10519453EC697E0FF1FE780C04C7C4470
:10404000194697F5FF1F9385252E138541E7829723
:10405000340017F6FF1F1306262D97750100938570
:10406000A535177501001305A536EF402016AA8463
:1040700015C9977501009385E5CF176501001305F4
:10408000E555EF403147A68517750100130505DE9C
:10409000EF4051462945EF40314AF2406244D24454
:1040A00005618280EFA0002D17750100130505D36F
:1040B000EF306031EF70401BEF00D13917F5FF1F73
:1040C0001305C5EFEF00B12617750100130505D2E2
:1040D000EF00113AAA84EF30100CEFC0205FEF2000
:1040E0007159EF403028EF30506BEFE0103C97757E
:1040F0000100938525C8176501001305254E89C861
:10410000EF40513FA68517750100130565D849B7E3
:10411000EF40513E177501001305C5D9EF40913DA1
:104120002945EF407141EFE0B01EEFB0E048630574
:10413000050E854537050400EF10304B97750100DB
:10414000938545C31765010013054549EF40913A32
:1041500017750100130585D7EF40D1392945EF4088
:10416000B13D97F7FF1F9387E7D883D7070017F76D
:10417000FF1F231EF71C854717F7FF1F2308F71C97
:10418000EF10C068EF10404B17F5FF1F0355251CBB
:10419000EF20F01C97F7FF1F83C7371BB9EFA3036E
:1041A000010083274417130671008545130550301D
:1041B0008297977501009385E5BB1765010013058C
:1041C000E541EF40313317750100130565D2EF402B
:1041D00071322945EF40513697750100938585B9B5
:1041E000176501001305853FEF40D13017750100B9
:1041F000130505D6EF40113071BD97750100938509
:1042000065B7176501001305653DEF40B12E1775C1
:104210000100130565D165BF97750100938585B5CC
:10422000176501001305853BEF40D12C1775010080
:104230001305C5E1EF40112C2945EF40F12F014551
:10424000EF20304551BF411122C437E404008327D9
:10425000041A06C68297EF2050198327040817F521
:10426000FFFF1305857F829797F7FF1F238CA70A0F
:1042700017F5FF1F1305C5D7EF20C0342244B24005
:104280004101B9BBB7E70400FC471171A2DDCAD9EF
:1042900086DFA6DBCED72E8432892E86AA851385AB
:1042A000C1EF82971387C1EF83470700930680020F
:1042B0009387E70793F7F70F63E4F676BA898A07DF
:1042C0001767010013078739BA979C43BA9782870B
:1042D0008D4797750100938525AC1765010013057F
:1042E000E52F630BF400EF40F12017650100130583
:1042F0006569EF403120FDA2EF40D11F1765010035
:104300001305C569EF40111F2945EF40F1229307BE
:1043100020F811469385C1EF4A85238EF1EEA38FD5
:1043200001EEEFF06FE02A840DC5977501009385CB
:10433000A5A6176501001305652AEF40B11BA285EC
:104340001765010013054569EF40D11A2945EF4073
:10435000B11E97750100938525A41765010013050B
:10436000E527EF4031191765010013052568EF4077
:1043700071182945EF40511C4165930730FA0546F5
:104380009385C1EF7D15238EF1EEEFF0EFD92A84EE
:104390000DC597750100938525A0176501001305CC
:1043A000E523EF403115A285176501001305C562AD
:1043B000EF4051142945EF403118B7E70400BC4FD6
:1043C0000566130606C8A14517F5FF1F034585F5C9
:1043D0008297FE506E54DE544E59BE591161828050
:1043E00091476301F402977501009385E59A17657B
:1043F00001001305A51EEF40F10F1765010013051D
:104400002562C5BDB7E70400FC4F914517F5FF1FB6
:10441000034545F18297977501009385E5971765E8
:1044200001001305A51BEF40F10C176501001305F2
:10443000E560EF40310C2945EF401110EF10B06BF3
:104440009145E1A285476301F402977501009385C8
:10445000A5941765010013056518EF40B1091765AC
:1044600001001305255F71B597F7FF1F239727ED0F
:10447000B7E704000566BC4F130606C8C145A9B7D7
:104480008D476301F402977501009385E5901765E8
:1044900001001305A514EF40F10517650100130590
:1044A000255D81BD930740F811469385C1EF4A858C
:1044B000238EF1EEA38F01EEEFF00FC72A84E30AFB
:1044C00005F0977501009385258D1765010013058B
:1044D000E510EF403102A285176501001305C54FB5
:1044E000EF4051012945EF403105E5B59147E31C07
:1044F000F4F8B7E70400FC4F9305000217F5FF1F1F
:10450000034545E28297977501009385E588176515
:1045100001001305A50CEF40E17D176501001305AF
:10452000A55601BF894763E187029775010093850E
:10453000A586176501001305650AEF40A17B176585
:1045400001001305A55575B383C4E1EF83C7D1EF0F
:104550009775010093854584A20417650100130532
:10456000E507DD8CEF400179A28517650100130591
:104570002554EF402178C2042945EF40E17BC184F6
:104580009305D4FF93960401C1824A8693F5F50FF3
:104590001385F1EFEF10F008E35D90E2930750F818
:1045A000238EF1EE83C7390022869385C1EF8507FC
:1045B0004A85A38FF1EEEFF02FB72A84E30B05E0D5
:1045C000976501009385457D176501001305050179
:1045D000EF404172A285177501001305E5A309B7E5
:1045E000894763E18702976501009385E57A17653E
:1045F00001001305A5FEEF40E16F176501001305EB
:10460000E54CC5B9EF10304FA2851385C1EFEF20FF
:104610009001C1B38D476301F40297650100938552
:10462000A57717650100130565FBEF40A16C1765C1
:1046300001001305654B75B9B76602000146B775F1
:104640000200054597E0FF1FE780E0EB930760F865
:10465000238EF1EEA38F01EE930700062380F1F085
:104660008947A380F1F0238101F0A38101F0C147C4
:104670002382F1F0930720F9A382F1F03146A3835E
:10468000A1F09385C1EF4A85238301F0EFF0CFA914
:104690002A84E30005D4976501009385E56F1765CB
:1046A00001001305A5F3EF40E164A2851765010041
:1046B0001305054535B5B1476301F402976501005F
:1046C0009385856D17650100130545F1EF40816203
:1046D000176501001305854429B9B7E70400FC4FAD
:1046E0009305000417F5FF1F0345C5C38297EF101C
:1046F0009040B14519BF914763E18702976501007A
:104700009385856917650100130545EDEF40815ECE
:104710001765010013054542E9BE83C401F083C754
:10472000F1EFA204DD8C8E04B77702006D14BE9405
:104730002286A6851765010013054541EF40815B80
:10474000B7E70400FC472286938511F02800829782
:1047500093160401C1823000A685094597E0FF1F2A
:10476000E78060DA2A8419C5176501001305C53F83
:10477000EF40016D930770F819469385C1EF4A85A4
:10478000238EF1EEA38081F0EFF00F9A2A84E302EA
:1047900005C4976501009385256017650100130521
:1047A000E5E3EF402155A285176501001305C53CDF
:1047B00005BB99476301F410976501009385C55DBA
:1047C00017650100130585E1EF40C152176501002F
:1047D0001305053C39BE914763E1870297650100E7
:1047E0009385855B17650100130545DFEF40815018
:1047F000176501001305453BEDBC83C401F083C779
:10480000F1EFA204DD8C8E04B77702006D14BE9424
:104810002286A685176501001305453AEF40814DB4
:10482000B7E70400FC472286938511F028008297A1
:1048300093160401C1823000A6850D4597E0FF1F45
:10484000E78060CC2A8419C5176501001305C538B7
:10485000EF40015F930780F819469385C1EF4A85C1
:10486000238EF1EEA38081F0EFF00F8C2A84E30217
:1048700005B697650100938525521765010013055C
:10488000E5D5EF402147A2851765010013050536E0
:1048900081B999476301F402976501009385C54F7B
:1048A00017650100130585D3EF40C144176501006A
:1048B000130545353DBCB7E70400FC4F93050004E4
:1048C00017F5FF1F034505A68297EF10D0229945E3
:1048D0002DBB8D476301F402976501009385C54B9D
:1048E00017650100130585CFEF40C1401765010032
:1048F0001305C532FDBA1765010013052533EF40D6
:1049000021541305C01297E0FF1FE780C0A20145A4
:10491000EFE0AFA90D45EF00F001294597E0FF1F3B
:10492000E78060A197E0FF1FE78080925DB4994720
:104930006301F40297650100938505461765010040
:104940001305C5C9EF40013B176501001305C52ECE
:104950004DB203C711F083C701F022075D8F916646
:10496000BA96C2061166C1821306F6EF8D476363DD
:10497000D60297E7FF1F9387A7679C4B03C6F1EF0B
:104980009386C70039C603D607005DCA8907E39C32
:10499000D7FE89471307A0F811469385C1EF4A85D2
:1049A000238EE1EEA38FF1EEEFE01FF82A84E302FD
:1049B00005A2976501009385253E17650100130543
:1049C000E5C1EF402133A2851765010013050528D5
:1049D00001BE03D607006302E60A8907E39BF6FEE1
:1049E0008D474DBF91476302F4029765010093859F
:1049F000A53A17650100130565BEEF40A12F1765A5
:104A00000100130525266FF0DF8EB7E70400FC4F89
:104A10009305000817F5FF1F0345C590829739BC21
:104A2000976501009385453717650100130505BBA0
:104A3000EF40412C17650100130545246FF07F8B73
:104A40002390E70017E5FF1F1305855AEFE0402A82
:104A5000976501009385453417650100130505B876
:104A6000EF4041291765010013054522EF408128D9
:104A70002945EF40612C814731BF2390070017E59E
:104A8000FF1F1305E556EFE0A0269765010093850B
:104A9000A53017650100130565B4EF40A125176522
:104AA000010013052520D9B7411122C406C683474A
:104AB00005002A849DC3976501009385A529176584
:104AC00001001305A5B1EF40E1224C40176501003C
:104AD0001305C55AEF40012275A05841B707CF0012
:104AE0009387777D6313F706976501009385852685
:104AF00017650100130585AEEF40C11F1C448356A6
:104B0000E4008355C40003C60700176501001305C0
:104B10006558EF40211E2945EF4001220357E4006C
:104B200097F7FF1F83D7A7826307F7008355C40059
:104B30000844EFE04F9B0356E4008355C40008444B
:104B40002244B24041016FF0EFF3B707CC009387E6
:104B5000777D631FF702976501009385A51F176591
:104B600001001305A5A7EF40E1181C448356E4009B
:104B70008355C40003C6070017650100130585515E
:104B8000EF4041172244B240294541016F40C11A0C
:104B9000B707CE009387777D6302F7029765010020
:104BA0009385451B17650100130545A3EF4081144C
:104BB0004C40176501001305254329BFB24022442C
:104BC00041018280B7E70400FC4741112E8606C6EA
:104BD00022C426C24AC02E842A89AA851385C1EF21
:104BE0008297976501009385E51C17650100130501
:104BF000E59EEF40211083C5C1EF17650100130545
:104C000065C3EF40210F2945EF4001139384C1EFA5
:104C100083C7040041479387070693F7F70F636143
:104C2000F74A176701001307A7AD8A07BA979C4395
:104C3000BA9782879D476303F402976501009385C5
:104C400065171765010013056599EF40A10A1765FF
:104C500001001305A5BEEF40E109F9AA83C7D1EF12
:104C6000C9C703C7F1EF83C7E1EF22075D8F83C791
:104C700001F0C2075D8F83C711F0E207D98F17E7F4
:104C8000FF1F2321F76C83C764009765010093859C
:104C90006512176501001305659417E7FF1F2302CE
:104CA000F76AEF40210597E7FF1F9387A7698C43B9
:104CB00017E6FF1F0346E668176501001305C5B92F
:104CC000EF4041032945EF402107A38E01EE224426
:104CD000B24092440249930700F8238EF1EE9D45BD
:104CE0001385C1EF41016F200014EF30300E238F88
:104CF000A1EE93578500A38FF1EE935705012A8407
:104D00002380F1F0935785010145A380F1F0EF3046
:104D1000B00C2381A1F0976501009385A509176563
:104D200001001305A58BEF30F17C03C621F0A285AD
:104D3000176501001305C5B361B7CD476301F402E0
:104D4000976501009385050717650100130505891F
:104D5000EF30517A17650100130505B3EDBD37E457
:104D600004007C4441469385D1EF138501EE829780
:104D7000138501EEEF00F022EF00100C83C7E1F085
:104D800003C7D1F0A20703238405D98F17E7FF1FBC
:104D90002318F75A1306000A89452244B240924468
:104DA000024917E5FF1F0345E557410102838D477F
:104DB0006301F402976501009385C5FF1765010043
:104DC0001305C581EF30117317650100130585BB0D
:104DD00059B503C4E1EF83C7D1EF9765010093850F
:104DE00065FD2204175501001305457F5D8CEF30EA
:104DF0007170A28517650100130585AAEF30916FC8
:104E00002945EF3071730D469385C1EF2285EFE0A0
:104E1000BFB1AA8415C9976501009385A5F91755F7
:104E200001001305A57BEF30F16CA6851765010025
:104E3000130545A8EF30116C2244B2409244024958
:104E4000294541016F30516F97E7FF1F2397874E28
:104E5000B7E70400116603A38705130606E891452A
:104E60002DBF8D476301F40297650100938585F49A
:104E70001755010013058576EF30D16717650100DE
:104E8000130505BFC9BB03C4E1EF83C7D1EF976525
:104E90000100938525F222041755010013050574BE
:104EA0005D8CEF303165A285176501001305C5A142
:104EB000EF3051642945EF3031680D469385C1EFDD
:104EC0002285EFE07FA6AA840DC197650100938536
:104ED00065EE1755010013056570EF30B161A685C9
:104EE000176501001305859FB1B797E7FF1F23954D
:104EF0008744B7E70400116603A38705130606E895
:104F00009305000259BD894763E187029765010057
:104F1000938545EA175501001305456CEF30915D07
:104F200017650100130585B73DB383C4E1EF83C75F
:104F3000D1EF976501009385E5E7A20417550100BD
:104F40001305C569DD8CEF30F15AA68517650100A0
:104F50001305459AEF30115A2945EF30F15D22864D
:104F60009385C1EF2685EFE03F9C2A8463090516EF
:104F700097650100938505E4175501001305056643
:104F8000EF305157A285176501001305E5975DB510
:104F9000854763F68714834519002244B240924442
:104FA0000249B335B00097E7FF1F2389B73817656B
:104FB00001001305A59641016F30D153A28522440B
:104FC000B24092444A8502494101C9A2994763010E
:104FD000F402976501009385E5DD1755010013057F
:104FE000E55FEF303151176501001305E5C4A5B148
:104FF00003C4E1EF83C7D1EF97650100938585DB9B
:105000002204175501001305655D5D8CEF30914E4C
:10501000A285176501001305E591EF30B14D2945D3
:10502000EF30915119469385C1EF2285EFE0DF8F74
:10503000AA840DC1976501009385C5D71755010056
:105040001305C559EF30114BA685176501001305EF
:10505000658FCDB397E7FF1F2398872EB7E704002E
:10506000116603A38705130606E89305000835B308
:105070008547976501009385E5D317550100130512
:10508000E5556309F400EF30F1461765010013059B
:10509000A58CD1B6EF301146176501001305458D7B
:1050A000EF3051452945EF3031492244B240924416
:1050B000024997E7FF1F2395072841016F3060459C
:1050C00097650100938505CF17550100130505511C
:1050D000EF30514217650100130545BAADBEB2402D
:1050E00022449244024941018280411106C622C4F1
:1050F000EFE09F839377F50F95CB2A8497650100A6
:105100009385C5CC175501001305454DEF30913EF1
:105110009375F40F17650100130505F0EF30913D0D
:105120002244B240294541016F301141B24022442E
:1051300041018280411122C491462A84138601FED6
:105140009D652D4506C697D0FF1FE780C03BB7F78A
:10515000070003C70701A5476313F70001A09306E3
:10516000001001469D65254597D0FF1FE780A039B7
:10517000238081FE2244B2409146138601FE9D6544
:105180002945410117D3FF1F6700E3375171CAD189
:1051900037E904008327C904A2D52E8686D7A6D373
:1051A0002E84AA851385C1EF829783C7C1EF1307A9
:1051B000700A638DE70C636CF7001307600A638263
:1051C000E704BE502E549E540E596D618280130721
:1051D000800A6382E7121307900AE394E7FE8D4783
:1051E000630BF41697650100938545F6175501008A
:1051F0001305C53EEF30113017650100130545F268
:1052000015A08D476306F40297650100938505F4A8
:10521000175501001305853CEF30D12D17650100AE
:10522000130545E9EF30112D2945EF30F13051BF1D
:105230008547176501001305A5E917E7FF1F230F31
:10524000F70EEF30F13FB7750200B7660200014676
:10525000054597D0FF1FE780002B930760F8238E4A
:10526000F1EEA38F01EE9307002623A0F1F0E5777E
:10527000938707212392F1F0B145238301F0A383A3
:10528000A1F01385C1EFEF10103A25BF914763E1FC
:10529000870297650100938565EB1755010013059B
:1052A000E533EF30312517650100130565E49DBF37
:1052B00083C401F083C7F1EFA204DD8C8327C90406
:1052C0006D142286938511F0280082978E04931620
:1052D0000401B7750200C1823000A695094597D038
:1052E000FF1FE7804022930770F8238EF1EE994567
:1052F000A380A1F079B7914763E187029765010028
:105300009385C5E4175501001305452DEF30911E17
:1053100017650100130545DF31B783C401F083C76A
:10532000F1EFA204DD8C8327C9046D1422869385D6
:1053300011F0280082978E0493160401B7750200BD
:10534000C1823000A6950D4597D0FF1FE780A01BB6
:10535000930780F859BF176501001305A5DDEF30ED
:10536000312E1305C01297D0FF1FE780C0FC014506
:10537000EFD0BF830D457D3B294597D0FF1FE780C8
:1053800080FB97D0FF1FE780A0EC25BD01114EC622
:1053900097E6FF1F83D6A6FBB28917E6FF1F0356C9
:1053A000E6F326CA4AC806CE22CCAA842E89252333
:1053B00097E7FF1F83C787F9B1CB03C4440083C7B6
:1053C000340017650100130565DC22045D8CEF30A5
:1053D00071124A86A6852285EFF03FD1638F0902BC
:1053E00097E7FF1F83C767F68DCB6308090297E72E
:1053F000FF1F83C7A7F495E36244F240B249CA8510
:1054000026854249D24405616F10F02117650100DD
:10541000130545D8EF30D122D1B7F2406244D244CF
:105420004249B24905618280834755008345450062
:1054300017650100130545D4A207DD8D6F30910B70
:1054400017650100130545D26F30911F8D4763F238
:10545000B70A011126CA06CE22CC0344350097E4D0
:10546000FF1F83C494EE97650100938565D3B3371E
:10547000800017E7FF1FA30AF7EC09C49765010036
:105480009385C5D2176501001305C5D2EF3091068B
:1054900097E7FF1F83C777EB63839700252C97E778
:1054A000FF1F83C797EA9DC385472306F100B7E72F
:1054B000040083A747177000854513055030829775
:1054C00017650100130505D0EF3091179967938791
:1054D00057EE2316F100680085479145A307810028
:1054E0002307F100EF103014F2406244D24405610A
:1054F00082808280894763F2B708011122CC06CEF0
:1055000026CA8344250085472A846398F40491477A
:1055100063F0B704034545008347340022055D8DE1
:1055200097E7FF1F239CA7DA1D299967938767EEEA
:105530002314F1008347340023059100A305F100F3
:1055400083474400954528002306F100EF10B00D75
:10555000F2406244D24405618280FDF899679387E6
:1055600067EE2314F10097E7FF1F83D727D7A30522
:10557000F10023050100A183F1B782800111996731
:1055800022CCD51717E4FF1F130444DC2314F100C9
:105590008347040026CA97E4FF1F938444DB230556
:1055A000F10083D7040028009545A305F100A183ED
:1055B00006CE2306F100EF10100703D60400834542
:1055C000040017650100130565C1EF30A172F240B8
:1055D0006244D244056182809D677971D917231690
:1055E000F10097E7FF1F83C767D606D62307F100B0
:1055F0009DCBB7E70400FC474146938501EE1305B8
:10560000F10082976800CD45EF10F00197E5FF1F8C
:1056100083C5C5D317650100130545BFEF30816D04
:10562000B25045618280B7E70400BC4741468145DE
:105630001305F1008297F9B7B76702036971938781
:1056400057AA3EC48967938727A02316F10097E7DE
:10565000FF1F9387A7CF83C7070023248112A307C7
:1056600001002307F10097E7FF1F938747CE83D7F9
:10567000070037E40400232611122318F10097E7EE
:10568000FF1F9387A7C583D7070041464808231902
:10569000F1007C44938501EE8297F1452800E52ACC
:1056A0002312A1027C442C002810794682973C44A6
:1056B000130561041306900D814582973010930500
:1056C000700F0145EFD05FB18320C1120324811216
:1056D00055618280B7C7A55A01119387C7333EC46D
:1056E00097E7FF1F83C777C63EC6B7F7070003C714
:1056F000070106CE22CCA5476313F70001A0116471
:10570000930504F0930600100146254597D0FF1F2E
:10571000E78060DF3000930504F0A146294597D06B
:10572000FF1FE78040DE97E5FF1F83C515C21765A1
:105730000100130565BEEF30E15BF2406244056194
:10574000828001119165A1463000938505F02D45B9
:1057500006CE97D0FF1FE78000DB2247B7C7A55AC8
:105760009387C7336312F702B2451765010013052B
:10577000E5ADB335B00097E7FF1FA388B7BCEF30A6
:105780006157F2400561828081451765010013056C
:1057900025AE97E7FF1FA38A07BAEF30A1551D3F3B
:1057A000CDB7B7C7A55A79719387F7353EC6B7E726
:1057B0000400FC47AA8506D622D4414608088297F1
:1057C000B7F7070003C70701A5476313F70001A058
:1057D0001164930504E8930600100146254597D00F
:1057E000FF1FE78040D27000930504E8D1462945A9
:1057F00097D0FF1FE78020D117650100130585B5FD
:10580000EF300164B2502254456182807971916514
:10581000D1467000938505E82D4506D697D0FF1F29
:10582000E78060CE3247B7C7A55A9387F73517652B
:1058300001001305E5AB631EF700B7E70400FC4762
:10584000138501EE41460C08829717650100130588
:1058500025A8EF30E15EB25045618280B7F70700BE
:1058600003C70701A5476313F70001A09165411124
:10587000930600100146938505E8254506C697D096
:10588000FF1FE78040C8B240176501001305459A25
:1058900041016F30E15AC16769768146FD170506FF
:1058A0001397060141836364B7003E858280330706
:1058B000D50003470700B98F214713F817008583E8
:1058C00063050800B18FC207C1837D171377F70FF7
:1058D0006DF78506F1B749C1A547054763FFB706D0
:1058E00083471500034705003168A207D98F139736
:1058F0008700A183D98FC207C1831308C855054704
:10590000639D0705411106C622C426C20344250033
:10591000914763FD8702930754006399F502A30141
:10592000C50021822302C5009304340091C6A3025E
:10593000D500A1822303D5002A84A685A93F2694F9
:105940002300A4002181A300A4000147B240224407
:1059500092443A854101828005473A858280B7C7E3
:10596000A55A01119387E7343EC42AC6B7F707004A
:1059700003C7070106CE22CC26CAA5476313F7004A
:1059800001A091642A84938504EE930600100146D9
:10599000254597D0FF1FE78000B73000A1469385CB
:1059A00004EE294597D0FF1FE780E0B5A285176573
:1059B000010013056598EF30E133EFF0FFC7F240C7
:1059C0006244D2440561828001119165A146300094
:1059D000938505EE2D4506CE97D0FF1FE780A0B238
:1059E0002247B7C7A55A9387E7346314F702B24535
:1059F000176501001305C58997E7FF1F2390B78E30
:105A0000C205C181EF30012FEFF01FC3F2400561E5
:105A10008280D147D145176501001305658917E7D5
:105A2000FF1F231DF78AEF30E12C17E5FF1F0355F9
:105A3000E58A3537E1BF011126CA06CE22CC93F79D
:105A40001500AE848DCBAD67371700409387A7AAAA
:105A50001CC3B7E70400BC4F13060019854517E5C2
:105A6000FF1F03458587829713C51400F2406244E7
:105A7000D2440561828093F72500638507129765FC
:105A80000100938525912D464800EF30411B97E595
:105A9000FF1F83C5B58B854793C4240063E1B7041A
:105AA00089CD97E7FF1F83C7478A85C385451705BB
:105AB000002013052594EF1000371395040197E794
:105AC000FF1FA3850788418155B7416505469705A6
:105AD0000020938525927D15EFF02FE1F9BF170483
:105AE0000020034424919707002083C7B790220425
:105AF0005D8CAD67C2059387B755C1816306F40815
:105B000063E68702A9679387A7556306F40897E7BA
:105B1000FF1F83C787838DE741652E867D15970517
:105B200000209385258DEFF04FDCB9A0B1679387F6
:105B3000C755630EF400B5679387D755E319F4FC96
:105B4000170500201305058BEF10E02D35A0054645
:105B5000170500201305058AEFF05F8397D7FF1F15
:105B600083C7C77E91EB4800EF30C135931505011F
:105B7000C1814800EFD02F97A2851755010013056A
:105B8000657FEF30211715BF1705002013058586A7
:105B9000EFF09F89D5B7170500201305A585EFF015
:105BA0003F8AD9BF93F745000145E38107EC1755BC
:105BB00001001305657DEF30A128EF10A03813C553
:105BC00044006DB5411122C437E404005C5C06C694
:105BD0003546975501009385652817650100130523
:105BE000E5BF829701E9175501001305657BEF308A
:105BF000212501A08327041C82972A840545EF8074
:105C0000C076EF10616AEF10A148EF70502B22852B
:105C1000B2402244410182801567B7170040130744
:105C2000575598C3D8439D66558FD8C3D843FD7642
:105C3000758FD8C3D8431367F70FD8C335671307D9
:105C4000C7CC98C3828041111305800406C622C4C4
:105C500026C297C0FF1FE780804585457D55EFC070
:105C60001FDC85457D55EFC0FFE5371400408327D5
:105C7000840A8D451305002093E707202324F40AA6
:105C8000EFC0FFD9B7E40400EFD0CF8BC858EF3096
:105C9000211B17650100130565B4EF30611A8327D6
:105CA000840C8545414593E707082324F40CEFC095
:105CB0007FE18D4513050008EFC0DFE0EFC05FFB1B
:105CC0000145EFC01FFE85450545894717D7FF1FD2
:105CD0002300F768EFC09FFE37070004B7E700E036
:105CE00023A0E710EFD0DF8BEFD05F9FE13DEFF017
:105CF0005FA5EFF07FCDEFE00FD5F5205D2083A706
:105D0000040817050000130545D3829797D7FF1F96
:105D10002385A75CBC4C1306006485458297ED3D46
:105D200097C0FF1FE780C06B01458280B7F707006F
:105D300003C70701A547AE866316F7009397450191
:105D400091C301A0AA850146254517C3FF1F67001F
:105D5000837B4111B2862E86AA852D4506C697C043
:105D6000FF1FE780407AB2400145410182809307DE
:105D7000000463E6C7021D71A2CC2A84080886CEFF
:105D800032C6EF20D16BB2461008A285294597C0D4
:105D9000FF1FE7804077F6406644256182803955D1
:105DA000828041110D658D4506C6EFC0BFD1B71782
:105DB00000408D6623A6D70C17F5FF1F13058573CA
:105DC0001387C70C9387870C1CC15CC585668967E0
:105DD0005CC958C114C518C9B7E70400B24003A391
:105DE000871E4101028382808280411126C2AE84D7
:105DF0008D4522C406C62A84EFC0DFCCB717004009
:105E000099C803A5C70C418D23A6A70CB240224414
:105E100092444101828003A5870C418D23A4A70CE5
:105E2000F5B78347050003471500A207D98FC207BE
:105E30006177C187130727206397E7008345250013
:105E4000370504005DB7828097D7FF1F938787507F
:105E500018429C4383D645000345070083C5C7000D
:105E6000035646006396A50083D5E700638DD502EF
:105E7000011106CE2386A7002397D700B705CF00D0
:105E8000DC4B9385757D05077D162EC2230001002E
:105E90003AC42316C1002317D10099C30A858297FB
:105EA000F240056182808280DC4DDC4B81CFB7E718
:105EB0000400904503A38705914517D5FF1F0345AF
:105EC000A549028382806D713C083EC6B707E50094
:105ED000232291103EC8AA843C0832852326111043
:105EE0003ECA23248110232021112E89EF20B06780
:105EF0002A84975501009385E55217450100130543
:105F0000E56DEF20315FA28517550100130585610E
:105F1000EF20515E2945EF203162B705CB00938514
:105F2000757D6800EF10C043A2856800EF205059CE
:105F3000014781467000CA852685EF10E06215C5CD
:105F40002A84975501009385E54D174501001305F7
:105F5000E568EF20315AA285175501001305455D0C
:105F6000EF2051592945EF20315D8320C1100324D2
:105F7000811083244110032901105161828097D739
:105F8000FF1F9387273D18429C43797122D406D680
:105F90000348070083C807012A8483D645000355B8
:105FA00046006396080183D82701638DD8022388B1
:105FB000070105072399D7003708CC00DC4B1308ED
:105FC000787D3ACC1307F5FF42CA23080100231E4F
:105FD000E100231FD10099C7080832C62EC482975A
:105FE0003246A2452285C535B25022544561828091
:105FF0006D713C083EC0B707E5003EC23C083EC498
:10600000232611102324811023229110231701002D
:106010002318010023190100231A0100231B01008A
:1060200097D7FF1F83D7C70099E3C167FD172316D2
:10603000F10097D7FF1F83D7C7FF91EB97D7FF1FBB
:10604000938747319C439C43DC4783D7070017D491
:10605000FF1F1304E4FD584C2317F100835744003D
:10606000484B2318F10005ED9755010093858542B3
:106070001745010013058556EF20D147175501003C
:1060800013058542EF2011472945EF20F14A83206F
:10609000C11003248110832441105161828097D75D
:1060A000FF1F83C757F989EBB7E70400BC578297F6
:1060B0005C4C23AA0700E1BFFD1797D6FF1FA38CF6
:1060C000F6F603560701834704014C470A85230B64
:1060D000F100EF20103D97D7FF1F9387A7279C4320
:1060E0000147814688430A866C00EF10E047AA8486
:1060F0001DC9975501009385E53917450100130522
:10610000E54DEF20313FA685175501001305853A6F
:10611000EF20513E2945EF203142584CB7E70400AB
:10612000BC57484B69B797D7FF1F83C7D7F0F5D740
:10613000B7E70400BC4F1044854517D5FF1F034542
:10614000A5218297A9B75C4EDC4BA9CBA1C941110F
:1061500022C417450100130565482E849755010098
:106160009385853106C6EF20F138A28517550100C9
:1061700013058536EF2011382945EF20F13BB7E7AD
:1061800004002244B24003A3870517D5FF1F03452F
:10619000A51C1306400691454101028382804111EE
:1061A00022C417D4FF1F1304A4E61C4C06C689C7DB
:1061B000DC4399C34C488297584CB7E70400BC575E
:1061C000484B82975C4CB240224423AA070041010D
:1061D000828017D7FF1F1307871083470700930696
:1061E000F00B850793F7F70F63E9F60097D6FF1FCB
:1061F0002387F60E034507008280930700F8FDB75A
:10620000835745006386070E01114AC817D9FF1F3F
:10621000130909E252C4032AC90106CE22CC03277E
:106220004A0126CA4EC656C2F15721EF1307D00DB8
:10623000FD576368C704B7E9040083A709072A84E8
:106240001305860042054181B284AE8A8297232AD3
:10625000AA000325C9015C499DEF9755010093856C
:10626000A51F1745010013056537EF20B128175505
:1062700001001305A52EEF20F1272945EF20D12B92
:10628000DD57F2406244D2444249B249224A924A1E
:106290003E850561828093874400B705CF002319AE
:1062A000F5009385757D3105EF10800B0325C9013D
:1062B000834564003105EF20B0200325C9012686FF
:1062C000D6853105EF20F01D7146A2854A85EF2065
:1062D0001117504419CA83A78905854517D5FF1F93
:1062E000034585078297814769BFEFF07FD0E5BFFF
:1062F000FD573E858280411126C297D4FF1F9384AB
:1063000024D3D84C22C437E404003C54484B06C67E
:106310008297DC4C0323C4052244B240924423AA52
:10632000070017D5FF1F034525038545410102835B
:10633000411126C297D4FF1F9384C4019C4006C616
:1063400022C44AC0C9CBDC43D9C75CC12300B50015
:106350002A84975501009385650B174501001305A5
:10636000E527EF2031192945EF20111D9C4023A47A
:10637000070023A2070097D7FF1F938767C9DC4F49
:10638000DC4B81C72955EFF09FE197D7FF1F93871B
:1063900027CADC4FDC4B91C3B93F37E904008327A0
:1063A000C905894517D5FF1F034505FB829783273C
:1063B000C905914517D5FF1F034505FA82979C40F3
:1063C00003A347016309030022852244B24092449B
:1063D000024941010283B2402244924402494101F0
:1063E00082800111328506CE22CC26CA2E84EF206F
:1063F0009017AA84975501009385850417450100DD
:106400001305C51DEF20110F030784000356640018
:1064100083554400A686175501001305E50DEF20AE
:10642000710D2945EF20511197D7FF1F83C7A7BED4
:10643000639897000145EFF09FD681450A85CD3DD1
:10644000F2406244D244056182806D712324811040
:10645000232611102322911093F745002E84638583
:1064600007123C083EC0B707E5003EC23C083EC4E8
:10647000231701002318010023190100231A01002A
:10648000231B010097D7FF1F83D787B899E3C16704
:10649000FD172316F10097D7FF1F83D787B791EB1E
:1064A00097D7FF1F938707EB9C439C43DC4783D719
:1064B000070017D7FF1F1307A7B52317F100544F85
:1064C000835747002318F100DC4A95EF97550100E8
:1064D000938545FB1745010013054510EF209101F9
:1064E00017550100130545FCEF20D1002945EF2089
:1064F000B104134544008320C11003248110832478
:1065000041105161828097D7FF1F83C7D7B02555AF
:10651000ADCBFD1717D6FF1FA30FF6AE03D60601AE
:1065200083470701CC460A85230BF100EF206077F3
:1065300097D7FF1F938707E29C4317D7FF1F1307C7
:1065400027AD976601009386A6C888430A866C002B
:10655000EF108001AA8451DD97550100938585F2E3
:106560001745010013058507EF20C178A68517554B
:106570000100130525F4EF20E1772945EF20C17BC9
:106580002685EFF0DFC1B5B793F725009DC3B7E7C8
:106590000400BC4741468145280882972555EFF005
:1065A0001FC028089305F00FEFF09FD81345240073
:1065B00099B793F7150001459DDFEFF07FA31345D1
:1065C000140015BF5C4D411106C688C317D7FF1FC5
:1065D0002322F7D8B7E7040083A7070817050000B0
:1065E0001305E5E68297B24097D7FF1F2386A7D60B
:1065F00001454101828001119307700F2316F100BC
:1066000006CE97D7FF1F83C7F7D58DE7B7E70400FE
:1066100083A7870D17D6FF1F0346C6CC6C0017D57E
:10662000FF1F035565D482973335A00097D7FF1F0E
:10663000A38AA7D2F2400561828041119397050198
:1066400022C406C626C2C1872E8463D40702B7E4DB
:106650000400FC5417D5FF1F0345C5C8829719C114
:10666000BC5482972165218DB2402244924441015D
:10667000828093F715008DC7B7E7040083A7471AF8
:1066800017D6FF1F1306C69C97F5FF1F938585EB52
:1066900017D5FF1F034505C5829713451400E9B7B9
:1066A00093F7250099CFB7E70400BC4F13060064A9
:1066B000894517D5FF1F0345E5C28297134524007E
:1066C00065B793F785009DC7B7E7040003A8871A4D
:1066D0001307401F97D7FF1F83C7C7C08146130604
:1066E0004006994517D5FF1F035505C80298134565
:1066F00084009DBF93F745000145BDD7B7E4040072
:1067000083A7041817D5FF1F035505C68297BC4CF5
:1067100013060064914517D5FF1F0345A5BC82975A
:106720001345440091B797D7FF1F83D7E7C36396FC
:10673000A70217D7FF1F231AB7C217D7FF1F2317A8
:10674000C7C217D7FF1F2314D7C22E8617550100C3
:10675000130585F6BE856F20E15917550100130515
:1067600025F76F20E16D03574500011106CE22CCBD
:1067700097D7FF1F83D747BF17550100130545F56E
:106780006310F706C167F91717D7FF1F232EF7BC51
:1067900037E4040097D7FF1F23AA07BC7C4C894528
:1067A00017D5FF1F034505B482977C4C914517D53B
:1067B000FF1F034525B3829797D7FF1F83C7F7B8FD
:1067C00095C78547A307F100832744171306F100F7
:1067D0008545130550308297175501001305C5E410
:1067E000EF200166F24062440561828097D7FF1F67
:1067F00083C7C7B5175501001305C5E7F5F38547EE
:10680000A307F100832744171306F10085451305FC
:106810005030829717550100130545E3D1B77D1518
:10682000954763E0A71A175701001307A7DC0A056D
:106830003A951C41011122CC06CE26CABA972E8465
:10684000828717550100130525E9EF20615F0DA22E
:1068500003C725009947631DF7002E85EFF0BFF0B1
:106860008345640017550100130505E8EF208148B2
:1068700097D7FF1F238B07AC17550100130585E839
:10688000E9B703C7250095476317F702C16717D714
:10689000FF1F035767ADF91703D5A5006307F7027C
:1068A000B7E7040083A7C7178297175501001305A0
:1068B00065E6EF20E158854717D7FF1F2307F7A8A4
:1068C00017550100130585E749B797D7FF1F239D8B
:1068D000A7A883D7E500B7E40400096617D7FF1F10
:1068E0002315F7A883D705011306069017D5FF1FB8
:1068F0000345459F17D7FF1F231AF7A683D7250106
:10690000A14517D7FF1F2314F7A6BC4C8297BC4C98
:1069100013060064914517D5FF1F0345A59C829778
:106920000356E4008355A400175501001305C5DF85
:10693000EF20413C49B7175501001305E5E031B799
:1069400083C525009147639AF502854717550100D5
:10695000130505E1A307F100EF20814EB7E704001E
:1069600083A747171306F10085451305503082971A
:10697000F2406244D244056182809947639EF500EB
:106980002285EFF05FDE8345640017550100130593
:10699000A5D5EF202136E9BF9547639FF5008347D2
:1069A0001400175501001305A5DBE39007EA1755FE
:1069B00001001305A5DC51BD17550100130585DC49
:1069C000C9BF82806D7123248110232611102322D8
:1069D0009110328401CD89476306F5028320C110EE
:1069E00003248110832441105161828017550100D6
:1069F000130505DAAE84EF20A144A2852685EFE0D9
:106A00006F9CE9BFB7E70400FC4728008297175541
:106A100001001305A5D8EF20A1428347810039C0AA
:106A20001307000B638EE7001387A7051377F70F93
:106A30008D4663E9E602A2852800EFE02FF579BFD5
:106A40008547E3FD87F8834591001745010013054D
:106A5000E5ECB335B00097D7FF1F2381B78EEF2049
:106A60006129ADBF03479100A207D98F356713078E
:106A7000D755638DE7066366F7022D671307B75591
:106A80006381E70631671307C7556386E704296703
:106A90001307A7556392E702A2852800EFE05F9AEB
:106AA00035BF39679306E7656383D70663E9F60068
:106AB0001307E7556388E704A285280089B73D6777
:106AC0009306F755638AD7041307F766E396E7FE44
:106AD000EFE09FB021B70146A2852800EFE01F8BB1
:106AE000F5BDA2852800EFE03F94CDBD8947E3F7CF
:106AF00087EE9305E4FFC205C1811305A100EFC035
:106B00008F9EE9BDA2852800EFE05F94C1BDA285FC
:106B10002800EFE03F9ED9B5EFE05FA6C1B5411177
:106B200022C417C4FF1F13046454AA861756010019
:106B30001306C6AD2285C14506C6EF206131035755
:106B4000440097C7FF1F938767532393E7000357BA
:106B500064002394E700B240224441018280011185
:106B600006CE22CC6D3F37E404008327841417C679
:106B7000FF1F1306A64FD54501458297832784172B
:106B80009305F1001305503082978347F100A1C7A8
:106B9000A3070100832744171306F1008545130559
:106BA000503082978327441717C6FF1F1306064DE0
:106BB000CD451305703082978547A307F1008327E1
:106BC00044171306F1008545130550308297F240B3
:106BD0006244056182808327441717C6FF1F13068E
:106BE000E649CD4513057030D5B7130101DE232CDE
:106BF000812037E4040083270408232E1120232A50
:106C00009120232821212326312117050000130577
:106C100005A3829717C9FF1F1309C96C99478544BB
:106C20002300A9002318F10097550100938505A7BB
:106C300093074006174501001305459A2314F110E8
:106C40002304910097C9FF1F93896970EF20810A7F
:106C500083D50900175501001305059CEF20810914
:106C60002945EF20610D03D509008569EFF03FEB61
:106C700083274417300085451305503082978327BA
:106C8000441717C6FF1F1306663FCD451305703026
:106C900082978327441717C6FF1F1306263CB54566
:106CA0001305603082978327441710088945130520
:106CB000103182978327441730028945130520310C
:106CC000829783274415938509C80D4582978327AA
:106CD0004415938509C811458297A30191002302A9
:106CE000910023049100232401102308010083272D
:106CF00084163002914513057040829783278416CD
:106D000013063100854513050040829783278416BA
:106D1000500085451305104082978327841610087C
:106D200085451305204082978327841630008545CA
:106D3000130550408297832704157D55829783273A
:106D400044137D5582977D55EFC0EFC18327440CD6
:106D50008297EFC02F9F8327841417C6FF1F130647
:106D6000E630D5450145829789471306700F814566
:106D700008082302F100EFA05FFF8D471306700F94
:106D8000814528022308F100EFA03FFE914723042C
:106D9000F11097C7FF1F93876755984383C7470034
:106DA0003AC42306F100EFE03F89500085450545D0
:106DB000EFC08FC210089305700F0945EFC0CFC117
:106DC00030029305700F0D45EFC00FC1300095459F
:106DD0001145EFC06FC0C16717C7FF1F1307C75822
:106DE000F9171CC32322070017C5FF1F1305454FC2
:106DF000EFC06FBD8327C41D17C5FF1F13050556C0
:106E000082973C4803450900854582978320C1212C
:106E10000324812183244121032901218329C120C5
:106E20001301012282800111C16726CA06CEAA84FD
:106E300022CC17C5FF1F03552553F9176306F50428
:106E400037E40400832784122E862315B1000147FE
:106E50008146ED4582977C440356A1002AC6A6854B
:106E600082972C0017C5FF1F03550550EFC06FC256
:106E700001CD1755010013056583EF10717C832741
:106E8000C412ED4528008297F2406244D244056165
:106E90008280011106CE22CC2DC9854717C7FF1F5E
:106EA000A303F71C97C7FF1F2380071C37E40400C8
:106EB000832784179305F100130550308297834789
:106EC000F100A9CBA3070100832744171306F100A3
:106ED00085451305503082978327441717C6FF1F37
:106EE0001306C617B5451305603082978547A3077B
:106EF000F100832744171306F10085451305503030
:106F00008297F24062440561828097C7FF1FA38C7D
:106F1000071449BF8327441717C6FF1F130606141B
:106F2000B54513056030E9BFC16717C5FF1F03559D
:106F3000A543F9176307F500B7E7040003A3C717D4
:106F40000283828001118547A307010017C7FF1F35
:106F5000230AF740B7E7040083A7471706CE1306B6
:106F6000F1008545130550308297F240056182801B
:106F7000EFA21FDB2A8408452E89B28909C900C106
:106F8000970500009385C5746105EF008101814478
:106F90007D5AEF10C00963C3A4048144EF10200A96
:106FA00063C6A40497E7FF1F9387875A9C43DC4777
:106FB000B307F94091872302F40063810904832712
:106FC000C900B307F4409587A302F4001C4C89C79D
:106FD0009C4799C3228582976FA0DFD75C441397A3
:106FE00014008504BA972390470165B71C4813978E
:106FF00014008504BA97239007004DB783278900B2
:107000000547B307F4409587A302F40083570400B3
:10701000638EE7028DC309476384E7040D47E39756
:10702000E7FA97570100938727CA1CCC97570100AE
:10703000938787CA11A897570100938767901CCC44
:10704000975701009387C7905CC849B797470100DD
:107050009387077C1CCC974701009387677CEDB72B
:1070600097570100938707CB1CCC97570100938754
:1070700067CBD9BF85E1EFA25FCC004618448347B8
:10708000940075839D8B6315F700EF00501C48C476
:107090006FA0FFCC8280EFA2BFC813893500C16406
:1070A00042094111AA890144F11413590901054A01
:1070B0002EC6EF00D077B2456346A40001454101DA
:1070C0006FA05FC983A7090013171400BA9783D76D
:1070D00007006388B7006394970063742A0105046E
:1070E000C1BF0545E9BFEFA2DFC2AA892E89328B55
:1070F000B6843A8ABE8AEF80204C55C12685EF10AF
:1071000030368D4763E5A7007D556FA01FC483DB34
:107110004400EF00D0772A84EF00B0789307740022
:1071200031443305850263C5A702EF005076EF00B6
:1071300010762A84EF00F07693077400314433050B
:10714000850263CDA702EF0090749307450019A84C
:10715000EF003075330585021307F0179307C0174A
:10716000E357A7FC2D55E3C277FB63000B02D686DD
:107170005286A6854A85EFE0106341BFEF0070722A
:10718000330585029307C5FFF1BF832749001385A7
:10719000C90083D52700EFF01FF071F9B5B7695525
:1071A000ADB797E7FF1F2397A73A97E7FF1F93878E
:1071B000273A904381470C463307F5004207418345
:1071C0006393B70082805446139847008507C296A0
:1071D0002390E600D5B797E7FF1F938767379C4357
:1071E00003C58700828017E5FF1F0355A5368280FF
:1071F000EFA2BFB4C1671387D7FF6307E5026368D7
:10720000A700F117630EF50001456FA05FB5138766
:10721000E7FF630EE500FD171D8D13351500F5B76B
:10722000EF40003D7D15D5BFEF40801AE5BFEF4030
:10723000E018CDBFEFA27FB04111AA8401442EC651
:10724000EF00F05FB2456346A400014541016FA025
:107250001FB19C48131514003E9583570500E38722
:10726000B7FE0504E9BF03485500814693F7F60FC2
:1072700063E5070181473E85828058459397560014
:10728000BA9703D727006316B70003D70700E304B4
:10729000C7FE8506E1BF8346450001479377F70F98
:1072A00063E4D700814711A81C4513165700050752
:1072B000B29703D60700E313B6FE3E858280EFA2A5
:1072C0003FA693170501C18797EAFF1F938A4A28B3
:1072D0006355F00883A70A00C0479C470357040082
:1072E000198D420541816366F500014422856FA036
:1072F0007FA612052A94DDBFDC4713944900014A9A
:107300003E94834744006341FA02014A8347540094
:107310006347FA028509C20993D9090183A70A00C4
:107320009847E3EBE9FCD1B71C4413195A00A68532
:107330003E994A85EFF01FF011ED050AD9B75C447C
:1073400013195A00A6853E994A85EFF0BFEE19E160
:10735000050A6DBFE30009FC51BFAA8481497DBFC6
:10736000EFA2BF9D1C452A8481E79307C5001CC579
:107370001C44231204001CC09307F00F63E9B700FC
:1073800093F5F50F2285EF10B0136FA05F9D9394D6
:107390000501C167C18063F7F500A6852285EF105E
:1073A000D015E5B7C18193F5F50F2285EF10501187
:1073B000A6852285EF101012C9BF97E7FF1F93879C
:1073C0002719884382801C4599C797E7FF1F23A18F
:1073D000A718014582807D55828097E7FF1F93871C
:1073E0002717984383474500484792073E95828078
:1073F000EFA2BF94617100451C183EC6B70780011B
:107400003EC81C183ECA8357440002CE02D002CCAC
:10741000231EF100834784002A8902D22301F1024E
:107420003C083ED402D6EFF05FFB835705002316DD
:10743000F102EF30706B2307A1025C40035564003A
:10744000F18313F717008347F10252055181F99B2D
:10745000D98FA307F102EFE0702639C5AA8403553E
:107460000500EF80401683D704002AD26800231C51
:10747000F10083D72400231DF1001C4803D64700E8
:107480008C43EF1010028347B400CA8617460100F0
:10749000130686318117A305F4006C004810EFE055
:1074A00090305D616FA0BF8B2155E5BF1C45B1CF0A
:1074B00003C5A700894613576500630BD7028D46A5
:1074C000630ED70285466300D702130740063305D3
:1074D000E50203C7B700418B15CB83C7B700BD8B4F
:1074E0003355F54082801375F5031307803EC5B709
:1074F00009671375F50313070771D1BF3727090013
:107500001375F5031307077CD9B701458280EFA2F5
:10751000DF8203A98500630509048347B900AE84AF
:1075200093F7070E91CF03459900930520030D8132
:107530000505B305B50288446105EFF0B0320DA032
:107540002E85EFF0BFF62A8401CD11238325C900D3
:10755000B307B54063F887002E94B305A440E1FD5E
:107560006FA0EFFF8545C1BFEFA22FFD2A8403D591
:107570000500011132C636C43AC22EC002CA02CC7E
:1075800002CEEF80400482452ACA22852ECCEFF03D
:10759000DFE403570500231EE100EF30F054A2465C
:1075A00032469247230FA10036874C08B2862285C7
:1075B0000146EFF05FB305616FA06FFAEFA2EFF73E
:1075C00061711C183EC6B70780013EC81C183ECA30
:1075D0003C0800453ED4AA8402CC02CE02D002D29E
:1075E00002D6EFF09FDF8357050035592316F102CD
:1075F000EF30904F2307A10209C48357440091E75D
:1076000021594A855D616FA08FF5035564005205CD
:107610005181EFE0B00A2A8965D58347B40093F71A
:10762000070E89C713058401EFF0502583574400E6
:10763000231EF100834784002301F1025C400355BF
:107640000900D98313F7070883471102231CA100FF
:1076500093F7F707D98FA300F10283572900231D61
:10766000F1005C40F18313F717008347F102F99BA7
:10767000D98FA307F102EF7010752AD251D1834739
:1076800094006800139757008347B400FD8BD98F8F
:10769000A305F4001C4803D647008C43EF1060603C
:1076A000A6871747010013072710740005464C10E2
:1076B0002685EFF05FA32A8929D58347B400A685E4
:1076C000FD8BA305F400EFF09FE425BFEFA2EFE6EA
:1076D000832485FE2A8441112685EFF03FDD834710
:1076E00034FF93F7070E9DC32AC62685EFF05FD0BF
:1076F00019C9834734FFB245FD8BA309F4FE81C548
:107700002285EFF0301641016FA06FE56DDD832714
:10771000C4FF2685829765F9834734FF93F7070EE8
:1077200081C72285EFF09015032584FEEFF01FE955
:10773000D9BFEFA28FDD9C4141112A8903C7070001
:1077400089472E8493566700638CF6020D46638248
:10775000C6049307F0076302F7022E85EF10A060BE
:10776000AA848149C16B130C490097E7FF1F9387D7
:1077700027DE9C43984763ECE90241016FA0AFDC30
:1077800003D745008547E3FAE7FE2E85EF108061B9
:10779000C1BF03D74500E3F2E7FE2E85EF10A05CE2
:1077A000AA842285EF10805DC204C98C5DBFDC47CE
:1077B0000355A900139A49003E9A93170501C18702
:1077C000635DF00083570A006395A70263E57403C5
:1077D0008327CA00034D5A001DA0A1672167A98F06
:1077E0001307F7EFE374F7FE63950900EFF05FA06E
:1077F00071FD85099DBF83278A00034D4A00835D83
:10780000A90003576900216A138BC7003AC6814A51
:1078100033CA4D01631E5D0197E7FF1F9387C7D3EE
:107820009C43E1DBA2866286814526858297D1B79B
:10783000A1679387F7EF930C4BFF63F04703B245C3
:107840005A85EFF05F8519CD03278B00104719CAC1
:1078500010436380C4023107D5BFEE856685EFF023
:107860007F9D71FD93861A0093FAF60F130B0B029E
:1078700055B7835644005C43E3EDF6F622853AC6DD
:10788000EF10603DA1679387D7042A8A035D440007
:10789000324763E897008347D90093E707F8A306C8
:1078A000F9001C4766852286E2858297C1670844F5
:1078B000FD17337AFA00529508C02312A40115BFB0
:1078C00097E7FF1F9387C7C89843814715C314479D
:1078D000814763FFD500939745004C47BE9519C972
:1078E00003C7550081476375E600DC451606B2976D
:1078F0003E85828003C745008147E37BE6FE16068E
:107900009C45F5B7EFA2CFC1AA892E8A814497EA98
:10791000FF1F938AEAC383A70A00984763E4E40041
:107920006FA04FC3DC471394440001493E9413BB3E
:10793000140083474400634BF900014913BB140052
:1079400083475400634FF9008504F1B70844931747
:1079500059005287DA860146A2853E95829905092B
:10796000C9BF4844931759005287DA860546A28555
:107970003E9582990509E9B7EFA22FBC814517F51D
:10798000FFFF1305255F97E7FF1F239507BCEFF067
:107990007FF76FA0CFBC97E7FF1F938767BB9C4320
:1079A00081CFEFA28FB9814517F5FFFF1305855CE5
:1079B000EFF05FF56FA0AFBA8280EFA26FB637E449
:1079C00004008327841241112315E100AE89328916
:1079D000368A3A8681460147ED45AA8482972AC6AF
:1079E00021C50356A100D285EF1061258327C4135A
:1079F000CE8526858297058915C58327440D2314D6
:107A0000210101462C00268582972A8401C9B7E707
:107A1000040083A7C712ED45280082972285410103
:107A20006FA04FB34944E5B76554CDBF5C41FD1726
:107A30005CC18280EFA26FB0B7E70400FC5F829761
:107A400095473305F50281450D816FA04FB1EFA237
:107A5000CFAEB7E70400FC5F829795473305F50288
:107A60000D816FA0CFAFEFA24FADB7E7040083A7A2
:107A7000870B0355050082976FA06FAEEFA2EFABA7
:107A8000035505003287AE8617B6FF1F03562665DD
:107A900097E5FF1F938585ACEFF03FF26FA02FAC09
:107AA000EFA2AFA9B7E7040083A7C71782976FA01B
:107AB0000FABEFA28FA8B7E7040083A7871397E562
:107AC000FF1F9385A5A9829701456FA04FA9EFA23B
:107AD000CFA6B7E7040083A7C71F814517B5FF1FCF
:107AE0000355E55B82976FA08FA7EFA20FA5B7E7BD
:107AF000040083A7871397E5FF1F938525A7829727
:107B000001456FA0CFA5EFA24FA3B7E7040083A75D
:107B1000C71F814517B5FF1F0355655E82976FA08C
:107B20000FA4EFA28FA12E85EF600055EF60900D9E
:107B30006FA0EFA2EFA26FA0EF60D0176FA02FA2EF
:107B40005C49E1175CC95CC583572501A10723196E
:107B5000F50083570501A1072318F5008280F1473E
:107B60003305F50297E7FF1F938747A29C433E9595
:107B700082808D476317F60603D74600854763F278
:107B8000E706EFA28F9B368536842E89EF10A01D65
:107B900039C18357440093140501C18063ED9702F6
:107BA0002285EF10401CFD14231294009307A002BD
:107BB000630EF5009307B0026301F502930790028C
:107BC000631BF5002285EFC0B07E31A00146CA8557
:107BD0002285EF80000F6FA08F982285EF0010594B
:107BE000DDBF828097E6FF1F9386869A9C420145FF
:107BF00099CF9843D44217E6FF1F232BE69863964C
:107C0000D70097E6FF1F23A7E6981385C7FE82805B
:107C1000EFA2AF92E9267144330585029145EF70DA
:107C2000606201E565556FA08F9397E7FF1F23AD55
:107C3000A7947526330585029145EF70A0607DD12C
:107C400097E7FF1F23A4A794592E97E7FF1F2397B9
:107C5000A792712697E7FF1F2393A79297470100EA
:107C60009387C7B917E7FF1F232EF79097070000E8
:107C7000938747ED17E7FF1F2324F790014565B76A
:107C8000EFA2AF8BAA8517E5FF1F1305258FEF1015
:107C900060216FA0CF8CEFA24F8AEFF07FFEEF1034
:107CA000E02197E7FF1F9387A78E9C4381CF13871F
:107CB000C7FE09CB83D5C7FF17E5FF1F1305C58D89
:107CC000EFF0403A6FA0AF89EFA22F87EFF09FF15E
:107CD00019C9834785002A8493F7070499E7035558
:107CE000E500EFF05FFB6FA08F878347C50093042B
:107CF000450117E9FF1F1309A98985E383270900B7
:107D00005CC997E7FF1F23A5978883274900E1FFF8
:107D100097E7FF1F23A09788F9B7FD172306F50003
:107D20006105EF60E07E8307840063CB070483472F
:107D3000840093E707F82304F400B7E704009C5F8E
:107D400082974205A94741813375F5028347840034
:107D500093F707FCC98F2304F4008347D4003E95B2
:107D60001C402318A40089CF984319CB8347C40033
:107D70005040814585073305F50242054181029750
:107D8000832709005CC897E7FF1F23A397808327F9
:107D9000490089E797D7FF1F23AE977E8347C4002A
:107DA000B9D38355040117D5FF1F1305E57EEFF006
:107DB000602B15BFEF927FF897E7FF1F938707A30C
:107DC0009C4701448583858B81EFAE84B2853A86DA
:107DD000EF1020142A8409C5EF10200B829408CCE0
:107DE00022856F90DFF7EF92BFF341112E8932C6E3
:107DF000AA89712C324713060502CA86970500002E
:107E0000938525D617D5FF1F13054577EFF09FFA09
:107E10002A8429CD9304C50065261946AA8526859E
:107E2000EF00306885452685EF0010651745010095
:107E30001305859A4E95834505002685EF00506809
:107E40005C4831468145A1075CC85CC48357240166
:107E5000E1172319F40083570401E1172318F400F4
:107E60001C4C3E85EF907FF0A30425012285410143
:107E70006F905FEEEF927FEC4111AA842EC632C460
:107E8000EF100003004DB2452246834784000CC02A
:107E900050C093F7F70393E707042304F400231873
:107EA00004002685EF00707E83479400A9462317BF
:107EB000A40013D7370005073307D7029D8B85072A
:107EC0002306F400A306E40083C70401D84885070D
:107ED000230FF7FE17D7FF1F1307876B5843232A7B
:107EE0000400930744011DEB17D7FF1F2324F76AF3
:107EF00017D7FF1F232EF76817D4FF1F1304C46979
:107F00002285EFF0A00B1C44858B5D8D09E5814532
:107F10002285EFF0201541016F907FE41CC317D735
:107F2000FF1F2329F766C9BFEF923FE197050000C5
:107F3000938565C40145EFF0DFBE01456F903FE2D8
:107F4000EF92BFDFEFF01FBF6F907FE18347C50067
:107F5000A1E7EF929FDE2A840355E500EFF05FD2A0
:107F600015C98347840093F7F7FB2304F4001C40F2
:107F700091C7DC4381C74C4001458297EFF09FC613
:107F800017D5FF1F13054561EFF0400F0355E400BF
:107F9000EFF07FD06F90BFDC8280EF921FDA97D72F
:107FA000FF1F9387E75E97050000938525D217D5BD
:107FB000FF1F1305655E23A0070023A20700EFE063
:107FC000507E6F90DFD91C4D91CBDC4381CBEF927B
:107FD000DFD68345070082976F907FD8828097D73E
:107FE000FF1F9387A75D9C4303C50700828097D737
:107FF000FF1F9387A75C9C4303C51700828097D718
:10800000FF1F9387A75B9C4303C52700828097D7F8
:10801000FF1F9387A75A9C4303C54700828097D7C9
:10802000FF1F9387A7599C4303C53700828097D7CA
:10803000FF1F9387A7589C4303C55700828097D79B
:10804000FF1F9387A7579C4303C56700828097D77C
:10805000FF1F9387A7569C4303C57700828097D75D
:10806000FF1F9387A7559C4303C58700828097D73E
:10807000FF1F9387A7549C4303C59700828097D71F
:10808000FF1F9387A7539C4303C5A700828097D700
:10809000FF1F9387A7529C4303C5B70011E11D45FD
:1080A000828097D7FF1F938767519C4303C5C70002
:1080B000828097D7FF1F938767509C4303C5D700E3
:1080C000828097D7FF1F9387674F9C4303C5E700C4
:1080D000828097D7FF1F9387674E9C4303D5070184
:1080E000828097D7FF1F9387674D9C4303C5270165
:1080F000828097D7FF1F9387674C9C4303D5470126
:10810000828097D7FF1F9387674B9C4303D56701F6
:10811000828097D7FF1F9387674A9C4303D58701C7
:10812000828097D7FF1F938767499C4303C5A701A8
:10813000828097D7FF1F938767489C4303C5B70189
:10814000828097D7FF1F938767479C4303C5C7016A
:10815000828097D7FF1F938767469C4303C5D7014B
:10816000828097D7FF1F938767459C4388578280FB
:1081700097D7FF1F938787449C4303D5C70282800C
:1081800097D7FF1F938787439C4303D5E70219E1E5
:108190001305800C828097D7FF1F938727429C434B
:1081A00003C50703828097D7FF1F938727419C430E
:1081B000C85B828097D7FF1F9387C73F8843828021
:1081C00097D7FF1F9387473F8843828019E17D55EA
:1081D0008280F5DE984265DFFDD917D7FF1F1307B0
:1081E000E7601847AA877155058B6319072203C5F5
:1081F00007001547E37DA7FC03C737001305F0050B
:108200007D171377F70FE364E5FC03C35700E30022
:1082100003FC83C86700E38C08FA03C7770049456D
:1082200079171377F70FE364E5FA03C7A70011483E
:108230001305F7FF1375F50FE36BA8F803CE97004E
:108240000D481305FEFF1375F50FE362A8F803C888
:10825000B7006309080065181378F80F1305600D5F
:10826000E36705F703C5C700794879151375F50F5E
:10827000E36FA8F403C8D7000D457D181378F80FF5
:10828000E36705F503D80701930E4017511842081C
:1082900013580801E3ED0EF303C8E7007D181378C7
:1082A000F80FE36605F303C827017D181378F80F6C
:1082B000E36F05F103C88700C54E75181378F80FF2
:1082C000E3E70EF103D86701856E938EBEE06D186B
:1082D000420813580801E3EC0EEF03D847016D186C
:1082E000420813580801E3E40EEF03D88701791818
:1082F000420813580801E36C05ED03C8A7017D1877
:108300001378F80FE36505ED03C5B7011D487D152A
:108310001375F50FE36DA8EA03C5D7017148791508
:108320001375F50FE365A8EA03D5E7011308E00F1D
:108330007D1542054181E36CA8E803C50702494861
:1083400079151375F50FE364A8E8C85301C937C858
:1083500034005915130858BFE36BA8E603A8870239
:1083600037C53400130555BF5918E36205E717D523
:10837000FF1F2323C52403C6050117D5FF1F232F85
:10838000F5220545E375C5E403D82501D0493376C8
:108390000603E31E06E203C61501E30A06E217D64A
:1083A000FF1F2329B62083C5270001466387A50048
:1083B00003C61700F1453306B60283C707039305CA
:1083C000C00272971A071307C70516031A97960873
:1083D0004697B387B70241553E973297420741838C
:1083E000636EE802EF927F953685EF60D06FEFD035
:1083F000B0212A84EF80B01D2A94EFC090252A94E2
:10840000EF7040072A94EFF0BF802A94EF2050636A
:108410002A94EF50406622956F907F948280EF926D
:10842000DF914111A307A100EF80801E9305F100A9
:1084300017050000130565B9EFF0CFCC01454101E8
:108440006F90FF91EF92FF8C17D4FF1F1304043A33
:108450000328840079599368180097D4FF1F23AB31
:10846000143913781800631E0800BA84BE89368B4D
:10847000328A2E89AA8AEFE01FD67D15269509E556
:1084800031594A856F907F8CEFE0FFD47D1526959A
:10849000A167E357F5FE97D7FF1F9387276C984393
:1084A0003E8C814B11C70145EFC0B03E933B150098
:1084B0004A85DA865686D285EF7070372A8911CDC3
:1084C0001C44F99B17D7FF1F2326F73283270C0084
:1084D000CDDBE3880BFA82976DB7268597D7FF1F10
:1084E00023A80730EFE0FFCB4146CE8517D5FF1F0D
:1084F00013054539EF00A174EFA070080325040BA4
:10850000EFA0700A0545EFA070100545EFF03FF1B0
:108510008DBF97D7FF1F9387672D9C47858BD5C746
:10852000EF92BF8117D5FF1F1305053497D7FF1FA3
:1085300023AE072A97D7FF1F23AC072A97D7FF1F21
:1085400023AA072AEFE09033EF40C002EFE0F00AE1
:10855000EFE0700F97D7FF1F9387C7279C4381C712
:108560000545EF60B03397D7FF1F938767109C4393
:1085700089C741657D15EF50A06BEFC0703AEFA041
:10858000F00097D7FF1F9387673B9C431397170112
:1085900063540700EFC0A04597D7FF1F23A4072E01
:1085A00097D7FF1F23A2072E97D7FF1F23A0072EC1
:1085B00097D7FF1F23AE072CEFF09F984923EFF0CA
:1085C000AFBBEFC080676F908FF9828097D7FF1F96
:1085D0009387C72188438280EF922FF6EF60B07EA9
:1085E000EF7080006F90AFF7EF928FF32A849304BF
:1085F000140201112E85B289A685214636C63A8914
:10860000EF0081611DE1B24638082686CE8513054C
:108610009404EF40604321462C084A85EF00C15F77
:108620001335150005616F90EFF20145E5BFEF923C
:10863000CFF09305450617D5FF1F130565F8EFE04A
:1086400070226F90CFF1EF924FEF41112EC6EFF0F5
:108650000FC0B24588C141016F906FF0EF924FECAF
:10866000AA842E84EF605078AA8985452285892DB9
:1086700083C7E4011389940899E313890403CE8521
:1086800022853D2D2146930519022285192D97D764
:10869000FF1F9387A7158C432285EF00E0682146D2
:1086A000938584022285F52B6F90CFEAEF926FE6D7
:1086B0003971EFC0E04E9305400645EDEF60D06F95
:1086C000630E051097D7FF1F83C747F113B7170035
:1086D00097D6FF1F2384E6F0014489CFC16417D9E0
:1086E000FF1F1309A9109309400EFD14EFF03F98E6
:1086F0006348A408EFF0AFB54169B7290900096ADA
:10870000FD7A2A8B81447D199389F97B130A0A71BA
:10871000938A8AC7EFF0BF9563D5A4041304400E73
:10872000B387840217D7FF1F1307470C0324070BD7
:108730003E948357C4016386270918403307EB40F2
:1087400063EAE900834744008507B3874703D69768
:108750006369F706014681450945EFF0CFE8AA8B2A
:1087600029E1EF20105A8547631FF5048965938539
:10877000057117D5FF1F1305A5E4EFE0B00EA1A802
:10878000B30734030327090BBA9703D7C70163085C
:10879000970003C75700A38207002382E700050460
:1087A000B1B79305C5002285EFF05FEB5E852286A9
:1087B0009735010093858503EFF0CFEB5E85EF00E1
:1087C000E06F850481BF97D7FF1F938727029C47DF
:1087D0008D83858BC1FF21616F902FD70146854521
:1087E000094502D002D202D402D6EFF0CFDFAA842C
:1087F0007DD1EFC0203A1389C4002A8481454A857F
:10880000C1210C4041464A85692983294400638877
:1088100009084E8502D802DA02DC02DEEF00816A26
:108820002ACE141005462C0808184ECCEF406019CB
:108830001375F50F2DE58355840093E525004A85D2
:108840006D2911460C104A85A9290146973501006A
:10885000938545FA2685EFF0EFE12685EF00006667
:108860005C40B5DB014685450D45EFF0CFD7AA84C6
:108870003DD148401389C400EF00C1642AC64A852F
:10888000C5263246636AC5004C404A85192901460F
:1088900081452685EFF00FDE26850D252DBF8355FA
:1088A000840071BFEF926FC997D7FF1F938707F4BA
:1088B0009C4719CD93E7870017D5FF1F130545D0B7
:1088C00017D7FF1F2328F7F2EFE060786F902FC9CA
:1088D000DD9B17D7FF1F232FF7F0EF2090427DF588
:1088E00017D5FF1F1305C5CDEFE04079C5B7EF924F
:1088F0004FC24169AA892E8AB28A368BBA8B8144CB
:1089000017DCFF1F130C8CEE930C400E7D19EFF05B
:108910000FF663C4A40001442DA03384940383277D
:108920000C0B3E948357C401638027055A87D68673
:108930005286CE8513050403EFF01FCB11C52380AB
:108940000B0022856F906FC08347F40191CF5A8747
:10895000D6865286CE8513059408EFF0FFC809C568
:1089600085472380FB00F1BF850455B78357450039
:10897000638D0716EF92CFBA01112A84ED2619C52F
:108980008547630AF50405616F90CFBCEFC04021B5
:108990007DF9835744004947ED9BE396E7FEC145C7
:1089A00022854524AA842285F52E0357440002CE51
:1089B00091472A896317F700228539293C082ACC78
:1089C0003ECEEFC0201D5C55DDDF74084A86A685CB
:1089D000054582974DBF03574400D147E3F5E7FAB9
:1089E000032A0400C169014997DAFF1F938A0AE04C
:1089F000130B400EFD19EFF08FE76344A90C22859D
:108A0000032A04008D26A1452A8922851D2CAA84CB
:108A10002285D92614402A86AA8978082685CA85FF
:108A2000EFF0FFECAA8425D103C7F4018947631551
:108A3000F7008347C101A1DB5546D2851385640049
:108A4000EF00E11F0145EF60103801C583D7C40175
:108A5000B1EB97D7FF1F938767D99C4793551900B0
:108A6000858913D73700058B11CB8983858B639755
:108A7000B70001452EC6EFF0FFE2B2454E85EF602C
:108A8000703C0346C1012A84937519002685EF7056
:108A9000703131C92685EF607037268511C00145D8
:108AA000EF60D061EF20F0258547E31EF5EC83C72A
:108AB00054001307F00FE388E7EC8507A382F40066
:108AC000D9B5B304690383A70A0BBE9483D7C40145
:108AD000638937015546D28513856400EF00C113C1
:108AE00071D1050909BF5DDC5DBF8280EF924FA3A4
:108AF000EF60902C11CDC164014417D9FF1F1309F9
:108B0000E9CE9309400EFD14EFF06FD6634AA4003E
:108B100017D5FF1F1305C5AAEFE060536F908FA311
:108B2000330534038327090B3E958357C5016386BC
:108B3000970023120500EF60702D0504F1B797D759
:108B4000FF1F9387A7CA9C478D83858B99EBEF9274
:108B5000CF9E17D5FF1F1305A5A6EFE020526F90FB
:108B60000FA08280EF926F9D97050000938545B41A
:108B700017D5FF1F1305C5A4EFE0A0426F902F9EED
:108B8000EF92AF9B8841B7E70400BC5B0505420547
:108B90004181829709C585472300F50005056F903F
:108BA0000F9C83C7F5FF2E858507A38FF5FE828076
:108BB00083C7F5FFFD1793F7F70FA38FF5FE99EB2A
:108BC000EF92AF97B7E70400BC571385F5FF829784
:108BD0006F90EF9882801C41035745008D8FBA95A6
:108BE0001CC12312B5003E85828093D78500A20563
:108BF0001441DD8D835745001387E6FF18C18907AF
:108C00002312F50013D685004111238FB6FEA38FE2
:108C1000C6FE4101828018419307F7FF1CC18357AC
:108C2000450085072312F500A30FB7FE8280835706
:108C300045008D8F2312F5001C41BE950CC12E8579
:108C40008280AA8703D7470008410D8FAA952392F7
:108C5000E7008CC38280184108453305A740828015
:108C600083574500035765001D8F1C410845338518
:108C7000A7403305A7408280EF922F8C41112EC66A
:108C80002A84EFF0FFFDB2456373B50001A083575E
:108C900044000840BE952312B4003E9541016F90F8
:108CA0000F8CEF928F8941112E84B28532C6EFF07E
:108CB000BFFC3246A285EFF0907841016F902F8A79
:108CC000EF92AF872E848545EFF01FFB23008500D0
:108CD0006F90EF88EF926F8641112317B10089459D
:108CE000EFF09FF98347E1002300F5008347F1008F
:108CF000A300F50041016F908F86EF920F8493D708
:108D00008500A2054111DD8D2317B1008945EFF0E3
:108D1000BFF68347E1002300F5008347F100A3007D
:108D2000F50041016F90AF83EF922F81139785017A
:108D300093D78501C166938606F0D98F13D7850036
:108D4000758FD98FA2053707FF00F98D4111DD8D91
:108D50002EC69145EFF05FF26C001146EFF0306ED9
:108D600041016F80DFFFEF825FFD1C41854503C439
:108D70000700EFF0DFEB22856F807FFEEF82FFFBC5
:108D80001C414111894503C7070083C7170023070A
:108D9000E100A307F100EFF09FE90355E100410175
:108DA0006F80FFFBEF827FF91C414111894503C7AA
:108DB000070083C717002307E100A307F100EFF0C6
:108DC0001FE78357E100410113D58700A2075D8D9E
:108DD000420541816F80BFF8EF823FF60C4141119F
:108DE0002A8411466800EFF0906591452285EFF0E6
:108DF0001FE4B247C166938606F01397870113D527
:108E00008701598D13D78700758F598DA2073707B2
:108E1000FF00F98F5D8D41016F807FF41C45BE9589
:108E20000CC18280AE87944391E6584101EF0CC19A
:108E30005CC1828003C7570013671700A382E70055
:108E4000B687D5B70CC3EDB7AA87084119CD18412D
:108E5000D44398C36313D500D8C32A870346570069
:108E60009376160081E6232007008280944381CA0E
:108E70008C4203A847008CC363930601CCC3799A44
:108E800014C3A302C7003687D1BF1C45DC471D8D24
:108E9000B777DBB6938777DB09853305F5024205A3
:108EA00041818280F147B385F50248452E95828045
:108EB0008347450085072302F5008280EF82FFE7A4
:108EC0002A8419E06F80BFE983474400E5DFFD177E
:108ED00093F7F70F2302F400F5F71C4403D727009C
:108EE00005072391E700DC4399C3228582974C480C
:108EF00089CD83475400898B99E71C4422859C4780
:108F00009C439C478297232A0400004023200400AE
:108F10004DBFEF829FE28357250041112EC691E796
:108F20000144228541016F809FE30357050081477B
:108F3000F146E307F7FEB385D702404585072E9437
:108F40008345440008C4F5F5B247AA8481E7232A83
:108F5000040009A81C456C0022859C439C43829711
:108F600048C85DDD85472312F400B2472320040082
:108F7000231804002319F4005C485CC483D7240040
:108F8000FD172391F40071BFEF823FDB97C7FF1FEE
:108F900093870765884323260500232405004105A0
:108FA000EFE0C00D6F80BFDBEF823FD917C4FF1F1A
:108FB000130404631C40411189CF9C472300B50072
:108FC0002AC65CC1EFF05FFC1C40DC4399C332450C
:108FD000829741016F80BFD8034745001DEB584D74
:108FE000AA877D550DCBEF825FD51CC3DC4797C6A2
:108FF000FF1F23A7E65EF156130507012390D70054
:109000009705000093858501EFD0B07901456F8009
:109010001FD57D5582808280EF823FD2011161464B
:1090200081452800EF807FD497C7FF1F9387475B58
:109030009C4328009305F00FDC473EC6EFF0DFF6B7
:1090400005616F80DFD197C7FF1F938767599C43E6
:10905000D847A1679387C7026312F70A397106DE02
:1090600022DC26DA80004AD84ED652D456D2328537
:10907000B284EFF05FCFAA892685EFF03FD02318A6
:10908000A4FC2685EFF09FCF2319A4FC2685EFF0E2
:10909000FFCE83D744000A8A231AA4FC858393F762
:1090A000F70F230EF4FC8607BD0793F7073F330144
:1090B000F1408A8A01498347C4FD6365F902CE8580
:1090C000130584FC232C54FDEFF01FEE5281130195
:1090D00004FCF2506254D2544259B259225A925A64
:1090E000216182802685EFF07FC993171900D697FA
:1090F00005092390A7001379F90F75BF828097C7E0
:10910000FF1F9387E74D9C43D847A1679387A7022A
:109110006310F70A397106DE22DC26DA80004AD8AD
:109120004ED652D456D23285B284EFF0DFC3AA892C
:109130002685EFF0BFC4FD572318A4FC268523190C
:10914000F4FCEFF0BFC383D744000A8A231AA4FCBF
:10915000858393F7F70F230EF4FC8607BD0793F77B
:10916000073F3301F1408A8A01498347C4FD6365A3
:10917000F902CE85130584FC232C54FDEFF0DFE2C9
:109180005281130104FCF2506254D2544259B25934
:10919000225A925A216182802685EFF03FBE9317B2
:1091A0001900D69705092390A7001379F90F75BF09
:1091B000828097C7FF1F9387A7429C43D847A16728
:1091C00089076318F708397106DE22DC26DA800089
:1091D0004AD84ED652D456D232853289EFF0BFB833
:1091E000AA894A85EFF09FB9835749000A8A231854
:1091F000A4FC858393F7F70F230CF4FC8607BD07C7
:1092000093F7073F3301F1408A8A8144834784FD05
:1092100063E5F402CE85130584FC232A54FDEFF0A8
:10922000BFD85281130104FCF2506254D254425907
:10923000B259225A925A216182804A85EFF01FB4B6
:1092400093971400D69785042390A70093F4F40F06
:1092500075BF828097C7FF1F938787389C43D84785
:10926000A1679387E7046312F70A397106DE22DCEF
:1092700026DA80004AD84ED652D456D23285B284ED
:10928000EFF07FAEAA892685EFF05FAF2318A4FC2C
:109290002685EFF0BFAE231AA4FC2685EFF01FAEA3
:1092A00083D744000A8A2319A4FC858393F7F70F18
:1092B000230EF4FC8607BD0793F7073F3301F14007
:1092C0008A8A01498347C4FD6365F902CE85130587
:1092D00084FC232C54FDEFF03FCD5281130104FC9C
:1092E000F2506254D2544259B259225A925A2161D0
:1092F00082802685EFF09FA893171900D69705095D
:109300002390A7001379F90F75BF828097C7FF1FBD
:109310009387072D9C43D847A1679387C7046310A1
:10932000F70A397106DE22DC26DA80004AD84ED6EA
:1093300052D456D23285B284EFF0FFA2AA89268594
:10934000EFF0DFA3FD572318A4FC2685231AF4FCB5
:10935000EFF0DFA283D744000A8A2319A4FC858397
:1093600093F7F70F230EF4FC8607BD0793F7073F2B
:109370003301F1408A8A01498347C4FD6365F902DC
:10938000CE85130584FC232C54FDEFF0FFC15281E0
:10939000130104FCF2506254D2544259B259225A79
:1093A000925A216182802685EFF05F9D9317190004
:1093B000D69705092390A7001379F90F75BF82800E
:1093C00097C7FF1F9387C7219C43D847A167DD0735
:1093D000631BF702EF827F96797132853284EFF05A
:1093E0009F982AC62285EFF07F992311A10222853A
:1093F000EFF07F97B2452300A1022808EFF0DFBA13
:1094000045616F80DF95828097C7FF1F9387471D57
:109410009C43D847A16793878704631BF702EF82B9
:10942000DF91797132853284EFF0FF932AC622856D
:10943000EFF0DF942311A1022285EFF0DF92B24515
:109440002300A1022808EFF03FB645616F803F91ED
:10945000828097C7FF1F9387A7189C43D847A167AF
:109460009387A704631CF700EF823F8D011128004A
:109470008145EFF07FB305616F807F8E828097C753
:10948000FF1F9387E7159C43D847A167938757022F
:109490006311F702EF827F8A01113285EFF0BF8CF2
:1094A0002308A10081452800EFF01FB005616F80FF
:1094B0001F8B828097C7FF1F938787129C43D847D3
:1094C000A1679387E702631FF702EF821F870111ED
:1094D00032853284EFF09F8AAA842285EFF01F8ABA
:1094E000854719E52285EFF01F884205B337A000B4
:1094F00028008145231891003ECAEFF0FFAA0561BC
:109500006F80FF85828097C7FF1F9387670D9C43FD
:10951000D8479947631FF704EF823F8279713285FC
:109520003284EFF05F842AC62285EFF03F85231056
:10953000A1022285EFF03F832301A1022285EFF0F3
:109540009F82A301A1022285EFF0FF812302A102E5
:109550002285EFF05F812313A1022285EFF0BF8007
:10956000B2452314A1022808EFF01FA445616F80C3
:109570000FFF828097C7FF1F938787069C43D847BA
:10958000A1679387C703631FF704EF820FFB79710D
:1095900032853284EFF02FFD2AC62285EFF00FFED0
:1095A0002310A1022285EFF06FFD2311A102228575
:1095B000EFF06FFB2302A1022285EFF0CFFAA302A6
:1095C000A1022285EFF02FFA2303A1022285EFF0FA
:1095D0008FF9B245A303A1022808EFF0FF9C456173
:1095E0006F80EFF78280EF824FF501112A84EFF050
:1095F0008FF7AA842285EFF06FF82285EFF00FF83D
:10960000035744008D4763F5E7002285EFF00FF71D
:109610002285EFF0AFF62800A685EFF0FF980561F0
:109620006F80EFF397C7FF1F938787FB9C43D84753
:10963000A167FD076319F700EF822FF03285EFF085
:109640009FFA6F80CFF1828097C7FF1F938747F9FA
:109650009C43D847A167E5076311F706EF82EFED5A
:10966000797132853284EFF00FF02AC62285EFF04F
:10967000EFF02285EFF08FF02310A1022285EFF0AA
:10968000EFEF520551812311A1022285230201022D
:10969000EFF06FEDA302A1022285EFF0CFEC2303E0
:1096A000A1022285EFF02FECB245A303A102280806
:1096B000EFF09F8F45616F808FEA828097C7FF1F11
:1096C000938707F29C43D847A1679387E703631901
:1096D000F700EF828FE63285EFF0FFF06F802FE822
:1096E000828097C7FF1F9387A7EF9C43D847A16746
:1096F000938747046314F702EF822FE47971328570
:109700003284EFF04FE62AC62285EFF02FE7B2450C
:109710002808EFF07F8945616F806FE4828097C7EA
:10972000FF1F9387E7EB9C43D847A1679387870286
:109730006316F702EF826FE0797132853284EFF0C1
:109740008FE22AC62285EFF00FE2B2452300A10284
:109750002808EFF07F8545616F806FE08280EF829F
:10976000CFDD0111EFF02FE0AA852800EFF0DF83B5
:1097700005616F80CFDE97C7FF1F938767E69C4325
:10978000D847A167D1076319F700EF820FDB328555
:10979000EFF0FFFC6F80AFDC828097C7FF1F9387DD
:1097A00027E49C43D847A167C5076319F700EF82F8
:1097B000CFD83285EFF0BFFA6F806FDA828097C71B
:1097C000FF1F9387E7E19C43D847A167B907631957
:1097D000F700EF828FD63285EFF07FF86F802FD8B9
:1097E000828097C7FF1F9387A7DF9C43D847A16755
:1097F000AD076319F700EF824FD43285EFF03FF6E3
:109800006F80EFD5828097C7FF1F938767DD9C43EA
:10981000D84789476310F702EF822FD201113285B2
:1098200032C8EFF04FD4AA852800EFF0EFF70561BA
:109830006F80EFD2828097C7FF1F938767DA9C43C0
:10984000D847A1678D076317F702EF820FCF011189
:1098500032853284EFF02FD113066100AA844C00C8
:109860002285EF20D00C2800A685EFF0EFF30561EC
:109870006F80EFCE828097C7FF1F9387A7D69C4348
:1098800081CBDC4391C7EF824FCB82976F802FCD86
:109890008280EF828FCA79713C08AE843ED2A16586
:1098A000B7070A002A843ED448103C08DD053ED69E
:1098B00036C432C63AC2EFD0BFAA12474810BA85A2
:1098C000EFF00FC032464810B285EFF0AFC0A246AD
:1098D0004810B685EFF0CFBE501001478146A685EF
:1098E0002285EFD07FC845616F806FC7EF82EFC4DC
:1098F00001117C000329C501AE843ECAA165B707EA
:1099000007002A843ECC48087C00C5053ECEEFD037
:109910003FA58345D9004808EFF08FBA50080147AA
:109920008146A6852285EFD03FC405616F802FC395
:10993000EF82AFC083C7950093F7F707A384F500C4
:10994000EFF0DFFA6F80AFC1EF822FBF79713C0873
:10995000AE843ED2A165B70709002A843ED44810E0
:109960003C08938545043ED632C636C4EFD05F9F8F
:10997000A2464810B685EFF0AFB432464810B28523
:10998000EFF04FB5501001478146A6852285EFD0F4
:10999000BFBD45616F80AFBCEF822FBA83C7950012
:1099A00041112A8493F7F707A384F50032852EC668
:1099B000EFF0CFBC85672AC4637CF500EF50B04060
:1099C0002246B24509E9114781462285EFF07FEC36
:1099D00041016F80CFB801478346F501FDB7EF82A3
:1099E0002FB401113C003ECAB7070A003ECC3C0030
:1099F0003ECE83C79500AA89328593F7F707A384E3
:109A0000F5002E84EFF08FB785676371F504A165CB
:109A1000AA84938585044808EFD09F942685EF504B
:109A2000903A2A891DE591454808EFF06FA9A6856F
:109A30004808EFF02FAACA854808EFF06FA8014741
:109A400081465008A2854E85EFD01FB205616F8018
:109A50006FB081454808EFF0AFA603490902C1BFC6
:109A6000EF820FAC79711C103ECAB7070F003ECCD5
:109A7000404D1C10AA84AE894808994532C63689E3
:109A80003ECEEFD0FF8D32464808B285EFF04FA3AF
:109A900063040902A5454808EFF00F9E2546CA85D4
:109AA000EFF0E019500801478146CE852685EFD0BA
:109AB000BFAB45616F800FAA8355C4024808EFF021
:109AC0006FA10355E402814515C185478545630FA4
:109AD000F500C167FD179305F00F6309F5007D15CB
:109AE000EF5020749305150093F5F50F4808EFF03B
:109AF0002F9D834504034808EFF08F9C8345140392
:109B00004808EFF0EF9B835524034808EFF08F9C43
:109B1000835544034808EFF0EF9B69B7EF82EFA14C
:109B200083C795008146014693F7F707A384F500A4
:109B3000EFF01FF36F80AFA2EF822FA079713E8408
:109B40001C103ECA2E89B7070F00A1653ECCFD054B
:109B50001C10AA84480842C03AC23ECE36C432C65F
:109B6000EFD01F8032464808B285EFF06F95A246CD
:109B70004808B685EFF00F9612474808BA85EFF00F
:109B80006F9502486304080291454808EFF0CF8EB4
:109B90001146A285EFF0A00A500801478146CA8508
:109BA0002685EFD07F9C45616F806F9B8945480873
:109BB000EFF08F8C834704002300F50083471400E7
:109BC000A300F500D1BFEF82AF9583C795000111C7
:109BD0002A8A93F7F707A384F5003285AE8432C64C
:109BE000EFF0CF9932462A893285EFF0CF9785671B
:109BF000637FF900AA894A85EF50F01C2A8419E98D
:109C0000114781464A86A6855285EFF09FC80561B7
:109C10006F804F949387E9FF93F7F70F0547E36849
:109C2000F7FE8347F50195E78947E382F9FE83460E
:109C3000F401528501474A86A685EFF09FC5A167CA
:109C4000D90748083ECC230A010002CEEFF0BFC27C
:109C50007DBF639CE7008947639CF9009307102050
:109C6000231FF500EF50901AD9B70947E391E7FC9D
:109C70008D47E39EF9FA2285EF50D03B97C7FF1F2F
:109C8000938747B59C4399E797C7FF1F9387479EE4
:109C90009C4389C703D50400EF60300C231F0400E8
:109CA0002285C9B7EF826F8901113C003ECAB70710
:109CB0000B003ECC3C003ECE83C795002A893285FE
:109CC00093F7F707A384F500AE84EFF02F8B93177B
:109CD0000501C187635EF004A1652A849385E502CE
:109CE0004808EFD0EFE7A2854808EFE0BFFE97C72E
:109CF000FF1F9387E7979C439DEF01449375F40FF3
:109D00004808EFE0FFFB9355844093F5F50F4808B2
:109D1000EFE01FFB9355044193F5F50F4808EFE082
:109D20003FFA014781465008A6854A85EFD0DF8378
:109D300005616F80CF82416585460546A2857D1508
:109D4000EF3070675DD95105EFD04027130440060E
:109D50003344850265B7EF725FFE0111B707060055
:109D60003EC683C7950021642A8993F7F707A38429
:109D7000F500AE8428009305A4040AC40AC8EFD0F5
:109D80002FDE300001478146A6854A85EFD0CFFD02
:109D9000EFE02FF813049404480822CC230A0100B2
:109DA00002CEEFF05FAD05616F707FFBEF725FF782
:109DB000C1642A89014497C9FF1F938929A3130A03
:109DC0008002FD14EFE0AFAB6345A40001456F7066
:109DD0007FF8B307440303A7C90ABA9703D707005C
:109DE0006306970083D72700638427010504D9BF42
:109DF0000545F1BFEF72DFF22A8A2E8999C123A0AF
:109E000005008149814497BAFF1F938AEA7D614B1F
:109E1000EFE02FAD63C5A4004E856F70BFF33384B0
:109E2000640383A70A003E948357040099E7630400
:109E30000900232089008504E1BF4146D28513052E
:109E40004400EFE0705D65F9A289F5B7EF725FED50
:109E500039717C083ED4B7070A003ED67C083ED84C
:109E600083C795002A8A328593F7F707A384F50004
:109E70002E8932C6EFE09FF085676373F5063246A0
:109E8000AA843285EFE03FEE8547AA8963EAA704FA
:109E9000A165938585042810EFD08FCC2685EF50DF
:109EA00080722A8429E191452810EFE07FE1A685A0
:109EB0002810EFE03FE2CE852810EFE07FE0014779
:109EC00081463010CA855285EFD00FEAA16793878B
:109ED000770448183EDC230A010202DEEFF0BF9946
:109EE00021616F703FE781452810EFE07FDDA68597
:109EF0002810EFE03FDE97C7FF1F9387E7C59C431D
:109F000091C7228563870900EFB0600C8345040286
:109F100065B7EFB0200BDDBFEF729FE083C7950000
:109F20004111AA8993F7F707A384F5003285AE841F
:109F3000328AEFE0BFE48567637BF5022A89EF5040
:109F400080682A84914621C18347F50105476383D0
:109F5000E70291C70D47636EF702AD462DA093054A
:109F6000050303250A004146EFE0104B1DE14101C6
:109F70006F705FDE9305950803250A004146EFE008
:109F8000B049814679F94A86A6854E85EFF0DF9B78
:109F9000F9BF83250A0013059408EF60600119C119
:109FA000C146D5B797C7FF1F9387C7829C4399E7E0
:109FB00097B7FF1F9387C76B9C4389C72285EF60C4
:109FC000A05479FD8547A30FF4002285EF80B05D92
:109FD0002285EF50A0634E8581464A86A685EFF024
:109FE000BF96A1679387570448003EC4230201002F
:109FF00002C6EFF05F88A5BFEF72BFD183C795009F
:10A000004111AA8993F7F707A384F50032852E89B9
:10A01000B28AEFE0BFD685676370F50CAA84EF5073
:10A02000805A2A841DE9416B014A97BBFF1F938B1D
:10A03000EB7B130C400E7D1B19A833048A0383A706
:10A040000B0B3E948357C401638D6703050AEFE051
:10A050000F82E344AAFE954639A88357C50163924F
:10A0600097029305050303A50A004146EFE0D03AA5
:10A07000994611E181462686CA854E85EFF0DF8C30
:10A08000A1A883A50A0013050403EF507072C1460E
:10A090007DF12285231E9400EF80F0502285EF5041
:10A0A000E05697C7FF1F938727AB9C438DCB2300B8
:10A0B00004022285EFA090614E8581462686CA85DE
:10A0C000EFF09F88A1679387070448003EC42302EE
:10A0D000010002C6EFF02FFA41016F701FC78947D8
:10A0E0002300F402D1BF397106DE22DC4AD8800099
:10A0F00052D456D25AD026DA4ED65ECE2E8A328925
:10A100002A8BEFD0DFF30605710541998A8A330166
:10A11000A140232224FC231404FCEFD05FF28347E8
:10A120009A000605350593F7F7072315A4FCA30449
:10A13000FA004A85232624FCEFE05FC4931705014B
:10A14000C1876340F0025681130104FCF25062544F
:10A15000D2544259B259225A925A025BF24B2161AF
:10A160008280AA844A85EFE07FC1AA894A85EFE010
:10A17000FFC0A1659385C5022A89130544FCEFD071
:10A180002F9E2685EFD0AF93854501C94A86CE859F
:10A19000EFD06F8DAA8B15ED8945130544FCEFE0D8
:10A1A0003FB2A685130544FCEFE0DFB2CE85130570
:10A1B00044FCEFE03FB2CA85130544FCEFE09FB1D9
:10A1C00001478146130644FCD2855A85EFD0CFB9AA
:10A1D0009DBF8145130544FCEFE09FAEA6851305A6
:10A1E00044FCEFE03FAFCE85130544FCEFE09FAEAB
:10A1F000CA85130544FCEFE0FFAD8144EFD03FE496
:10A20000E3D0A4FC83A70B0113971400BA9783D55E
:10A21000070089C5130544FCEFE0DFAB8504F9BFF7
:10A22000797106D622D44AD000184ECE52CC56CAE6
:10A2300026D25AC8AE893289AA8AEFD05FE00605D5
:10A24000690541990A8A3301A140232A24FC231C71
:10A2500004FCEFD0DFDE83C7990006052D0593F7D8
:10A26000F707231DA4FCA384F9004A85232E24FCB0
:10A27000EFE0DFB093170501C187634FF000528113
:10A28000130104FDB250225492540259F249624A19
:10A29000D24A424B45618280AA844A85EFE01FAED4
:10A2A000A1659385A5022A89130544FDEFD04F8B44
:10A2B0002685EFD0CF80854519C5CA85EFC0BFFD83
:10A2C0002A8B0DE98945130544FDEFE07F9FA685A4
:10A2D000130544FDEFE01FA0CA85130544FDEFE020
:10A2E0007F9F01478146130644FDCE855685EFD0FA
:10A2F000AFA771B78145130544FDEFE07F9CA685AC
:10A30000130544FDEFE01F9DCA85130544FDEFE0F2
:10A310007F9C8144EFD0BFD2E3D5A4FC83270B01FF
:10A3200013971400BA9783D5070089C5130544FD18
:10A33000EFE05F9A8504F9BFEF723FA083474500C5
:10A34000404DD5E7FD574DC0834694000947636DE6
:10A35000D7080346B400854663E8C6088306E400D0
:10A3600063C406085C45F9562390D70097B7FF1FD2
:10A3700083C7C72799E3A304E40097B7FF1F938718
:10A38000272F9C4381E78947A306F40097B7FF1F57
:10A390009387877C9C4381E789472306F4009705D0
:10A3A000000093854505AA8413050401EFC0703FA2
:10A3B000FD57231AF40281471CDC014897B7FF1FA1
:10A3C00023A2872297B7FF1F93870722232E040318
:10A3D00004C08043EFD0FFD061463306C5028145FB
:10A3E0002285EF709F9881473E856F705F97FD577C
:10A3F000E5BFEF729F942A8403554502EF50A01CDD
:10A4000009E5231E04006F709F958357E401E5DF83
:10A41000930504FF1715010013058577EFB010634E
:10A42000DDB7EF729F912E89A16541119385E503F8
:10A430002A8436C432C6BE843AC2EFC07FF21247C5
:10A440002285BA85EFE0DF8732462285B285EFE0CC
:10A450007F88A2462285B685EFE0DF87630D09007D
:10A4600091452285EFE05F811146A685EFE0207DD2
:10A4700041016F70DF8E89452285EFE0EFFF83C7D2
:10A4800004002300F50083C71400A300F500CDB736
:10A49000EF72BF8A83C79500444D054793F7F707CE
:10A4A000A384F5001C42411183C70700636DF704C4
:10A4B0002E842A8985CC03C7D4006309F70217B715
:10A4C000FF1F1307E71A184301CFA386F400EF809C
:10A4D000902B83C7D40089E741657D15EF30407527
:10A4E00083D72403918B99C3EFB0B0624A85A285CC
:10A4F000EFF0CFBFA167C10748003EC423020100AF
:10A5000002C6EFF04FB741016F707F85EF72FF8297
:10A5100003D745008D47AA8441112E8432892E85A8
:10A5200063EDE700EFE09F85AA85230009002685FB
:10A53000EFC07FD641016F709F82EFE03F842AC653
:10A540002285EFE0BF83B24585472A862300F900C4
:10A550002685EFC05FD1F9BF397106DE22DC26DA2D
:10A5600080004ED652D456D24AD85AD05ECEAE894A
:10A57000B284AA8AEFD0BFAB060513052502419924
:10A580000A8A3301A140232224FC231404FCEFD0C7
:10A590001FAA83C7990006054D0593F7F7072315F2
:10A5A000A4FCA384F9002685232624FCEFE00FFDFC
:10A5B00093170501C1876340F0025281130104FC27
:10A5C000F2506254D2544259B259225A925A025B02
:10A5D000F24B21618280AA8B03AB0400EFC03FCE17
:10A5E00035E983D7440001498544F11793B7170033
:10A5F000A301F4FC834734FCA165BDC79385E50442
:10A60000130544FCEFC0DFD5A685130544FCEFE03D
:10A610002FEBDE85130544FCEFE0CFEB834734FCE2
:10A62000114691E30946DA85130544FCEFE06FE734
:10A63000814463080900416B7D1BEFD05F9F63C8B5
:10A64000A40201478146130644FCCE855685EFC01F
:10A65000BFF1A5B7A685130634FCEFF03FEB9334AA
:10A6600015002A89860479B79385C50451BF8327CD
:10A67000C90013971400BA9783D507006386650154
:10A68000130544FCEFE00FE5850445BFEF726FE86A
:10A6900079711C103EC4B7070F003EC61C103EC89F
:10A6A00083C79500AA8A328593F7F707A384F5003C
:10A6B000AE893284EFE08FEC93170501C1876350B8
:10A6C000F0062A8A2285EFE06FEB2A895285032B58
:10A6D0000400EFC0DFBE39E58357440081440544E0
:10A6E000F11793B71700A303F10083457100DA87D0
:10A6F0002287CA8652862800EFF0BFD201478146E2
:10A700003000CE855685EFC03FE6A1679387D7031B
:10A7100048083ECC230A810026CEEFF0CF95456154
:10A720006F70AFE2A28513067100EFF03FDEAA84DE
:10A73000094445DD3544E30A55FB4A85EFF00FE750
:10A740000D4445D50144EFD09F8E634BA400C16BEF
:10A750000144FD1BEFD0BF8D634EA400154471B7BB
:10A76000DC4413171400BA9783D7070063812703CB
:10A770000504D1BFD84493171400BA9703D7070034
:10A7800063197701239027012685EF80C054014487
:10A79000A9BF0504C1B7EF72AFD883C795004111B7
:10A7A0002A8A93F7F707A384F50032852E8932842D
:10A7B000EFE0CFDC93170501C187635BF004AA8942
:10A7C0002285EFE0AFDB2311A1004E85832A040030
:10A7D000EFC0FFAE29E18357440085440144F117DF
:10A7E00093B71700A300F10003481100035721009D
:10A7F000D6875285CE862686CA85EFF0EFB3A1674D
:10A80000F10748003EC42302910022C6EFF0AF8654
:10A8100041016F702FD4A28513061100EFF01FCFF6
:10A820002A84894471D18357210011678544BA97DE
:10A83000C2071167C1831307F7EFE367F7FA97B70A
:10A84000FF1F938727F99C4391C785451305210076
:10A85000EF40300E8355210022858144EFC09F9D3B
:10A8600041D5231005002285EF808048B5BFEF72E7
:10A870004FCA83C7950041112A8B93F7F707A3842A
:10A88000F50032852E8A3284EFE04FCF9317050111
:10A89000C1876359F004AA8A2285EFE02FCE2A8966
:10A8A0005685832B0400EFC09FA121E1835744000C
:10A8B00081440544F11793B71700A301F100034841
:10A8C0003100DE875A854A87D6862286D285EFF008
:10A8D000AFA6A167ED0748003EC42302810026C64B
:10A8E000EFE07FF941016F704FC6A285130631007A
:10A8F000EFF0DFC1AA84094479D19167CA97C207F2
:10A900001167C1831307F7EF0544E36AF7FACA85B5
:10A91000EFC05F92014445F58149EFD04FF263DB10
:10A92000A900984893971900BA9703D7070015E72D
:10A9300023902701EFD0AFF01544E382A9F82685D4
:10A94000EF80003B97B7FF1F9387C7E89C43014404
:10A95000BDD74A85EF4040769DB785097DBFEF7230
:10A960002FBC79713E847C083EC82E8AB70714003C
:10A97000A1653ECAE5057C08AA89080836C4428953
:10A9800032C6BA8AC6843ECCEFC09F9DCA850808ED
:10A99000EFE00FB332460808B285EFE0AFB3A2464E
:10A9A000630E09029D450808EFE00FAD1D46814585
:10A9B000EF70AFBB63870A0691450808EFE0CFABA5
:10A9C0001146A685EFE0A027100801478146D285F1
:10A9D0004E85EFC07FB945616F70CFB7B685080867
:10A9E000EFE04FAF1C400808D8439355C701858955
:10A9F00012075183B205D98DEFE0CFAD1C40080896
:10AA000083C58700EFE0CFAB1C40080883C5A700D3
:10AA1000EFE00FAB1C40080883C59700EFE04FAA9A
:10AA200051BF89450808EFE02FA583C70400230024
:10AA3000F50083C71400A300F50079B7EF724FAE9D
:10AA400083C795004111AA8993F7F707A384F500FE
:10AA50003285AE843284EFE06FB293170501C1876F
:10AA60006357F0042A89032A0400EFC05F8519E9BF
:10AA7000835744000548F11793B71700A307F10067
:10AA8000814621A81306F100A285EFF03FA81DC161
:10AA90001C459DC383D6470001480347F100930737
:10AAA0008500D2884A86A6854E85EFF05FEB41018E
:10AAB0006F704FAA0948E9B71D48D9B7EF724FA682
:10AAC00065715C083EC4B7077B013EC65C083EC8A2
:10AAD00083C795002A8A328593F7F707A384F50088
:10AAE000AE89EFE04FA88357E100C5C38945280030
:10AAF000EFC01F8781452800EFE08F9CEFC0FF8BE0
:10AB000097B7FF1F938747059C4317B4FF1F034464
:10AB1000E4ADAA843334800099C31364240097B74A
:10AB2000FF1F9387E7B49C4399C31364440097B70E
:10AB3000FF1F938727CA9C4399C31364840083D55E
:10AB4000040028000149EFE0EF9883D52400280095
:10AB5000EFE04F9883D544002800EFE0AF97EFD0A7
:10AB60000FC993150501C1812800EFE0AF96A285BA
:10AB70002800EFE02F969C44636CF9000147814662
:10AB80003000CE855285EFC03F9E59616F708F9C1B
:10AB9000DC441314490028003E94EFE06F8C834797
:10ABA00044000347540089070607BA978607E36EF7
:10ABB000F5FC835524002800814AEFE0AF918345DE
:10ABC00044002800EFE0CF8F834554002800EFE0D9
:10ABD0002F8F8347440063C9FA00814A834754009A
:10ABE00063CFFA00050941BF1C4413975A0028009F
:10ABF000BA9783D50700850AEFE0CF8DD9BF032B25
:10AC0000C40093975A0028003E9B83552B00850A69
:10AC1000EFE04F8C83550B002800EFE0AF8B7DBF3A
:10AC2000EF72AF915C4993E717005CC9EF80203366
:10AC30006F70EF92EF726F902E848145EFF08F9BD3
:10AC400005C183570500FD172310F50009C483577C
:10AC500025002310F400EFF0BFFC01456F702F902A
:10AC600031456DDC23100400D5BFEF726F8B83C7B5
:10AC7000950041112A8A93F7F707A384F5003285DE
:10AC80002E893284EFE08F8F93170501C187635EB1
:10AC9000F004AA89C1452285EFD0BFFA2A8B4E85E0
:10ACA000832A0400EFC0AFE121E58357440023115C
:10ACB00001000544F11793B71700A300F100814488
:10ACC0000348110003572100D6875285CE8622867D
:10ACD000CA85EFE07FE6A1679387170248003EC46C
:10ACE0002302810026C6EFE01FB941016F708F86F5
:10ACF00013061100A285EFF07F81AA8409E52311D4
:10AD00000100094475BF930521005A85EFF09FF2B9
:10AD1000835721002A84CDD797B7FF1F938787AB2E
:10AD20009C4391C7854513052100EF408040835522
:10AD3000210026853144EFC0EFCF59D12310050003
:10AD40002685EF70F07A0144A5BFEF621FFF411125
:10AD50002E896C00AA8402C6EFF0CF8909CD035773
:10AD6000050005072310E500EFF09FEB81473E85C6
:10AD700041016F60DFFE3247954775DBCA85268546
:10AD8000EF20D008C147E34405FE324485474146E1
:10AD90002310F40083570900A685130544002311EE
:10ADA000F400EFD0D0692285C1B7EF627FF783C787
:10ADB00095004111AA8A93F7F707A384F50032851D
:10ADC000AE893284EFD09FFB93170501C187635E84
:10ADD000F0042A8AC1452285EFD0BFE6AA845285B5
:10ADE000032B0400EFC0AFCD21E5835744002311AE
:10ADF00001008544F11793B71700A300F100014447
:10AE00000348110003572100DA875685D28626862B
:10AE1000CE85EFE07FD2A1679387070248003EC44A
:10AE20002302910022C6EFE01FA541016F609FF24F
:10AE3000A28513061100EFF06FED2A8409E52311B6
:10AE40000100894475BF268593052100EFF0FFEFCF
:10AE5000AA845DF5835521002285EFC0AFBD4DF179
:10AE60000149EFD0CF9D635DA900184893171900E1
:10AE7000BA9703D707001DE7035721002390E70087
:10AE8000EFD0EF9B6302250397B7FF1F938787944B
:10AE90009C4389C703552100EF4000222285EF70B3
:10AEA0003065B9BF050975BF954499BF05C19307C2
:10AEB000F00F630FF500C547630CF5009307F5FF2E
:10AEC00005453315F50042054181828001458280A8
:10AED00041657D158280B9E1EF623FE603450603D7
:10AEE0003284EFF0BFFC9305803EB305B502C20586
:10AEF000C18191C90357E402854763F6E700130552
:10AF00000401EFC020168357E40241677D17638573
:10AF1000E700FD172317F4026F607FE48280EF6281
:10AF20005FDF004283C79500444D0349140093F747
:10AF3000F707A384F50083470400220911673369EA
:10AF4000F900A167B347F90041112A8BAE8A63EC7F
:10AF5000E70C834724001307C00EB91793F7F70FC8
:10AF60006371F70E03473400C14763ECE70C834776
:10AF700044001307E00793C707086373F70A834980
:10AF8000840083477400A209B3E9F900856763F977
:10AF9000F908034A6400834754004E85220A336A45
:10AFA000FA00EF40406245C123962403834B3400EE
:10AFB000137AFA00239A34032388740323994403F1
:10AFC00093890401631A090023A60402239804024A
:10AFD0004E85EFC0A00A1DA0034924004A85EFF06A
:10AFE000FFEC2397A402834744004E85A388F40214
:10AFF000E3810BFEE30F09FCEFC06005EF70907971
:10B0000081460146D6855A85EFE09FA5A1679387C3
:10B0100097033EC423020100480002C6EFE0BF854B
:10B0200041016F609FD28544A2862686D6855A85C7
:10B03000EFE01FA3A167938797033EC4230291000B
:10B04000E1BFBD44D5B79144C5B7EF627FCD0111D3
:10B050001C08404D3EC2B7070F003EC41C083EC648
:10B060002A89AE89EFC01F9D585C1C5C634CB70AEF
:10B070006394E50063E8A70A3385A740B3B7A70048
:10B08000B305B7401306803E81469D8DEFD0407BCF
:10B0900093140501C180A1659385C5034800EFC0E5
:10B0A0002FAC81454800EFD0BFC183550404480050
:10B0B000EFD05FC2835524044800EFD0BFC1814563
:10B0C00099C8C167FD179305F00F6386F4002685C4
:10B0D000EF402015AA854800EFD09FBE03554404D9
:10B0E000814511C9C167FD179305F00F6305F50090
:10B0F000EF402013AA854800EFD09FBC834564042D
:10B100004800EFD0FFBB834574044800EFD05FBB1D
:10B11000500001478146CE854A85EFC0EFC40561E6
:10B120006F605FC3814485BFEF623FC183C79500F5
:10B1300093F7F707A384F500EFF03FF16F603FC28C
:10B14000EF621FBE83C795004111404D93F7F7078B
:10B15000A384F5002A8A3285B284AE89EFD01FC25B
:10B160002A8B2685EFD09FC12A892685EFD0BFBFC5
:10B1700093170B0163CA0702E177CA97C207C1831D
:10B18000116763E3E70293070910C207C18313073E
:10B19000B00F637BF70093170901C187AA8A634840
:10B1A000F000C54763FA570141016F60BFBAEFC0B5
:10B1B0008F83E31B25FFF5B763060B0263040902C7
:10B1C000814463870A02B7077F00231064052311B7
:10B1D00024057CC05685EFF07FCD9304803EB304F8
:10B1E000950239A0B7077F00232004047CC0814466
:10B1F00003552404EFB0101095CCEFC0BF83269503
:10B2000093D7F44133379500AE97BA9708DC5CDCEE
:10B21000CE855285EFF07FE399E023220404A167F5
:10B220009387B70348003EC42302010002C6EFE043
:10B230008FE49DBF814701481CDC232E0403C9BF56
:10B24000EF62BFAFEFC0FFE9E1473305F50291457B
:10B25000EF30507FE55711C597A7FF1F23A6A738EA
:10B2600081473E856F60BFAF854717A7FF1F230F3C
:10B27000F7368280EF627FAC97A7FF1F93878736F0
:10B2800080432DC083570404639EA704835724047E
:10B29000639AB7043689B284EFC0CFF95C5C63C3AC
:10B2A000B7046395B7001C5C63EEA7028347640490
:10B2B00063F3F400A6872303F4048347740463F361
:10B2C0009700A687A303F4048357440441677D17BE
:10B2D0006385E70085072312F4043C4481C7CA85CF
:10B2E000268582976F60BFA797A7FF1F9387872F39
:10B2F0009C43014599C303C587008280EF62FFA389
:10B300000111B70707003EC683C79500584D0AC410
:10B3100093F7F7070AC8A384F5002A89AE8401CB06
:10B320001C4283C707002304F700EF70D045216457
:10B33000930554022800EFC0AF82EFF0FFFAAA8510
:10B340002800EFD0FF97300001478146A6854A8547
:10B35000EFC08FA113044402480822CC230A010045
:10B3600002CEEFE04FD105616F607F9FEF62FF9CDF
:10B3700001117C003ECAB70707003ECC7C003ECEE0
:10B3800083C795002E84AA8493F7F707A384F5005A
:10B39000A165938555024808EFB09FFCEFF0DFF4FC
:10B3A000AA854808EFD0DF91500801478146A28561
:10B3B0002685EFC06F9B05616F607F9A97A7FF1F7F
:10B3C000938747229C43094599C303C59700828010
:10B3D00097A7FF1F938707219C43094599C303C57E
:10B3E000D700828097A7FF1F9387C71F9C43014503
:10B3F00099C303C5A7008280EF629F920111B7072E
:10B4000008003EC683C79500404D0AC493F7F7076E
:10B410000AC8A384F5002A89AE8429C0144285474E
:10B4200003C7060063EEE706834794000946814997
:10B43000638EC700B307F740A304E400B339F000FC
:10B4400083C716002305F400EF70F033035724037D
:10B45000058B09C763840900EFA0B06B21649305D5
:10B4600084022800EFB0DFEFEFF05FF5AA85280037
:10B47000EFD01F85EFF01FF7AA852800EFD05F847B
:10B48000014781463000A6854A85EFC0EF8D130441
:10B490007402480822CC230A010002CEEFE0AFBDBF
:10B4A00005616F603F8BEF625F8901117C003ECACE
:10B4B000B70708003ECC7C003ECE83C795002E84A3
:10B4C000AA8493F7F707A384F500A1659385850205
:10B4D0004808EFB0FFE8EFF07FEEAA854808EFD00C
:10B4E0002FFEEFF03FF0AA854808EFD06FFD50081F
:10B4F00001478146A2852685EFC00F8705616F60F1
:10B500001F8697A7FF1F9387E70D9C43014599C3AB
:10B5100003C5B7008280EF625F820111B7070700A1
:10B520003EC683C79500404D0AC493F7F7070AC883
:10B53000A384F5002A89AE8405C41C42054783C74D
:10B540000700636AF7040347B400630BF700A30521
:10B55000F400EF7050238347B400A9C3EFD00FD994
:10B5600021649305B4002800EFB09FDFEFF07FF96E
:10B57000AA852800EFD0CFF4014781463000A68588
:10B580004A85EFB07FFE2904480822CC230A010037
:10B5900002CEEFE04FAE05616F606FFCEFD02FDAA7
:10B5A000C1B7EF628FF901117C003ECAB7070700EF
:10B5B0003ECC7C003ECE83C795002E84AA8493F7B0
:10B5C000F707A384F500A165AD054808EFB05FD982
:10B5D000EFF03FF3AA854808EFD08FEE50080147FF
:10B5E0008146A2852685EFB03FF805616F602FF791
:10B5F00097A7FF1F938707FF9C43094599C303C57E
:10B60000C7008280EF626FF301117C00AE843ECAF6
:10B61000A165B70707002A843ECCD1057C00480805
:10B620003ECEEFB0FFD3EFF0BFFCAA854808EFD0C5
:10B630002FE9500801478146A6852285EFB0DFF249
:10B6400005616F60CFF1EF624FEF83C7950093F70D
:10B65000F707A384F500EFF0FFFA6F604FF0EF6299
:10B660002FEC83C795000329C501411193F7F70714
:10B67000A384F5001C4283C90700854763EC3705A6
:10B6800097A7FF1F9387474D9C432E84AA8495C795
:10B69000EFF01FF689476302F50263000902834752
:10B6A000C900638C370123063901EF70D00D835731
:10B6B0002903898B99C3EFA0D0452685A285EFF099
:10B6C0007FF4A167CD0748003EC42302010002C6F3
:10B6D000EFE06F9A41016F60EFE797A7FF1F938735
:10B6E00067F09C431D4599C303C5E7008280EF6264
:10B6F000CFE40111B70707003EC683C79500584D38
:10B700000AC493F7F7070AC8A384F5002A89AE8410
:10B7100005C71C4283C7070093968701E18663C86B
:10B72000060485466385D7048346E7006386F600F2
:10B730002307F700EF70300521649305E40028002B
:10B74000EFB01FC2EFF07FF9AA852800EFD04FD7E6
:10B75000014781463000A6854A85EFB0FFE03504F9
:10B76000480822CC230A010002CEEFE0CF90056109
:10B770006F60EFDEEF626FDC01117C003ECAB7073D
:10B7800007003ECC7C003ECE83C795002E84AA8461
:10B7900093F7F707A384F500A165B9054808EFB052
:10B7A0003FBCEFF09FF3AA854808EFD06FD1500857
:10B7B00001478146A2852685EFB01FDB05616F60DA
:10B7C0000FDAEF62EFD5AA84014417A9FF1F13090E
:10B7D000A9E1E149EFC0FF906344A400014519A825
:10B7E00033053403832709003E958357250063956D
:10B7F000970011056F600FD60504E9BF032E850081
:10B8000063040E1017A3FF1F1303C3FC03230300DD
:10B81000631503002943639A060E03234E01631543
:10B8200003001D436393070EEF62AFCEC689428AC1
:10B830003E89BA8AB684328BAE8B2A84A1E903553D
:10B840004E0009E501431A856F602FD0A167A98FCB
:10B85000116763F7E700EFF0DFF68145EFF08FBD8A
:10B860000844B70700E05841F98F18455CC1B70795
:10B87000001FF98F1CC55C4981C76105EFB010003E
:10B88000E38209FC2285EF70606E6DBF3285EFA008
:10B89000E0620D434DD91C44116703D54700A167F1
:10B8A000A98F63F7E700EFF0DFF18145EFF08FB884
:10B8B0000323840093164B01D1828347B3000356C0
:10B8C00063008588FD8BA305F300FD777D8E558E83
:10B8D000FD76FD16B204F18E83274301C58E231237
:10B8E00073012313D3002304530123052301A3046D
:10B8F0004301D9D72285EFB07FBBAA850844B5DDC7
:10B900006105EFB02076ADBF1D431A858280EF62DE
:10B910002FC10569AA84AE89328A0144FD5A7D1976
:10B92000EFC0EFF06345A40001456F60AFC2D8449B
:10B9300093171400BA9703D70700631B37032390AC
:10B94000570163050A002685EF70E0389C448DC3DB
:10B9500083D76700B3F72701639C3701D28801487A
:10B96000814701478146014681452685EFF01FE961
:10B9700005047DB7EF62CFBA79711C103EC4B707DA
:10B980000F003EC61C103EC883C79500AA8A3285A8
:10B9900093F7F707A384F5002E893284EFD00FBE0A
:10B9A00093170501C1876350F006AA892285EFD05D
:10B9B000EFBC2A8A4E85032B0400EFB05F9039E577
:10B9C0008357440081440544F11793B71700A3033C
:10B9D000F10083457100DA872287D2864E862800DF
:10B9E000EFE03FA4014781463000CA855685EFB09D
:10B9F000BFB7A1679387F70348083ECC230A8100AD
:10BA000026CEEFD05FE745616F60CFB4A285130605
:10BA10007100EFE0BFAFAA84094445DD5285EFE035
:10BA2000EFB80D445DD50546D2852685EFF03FEE93
:10BA30002A8445B7EF626FB083550700034627009D
:10BA400041112A842E8532C62EC4EFE02FB611C5CF
:10BA50003246A2452285EFF09FEB41016F602FB087
:10BA6000EF622FAB83C795004111AA8A93F7F707BE
:10BA7000A384F5003285AE893284EFD02FB09317BE
:10BA80000501C1876357F008C1452A8A2285EFD096
:10BA90004F9B2A8D2285EFD06FAE2A892285EFD069
:10BAA0008FAC930705F893F7F70F1307E007AA8BFE
:10BAB0006371F7062285EFD00FAB2A8C2285EFD079
:10BAC0008FAAAA8C5285032B0400EFB04FFF29E503
:10BAD00083574400231101008144F11793B71700E5
:10BAE000A300F1000544034711008356210093870A
:10BAF00084005685DA8822885286CE85EFE03FE6BC
:10BB0000A167E90748003EC42302810026C6EFD0A2
:10BB10009FD641016F606FA313061100A285EFE06D
:10BB2000FF9EAA8409E52311010009446DBF930516
:10BB300021006A85EFF06FA12A8455F58355210015
:10BB40009356C9001316490185486688E2875E87C7
:10BB5000858A51822685EFF07FCA2A8469B7EF6211
:10BB60004F9B83C7950041112A8B93F7F707A38456
:10BB7000F5003285AE893284EFD04FA093170501CE
:10BB8000C1876352F0082A8A2285EFD02F9FAA8AA4
:10BB90002285EFD0AF9E2A892285EFD0CF9C9307D4
:10BBA00005F893F7F70F1307E0072A8C637DF70476
:10BBB0002285EFD04F9BAA8C2285EFD0CF9A2A8D79
:10BBC0005285832B0400EFB08FEF29E183574400A7
:10BBD00085440144F11793B71700A301F10003470F
:10BBE0003100930784005A85DE882688D6865286DF
:10BBF000CE85EFE0DFD68D4748003EC4230291009A
:10BC000022C6EFD05FC741016F602F94A285130653
:10BC10003100EFE0BF8F2A84894471D19356C90067
:10BC20001316490185486A88E6876287858A5182AA
:10BC3000D685EFF0BFBCAA845DB7EF626F8E2A890C
:10BC400081440144617A916A17ABFF1F130B8BB8D3
:10BC5000EFC0EFBE63C5A40022856F60AF8F83275E
:10BC6000090093991400CE9703D5070033074501C7
:10BC7000420741836362570311CD03270B0009C7B5
:10BC800085453E85EF30E04A832709000504CE97BD
:10BC90002390070085046DBFEFF0BFB28327090032
:10BCA0000504CE972390070075D58145EFE09FF8F6
:10BCB000D5B7EF62EF8683C7950041112A8A93F7C3
:10BCC000F707A384F50032852E893284EFD00F8BDD
:10BCD00093170501C1876354F004AA89832A0400DD
:10BCE000EFB0EFDD21E18357440085440144F117B3
:10BCF00093B71700A301F10003483100D68752859E
:10BD00000147CE862686CA85EFD01FE3A167F507D7
:10BD100048003EC42302910022C6EFD0DFB54101A6
:10BD20006F604F83A28513063100EFE02FFE2A8457
:10BD3000894479D197A7FF1F9387C7A99C4381CBDB
:10BD40000449EFC0CFAFAA852685EF30803E1305AA
:10BD50000401EFF09FEE2285EF609079814469BF86
:10BD6000EF523FFB83C795004111AA8A93F7F7076B
:10BD7000A384F5003285AE89328423110100EFC01F
:10BD8000FFFF93170501C187635CF0042A8AC14550
:10BD90002285EFC01FEBAA8B5285032B0400EFB066
:10BDA0000FD231E18357440085440144F11793B722
:10BDB0001700A300F1000348110003572100DA87A0
:10BDC0005685D2862686CE85EFD01FD7A16793876A
:10BDD000270248003EC42302910022C6EFD0BFA92B
:10BDE00041016F509FF6A28513061100EFE00FF29C
:10BDF0002A84894469D197A7FF1F9387A79D9843F9
:10BE00003E8901CB0449EFC08FA3AA852685EF3078
:10BE1000403213050401EFF05FE2EFC04FA29544FA
:10BE200059D9930521005E85EFE03FF2AA8441F5E0
:10BE30001C480357210022852390E700EF60506BD8
:10BE400083270900ADDB03552100EF30E026A5B7BD
:10BE5000EF523FEC83C795004111AA8A93F7F70789
:10BE6000A384F5003285AE893284EFC03FF1931789
:10BE70000501C1876359F0042A8A2285EFC01FF0AB
:10BE80002A895285032B0400EFB06FC321E1835749
:10BE9000440085440144F11793B71700A301F10052
:10BEA00003483100DA8756854A87D2862686CE85B2
:10BEB000EFD09FC8A167F90748003EC42302910054
:10BEC00022C6EFD05F9B41016F503FE8A285130669
:10BED0003100EFE0AFE32A84894479D19167CA97B2
:10BEE000C2071167C1831307F7EF8544E36AF7FAC6
:10BEF00097A7FF1F9387078E9843BE8B01CB0449FA
:10BF0000EFC0EF93AA852685EF30A0221305040128
:10BF1000EFF0BFD2EFC0AF92954459D11C482285B3
:10BF2000814423902701EF60B05C83A70B00ADDB59
:10BF30004A85EF306018ADB7EF523FE02A844105E3
:10BF4000B284EFF09FCF01C52285EF60705A814621
:10BF50000146A6852285EF70C00B1C4C89C7DC47C3
:10BF600099C3228582976F509FDF9797FF1F938712
:10BF700067679C43014599C31385070182809797A2
:10BF8000FF1F9387276688438280EF521FDB93173A
:10BF9000C600DD8DC2054111C1812A8432C6EFC0C1
:10BFA0007FD33246228511829375F60FEFC05FD1A1
:10BFB00041016F50DFDAEF52BFD679713C083ED2B3
:10BFC000B7070C003ED43C083ED683C79500AE842C
:10BFD0002A8993F7F707A384F500A16593853504B3
:10BFE0004810EFB0EFB7C165FD150144179AFF1F68
:10BFF000130ACA7F930A400EAE892E8B2EC6EFC05D
:10C000000F874205931704014181C183B24563E361
:10C01000A702C167FD176385F5004810EFC09FCBED
:10C02000501001478146A6854A85EFB0EFD34561A0
:10C030006F505FD23307540383270A0BBA9703D696
:10C04000C70163083601638835014810EFF0FFF33C
:10C05000DA85050465B7B285EDBFEF529FCB7971E4
:10C060007C083EC8B70711003ECA7C083ECC83C797
:10C070009500AA89328593F7F707A384F5002E89E6
:10C08000EFC0DFCF8567637EF502A165AA848905CD
:10C090000808EFB0EFAC2685EF30E05213341500FE
:10C0A0000A04A2850808EFC0BFC1A6850808EFC032
:10C0B0007FC235C0014781461008CA854E85EFB062
:10C0C000AFCA45616F507FC8B30754030327CA0A3C
:10C0D000BA9703D70700631A970003D62700638A2D
:10C0E00065030808EFF07FEADE8505042EC6EFB091
:10C0F0001FF94205931704014181C183B245E3E56D
:10C10000A7FCC167FD17E387F5FA0808EFC09FBCDD
:10C1100055B7B285D9BFC165FD150144179AFF1FF8
:10C12000130ACA6C930A80022E8BAE8BC1B7EF52F2
:10C13000DFC018418347170083460700A207D58F49
:10C14000D207D1832390F5008347270003471700C8
:10C150008D45A207D98F91832310F600EFC03FAD24
:10C160006F50FFBFEF52DFBBC16401441799FF1F3F
:10C170001309C96793098002FD14EFB05FF06345AE
:10C18000A40001456F501FBD330534038327C90A3E
:10C190003E9583570500E38797FE0504F9BFEF52EC
:10C1A0003FB82A8AAE89B284B68AEF30C04109E529
:10C1B00091473E856F501FBA2A894E85EF901050E7
:10C1C0002A84638A0A048D476DD503570500C54745
:10C1D000E31147FF0347F9018546AD47E31BD7FC51
:10C1E0008347450091CB4146A6855D05EFC0D0222F
:10C1F000814761D1AD4775BF130965012302E50091
:10C20000CA852685EF10202D15CDA547E3830AFAB0
:10C210002302040079BF11CD83570500E39A47F943
:10C220004146A6851905EFC0301F814759D199476E
:10C2300049B74E85EFF01FF32A8495473DD913097E
:10C2400055007DBF4146A6852310440123113401CA
:10C2500013051900EFC0B01E2285EF60B03C814786
:10C2600089BFEF529FAD79717C003ECCB7070A00C1
:10C270003ECE7C003ED083C79500B2842E8493F7D7
:10C28000F707A384F5001306A1002A892C00268550
:10C29000EFF0FFE9A16528088D05EFB06F8C9040A5
:10C2A0008355A100035581008546EFF05FEFAA8416
:10C2B000AA852808EFC0DFA00356A100835581009E
:10C2C0002808EFF09FCC300801478146A2854A85B7
:10C2D000EFB08FA9854748103ED42302910202D6C1
:10C2E000EFD06FD945616F509FA7EF521FA57971AD
:10C2F0007C003ECCB7070A003ECE7C003ED083C710
:10C300009500B2842E8493F7F707A384F5001306F3
:10C31000A1002A892C002685EFF07FE1A16528087D
:10C320008D05EFB0EF8390408355A1000355810048
:10C330008146EFF0DFE6AA84AA852808EFC05F985F
:10C340000356A100835581002808EFF01FC4300870
:10C3500001478146A2854A85EFB00FA1481023020C
:10C36000910202D402D6EFD00FD145616F503F9FAA
:10C37000EF52BF9CEFF0BFE26F507F9E9797FF1F79
:10C380009387872688438280EF523F9B83572500FF
:10C390004111AE842A842307B10017F5FFFF13056E
:10C3A000A5696C002316F100EFB0CFD581C42285BA
:10C3B000EF60B02DFD572310F400130620028145D5
:10C3C00013055400EF507F9A41016F505F99EF526F
:10C3D0003F9579717C003ECCB7070A003ECE7C00C9
:10C3E0003ED083C79500AA89AE8493F7F7073285BC
:10C3F000A384F5001306A1002C00EFF05FD30355D2
:10C4000081001144EF30201C15C10355A1000144E7
:10C41000EF90D02A01CD0357050083578100454492
:10C420006316F7008545EFF03FF601442169930557
:10C4300039002808EFA0DFF2A2852808EFC05F8846
:10C440000356A100835581002808EFF01FB430087F
:10C4500001478146A6854E85EFB00F9148104AD41A
:10C460002302810202D6EFD00FC145616F509F8E2B
:10C47000EF521F8B9797FF1F9387C7162A84884315
:10C480002E8915C1035745038357C401631DF70067
:10C4900023260502231805024105EFA0303E630460
:10C4A0000900EF60302F81449799FF1F9389093469
:10C4B000130A8002EFB0BFBC63CCA4029797FF1FA2
:10C4C0009387071B9C4389C70355C401EF1040762F
:10C4D000630509002285EF6050031306400E814575
:10C4E0002285EF509F88FD57231EF4006F509F86D2
:10C4F0003385440383A7C90A3E9503570500835734
:10C50000C4016315F700CA85EFF01FE885045DB725
:10C51000EF521F8183C795004111AA8993F7F7074E
:10C52000A384F5003285AE84EFC05F8585676370B4
:10C53000F5042A89EF302009014411C983D704008A
:10C540003144638627018545EFF09FF201444E8513
:10C55000A2864A86A685EFD02FBFA16793871704CE
:10C5600048003EC42302810002C6EFD0CFB0410193
:10C570006F504FFEEF52CFFA9797FF1F93878706B2
:10C5800080431DCC0145EFA0E05681470148C164BE
:10C590001CDC232E0403232004041799FF1F130916
:10C5A000E92401449309400EFD14EFB05FAC634BE6
:10C5B000A40081451705000013054598EFB08FB41E
:10C5C0006F504FF9330534038327090B3E9583578A
:10C5D000C501638597008545EFF09FE90504F1B734
:10C5E0009357050113D78700A380F5009317050122
:10C5F000C183A1832380E5002381F500A381A500E9
:10C600008280EF528FF32300050083C71500A3003B
:10C61000F50083C725002301F50083C73500A3017A
:10C62000F50083C745002302F50083C75500A30228
:10C63000F50083C7650093059500A3030500230358
:10C64000F500230405003285EFF09FF96F502FF1BC
:10C65000EF520FED4111E9541DC995C993F9C5FF7A
:10C660002E842A89AA84338AA900B7EA04006314B5
:10C670009A020D88854401CCB7E704009C5F82973D
:10C680002AC622866C0033053901EFC0405B26853F
:10C6900041016F502FEC83A78A039104829793176F
:10C6A0000501C183A183A38EF4FE93570501238F57
:10C6B000F4FEA183238EA4FEA38FF4FE4DBF63E09E
:10C6C000D502EF528FE7B28741113686BE8536C656
:10C6D000EFC0E056B246410136856F504FE88146C3
:10C6E00036858280838705001387F5003D05FD8729
:10C6F00093F77708834607007D158606B58FA3005C
:10C70000F5006307B7007D17834717009D83DDB7EA
:10C710008280EF528FE2B7E7040083A707093287D0
:10C720002A863A858297133515006F504FE301CD65
:10C73000814799C9EF526FE04146EFC040508547AD
:10C740003E856F50CFE181473E8582801DC5EF5207
:10C75000CFDE414681452A84EF502FE14146814595
:10C7600013050403EF506FE00147C167232204045F
:10C7700038C87CC805456F508FDE014582808147EF
:10C7800029CDA1CDEF526FDBB2842E89130680052F
:10C7900081452A84EF506FDDCA8524C42685EFF0D9
:10C7A0001FF9414681452285EF502FDC3044A28598
:10C7B0002285EFF01FF693040401A2852685EFF091
:10C7C0007FF2A68513050402EFF0DFF12285EFF07A
:10C7D000FFF785473E856F508FD83E858280EF52A8
:10C7E0002FD44111E9541DC995C993F9C5FF2E8471
:10C7F0002A89AA84338AA900B7EA0400639444030F
:10C800000D88814401CCB7E704009C5F82972AC65B
:10C8100022866C0033053901EFC060422685410154
:10C820006F504FD383A78A03910482979317050112
:10C83000C183A183A38EF4FE93570501238FF4FED9
:10C84000A183238EA4FEA38FF4FE4DBF71CDEF52C2
:10C850002FCDB28401E605456F50CFCF2A842E89B3
:10C860000145FDD93C487848B3E6E700F5D6938604
:10C87000F7FFB3B7F6007D17032A4404BA9734C80C
:10C880007CC8630F0A04C14913050A03B3894941EF
:10C890002295637B3601B2862E86A685EFF03FE2B5
:10C8A0007C40BE9464C045BFCE862E86CE85EFF018
:10C8B0001FE1C114D2944E9923220404A287930647
:10C8C000040103C7070003C607038507318FA38F41
:10C8D000E7FEE398F6FE3044A2852285EFF07FE381
:10C8E0002699C1493306994063EA9900ADD4A686DA
:10C8F000A68513050403EFF09FDC6DB78147B306EF
:10C90000F4003307F6000347070083C506008507D8
:10C910002D8F2380E600E39437FF3044A2852285E3
:10C92000EFF03FDFC1147DBF0145828019C9EF528E
:10C93000CFC0130680058145EF502FC305456F50CA
:10C940000FC20145828081473DC9B5C9EF52EFBE94
:10C95000FC4141462E84AA846393C70413860501D3
:10C96000A2878146C14503C7070003C507038507A2
:10C97000298F3305D600034505008506298FA38F2F
:10C98000E7FEE392B6FE3044A2852685EFF07FD81D
:10C990002285EFF0BFF985473E856F504FBC138568
:10C9A00007031D8E81452295EF502FBC7C40130755
:10C9B00000F813060402A2972388E70255B73E85C4
:10C9C0008280EF528FB76D712E84B284AA85901049
:10C9D00028003689EFF0BFDA19E9D55705A0504095
:10C9E0000C402800EFF09FE66DD9FD142104E5F816
:10C9F0002C004A85EFF03FF5814765D13E855161B6
:10CA00006F50EFB5EF526FB341112EC432C62C00F8
:10CA10000546EFF01FFB41016F506FB4EF52EFB1CD
:10CA200001112A842EC602C802CA02CC02CEEFC06F
:10CA30006049B2462A86A2850808EFF0BFFC13754C
:10CA4000F50F05616F50AFB1EF522FAF7971B2871B
:10CA50002A8421462308B10013051101BE853AC47A
:10CA600036C6EFC0C01DB246930591013685EFF082
:10CA70003FB72285141035460C08EFF0BFF82A8422
:10CA8000224711E521460C103A85EFC0401B228554
:10CA900045616F50CFACEF524FAA7171AE84AA8539
:10CAA0000A853284EFF0BFC801C90A86A6852285AF
:10CAB000EFF03FC6814711E1C5473E854D616F509C
:10CAC0000FAAEF528FA41D712A8AB289BE843546FF
:10CAD0008547130511012E8CB68A3A8BC28C468D80
:10CAE0002308F100EFC0A01510100C085285231F79
:10CAF0000100EFF05FFA2A842DE9A147631BFD06D0
:10CB00009307900591E0E5473546E285130511014D
:10CB100013990A012308F10013590901EFC02012EB
:10CB20001357890093978A00D98F90080C08528573
:10CB3000231FF100EFF03FF62A8405E9A1E0938777
:10CB4000FA0091831379F9003EC663130900414945
:10CB5000668B8144C14B854DB2476397970C6A86BB
:10CB60008C0033855C01EFC0800D228525616F50FC
:10CB70008F9D93079004C9F8A54779B783470105AE
:10CB80000947C14B2308F10083471105A58FA3086E
:10CB9000F10093872400814463EFFB0201471408EE
:10CBA0003386E6008C08B386E400BA95DA9683C62D
:10CBB000060083C505000507AD8E2300D600E3906F
:10CBC000E7FE41476398E70490080C085285EFF0B0
:10CBD0009FEC35D535A8B3069B00BA871008B3057E
:10CBE000F60090083E9603C506000346060085073A
:10CBF0008506298E2380C500E39277FF998F9008E0
:10CC00000C085285BE94EFF01FE98947014749D5CA
:10CC10002A84A1BF90083E96034606001408BE96DB
:10CC20002380C600850779BFB2478504638B9712BE
:10CC300081471808B306F70098083E973386F90035
:10CC400003470700034606008507318F2380E6006F
:10CC5000E39177FF90080C085285EFF0DFE34DF980
:10CC60003546E285130511012308B101EFB0307D8F
:10CC7000139704014183939784002183D98F10185F
:10CC80000C085285231FF100EFF0FFE051F18147BE
:10CC900010183387F9003E96034707000346060045
:10CCA000B306FB008507318F2380E600E39277FF10
:10CCB00075A01808B306F70098083E973386F90068
:10CCC00003470700034606008507318F2380E600EF
:10CCD000E3E127FFCA876398770990080C0852851B
:10CCE000EFF07FDB15F581479800B306F700900859
:10CCF00018103E973E960347070003460600850737
:10CD0000318F2380E600E39177FF3546E2851305F6
:10CD100011012308B101EFB0907213970401418310
:10CD2000939784002183D98F10180C085285231FF4
:10CD3000F100EFF05FD6E31D05EC81471018338753
:10CD4000F9003E960347070003460600B306FB00C2
:10CD50008507318F2380E600E3E227FFC109410BFD
:10CD6000E5BB8147B5B79408BE9683C60600180890
:10CD70003E972300D7008507B9BF638E062CEF428C
:10CD8000DFF859712A84BE89B28B85473546130571
:10CD900011022E8B468C4289BA8A368A2300F10210
:10CDA000EFB0F06910180C10228523170102EFF084
:10CDB0009FCE631E0510A1476319FC0693079005DB
:10CDC00063930900E5473546DA851305110293148C
:10CDD0000A012300F102C180EFB0706693178A0048
:10CDE00013D78400D98F90080C1022852317F102E5
:10CDF000EFF07FCA69ED639009049307FA00BD88DC
:10CE0000918391E0C144C207C183DE8C814A3EC652
:10CE1000414DB24763EAFA0C6286B3854B01881034
:10CE2000EFB0905F4DC53D555DA093079004E39C26
:10CE300009F8A54749BF834701050947C14C2300AD
:10CE4000F10283471105B3C7F900A300F1029387EC
:10CE50002900814963EFFC02814618103306D70090
:10CE60008C083387D900B69556970347070083C5CA
:10CE7000050085062D8F2300E600E390D7FE41478D
:10CE8000639AE70490080C102285EFF0DFC035D5D7
:10CE90003DA8B3863A01BA871010B305F600900892
:10CEA0003E9603C506000346060085078506298EC3
:10CEB0002380C500E39297FF3387EC4090080C1065
:10CEC0002285BA99EFF03FBD8947014741D5656199
:10CED0006F407FE790083E96034606001410BE960A
:10CEE0002380C600850769BFB247850A93990A0166
:10CEF000939D8A0093D909016399570D854735465B
:10CF0000DA85130511022300F10293D98900EFB0ED
:10CF10001053B3ED3D0190000C1022852317B1038F
:10CF2000EFF07FB74DF58147A68963E69706268621
:10CF30000C084A85EFB0B05081471810B306F700CF
:10CF4000100898083E973E960347070003460600E0
:10CF50008507318F2380E600E3E197FE639DA905F5
:10CF600090080C102285EFF01FB335F1814798101F
:10CF7000B306F700900818183E973E96034707003F
:10CF8000034606008507318F2380E600E391A7FF63
:10CF90004109C10CBDBD18089000B306F7003E96CC
:10CFA0003387FC0003470700034606008507318FDF
:10CFB0002380E60095BF98084E97034707001C1092
:10CFC000CE972380E700850951BF85473546DA852E
:10CFD000130511022300F10293D98900EFB0304606
:10CFE000B3ED3D0190000C1022852317B103EFF043
:10CFF0009FAAE31E05EC814718089000B306F700CE
:10D000003E963387FC00034707000346060085076A
:10D01000318F2380E600E391A7FF41460C084A8543
:10D02000EFB0F04181471810B306F70010089808D8
:10D030003E973E9603470700034606008507318F5B
:10D040002380E600E391A7FF90080C102285EFF003
:10D050009FA41DDDADBD7D558280EF421FCE011125
:10D060002A842E8593055100328902C002C202C46F
:10D0700002C693047400EFF0AFD61D46A6851305D3
:10D080009100EFB0D03B10088A854A85EFF0BFA031
:10D0900019ED93071400180883C60700034607001C
:10D0A00085070507B18EA38FD7FEE397F4FE0561D0
:10D0B0006F40FFCAEF42DFC62E848C414111AA891E
:10D0C000838715003289914463D30700A144979761
:10D0D000FF1F938767A89C43B1C3B5CE8D4723102C
:10D0E000F10083C725004A852301F10083C735007D
:10D0F000A301F10083C745002302F10083C7550057
:10D10000A302F10083C7650093059100A30301000A
:10D110002303F10023040100EFF08FCC0C404A867A
:10D120000A85EFF00FCE0328040083564400A6883A
:10D130001D0881470147E51642868A854E85EFF036
:10D140005F982A8909E5A6852285EFB0FFB24A8556
:10D1500041016F403FC04A860A85EFF08FCA7DBF0C
:10D16000EF421FBC2E848C414111AA898387150090
:10D170003289914463D30700A1449797FF1F938797
:10D18000A79D9C43B1C3A5CE8D472310F10083C753
:10D1900025004A852301F10083C73500A301F10072
:10D1A00083C745002302F10083C75500A302F100A5
:10D1B00083C7650093059100A30301002303F100D9
:10D1C00023040100EFF0CFC10C404A860A85EFF03E
:10D1D0004FC383564400032804008A85858EC20607
:10D1E0001D08C1822312D400A68881470147E51695
:10D1F00042864E85EFF07FB841016F40BFB54A8649
:10D200000A85EFF00FC0C9B7EF423FB3B335B000A6
:10D21000011185052A891315F601336515012308C7
:10D22000B1009305110136843AC632C03EC442C2F1
:10D23000EFF00FBBA2471248425593D68700230B4D
:10D24000F1009305910193578800A30AD100A30B25
:10D25000F100230C0101EFF0AFB83247024603287A
:10D260000400B337E000835644009207914411C292
:10D27000A1444A85A68842860C08EFF09F842A893B
:10D2800009E5A6852285EFB03F9F4A8505616F407D
:10D290001FADEF42FFA801113EC68647B335B0006F
:10D2A0008505AA891315F6015D8D2308B100930544
:10D2B000110136843A89B28442C446C2EFF04FB2BB
:10D2C00022489248164593578800A30AF100930517
:10D2D000910193D78800230B0101A30BF100230CCC
:10D2E0001101EFF0EFAF3247104083564400B337DF
:10D2F000E000920703280900914891C0A1480C085A
:10D300004E85EFF09FA7AA8411E5835544004A8516
:10D31000EFB09F96268505616F40DFA3AA9593071E
:10D32000F00F17F700001307278A6317B50013C51E
:10D33000F7FF1375F50F828005058346F5FFB58F5E
:10D34000BA9783C70700D5B7035745001441930721
:10D35000F00F17F600001306268736974207418321
:10D36000139506014181631BE500AD8FB29703C59C
:10D370000700130515F3133515008280850603C5D4
:10D38000F6FFA98FB29783C70700D9BFEF42FF9A74
:10D39000B28736842E86BA86AA853E85BA84EFF097
:10D3A0006FE6634B05002285EFB0D0312A86A68652
:10D3B000A2852685EFF00FE56F407F9AEF425F96DA
:10D3C0005D712A8BAE8A17E500001305657D2C0080
:10D3D000B284368ABA893E89EFF04FE42A8459E54F
:10D3E00034104146DA852800EFF0CFE12A843DED84
:10D3F0008547A303F100A6C2930771002408BEC4A9
:10D40000A68685470D462C18281002DC02DED6C001
:10D41000BEC6EFF00FDB2A8431E983477102A6868E
:10D420000D4693F7F7072300FA00C1473EDE2C189C
:10D430008947281026DCA303F100EFF08FD82A8457
:10D4400015E54146A6854E85EFB0607F8D47A686DF
:10D450000D462C182810A303F100EFF08FD62A8474
:10D4600011E54146A6854A85EFB0607D2285616160
:10D470006F405F8EEF427F8C97D700009387070C39
:10D48000984383C7470079712A89AE8417E5000065
:10D49000130585710C083AC42306F100EFF00FD88C
:10D4A0002A8415E514104146CA850808EFF08FD587
:10D4B0002A8411ED140815462C000810EFF08FD4C3
:10D4C0002A8411E521462C082685EFB04077228575
:10D4D00045616F40DF88EF425F8697D700009387F2
:10D4E000E7059C477971AA842E8417E5000013058F
:10D4F000256C0C083EC6EFF06FD20DE514104146C6
:10D50000A6850808EFF00FD011ED140811466C0045
:10D510000810EFF02FCF19E58347F10193F7F703D8
:10D520002300F40045616F409F83EF421F813688DE
:10D53000A14881470147E546EFF0AFD86F403F82F1
:10D54000EF42AFFF3688A14881470147E546EFF03B
:10D55000DF826F40DF80EF424FFE01112A842E856B
:10D560000C0832C6EFF08FCB19E9324797E600007E
:10D57000938686621008C1452285EFF03FE1056180
:10D580006F40EFFDEF426FFB4111C1472EC032C427
:10D590008A8509463EC23EC6EFF0AFC241016F40E8
:10D5A0000FFCEF428FF94111AE8613061009AA85D0
:10D5B0000A8502C002C202C402C6EFF0AFC4410134
:10D5C0006F40EFF9EF426FF7328797E600009386DE
:10D5D000A65E2E8693050002EFF05FDB6F402FF80A
:10D5E000EF42AFF57971C1472ACC2ED032D42C0846
:10D5F0000D4628003ECE3ED23ED602C402C602C828
:10D6000002CAEFF00FBC45616F406FF5EF42EFF2D9
:10D610000111AA842E8417E500001305655A8A8536
:10D62000EFF0CFBF05E514084146A6850A85EFF067
:10D630006FBD09ED8347E1010347F101A207D98FCF
:10D64000CA07C9836177D98F2310F40005616F4041
:10D650000FF105C9EF426FEE9787FF1F938747FDD4
:10D6600090439785FF1F9385E5FC1785FF1F1305E2
:10D6700025F8EFB080091785FF1F130565F76F4088
:10D680000FEE1785FF1F1305A5F682809DC5EF429B
:10D69000CFEA9787FF1F9387A7F9944301112E8440
:10D6A0000A869785FF1F9385E5F8EFB0800A0A8503
:10D6B0000294014505616F408FEA7D558280EF42FB
:10D6C000CFE7EFB080149787FF1F23A3A7F617F5C6
:10D6D000FFFF130525F8EF90D0406F404FE8178704
:10D6E000FF1F130727F79317150008433E95FD57B3
:10D6F0002310F5008280EF424FE42A84084019E1AC
:10D700006F40EFE51C4158401CC06313E5005CC04E
:10D710008347550023200500F99BA302F500EFB0D5
:10D72000EFF9E9BFEF42CFDF9787FF1F938787F4B9
:10D7300098432A8411CB8347350093F7070289C7A2
:10D74000035505008945029713054401EF90101316
:10D75000835504000355E400EF20701B485809C5A9
:10D76000EFB0CFF5232A040213058403EFF0BFF8CE
:10D770008144B149EFA0FF9A63C5A40283473400F6
:10D780002320040493F727FCA301F4000048EFA032
:10D790005F9A1316150081452285EF400FDD6F401B
:10D7A0006FDBB38734030329040385043E994A855C
:10D7B000EFF07FF42304090075BF8347350093F72A
:10D7C000070299E3014582808357E500E39CB7FE99
:10D7D000C167FD176316F600054582800545B9A0AF
:10D7E000EF42AFD593170601C187B2842A8401495D
:10D7F0006359F002835705008DCB01456367F6003E
:10D80000034584003E953325A6001375F50F39A80E
:10D810001C4813171900BA9783D70700E38097FCB9
:10D820000509EFA01F91E345A9FE01456F402FD3E5
:10D83000EF420FCFAE89AA84EFA07F852A84EFD074
:10D84000BFAAAA86014713068401970500009385A5
:10D8500045E91785FF1F130525E0EFA0AFD52A89FD
:10D8600021CD8C441304C50022859E0593F505083F
:10D87000EFB00FC5CC4083877400E18163D107040A
:10D8800093E505082285EFB0AFC30D4693854400AC
:10D890002285EFB00FC183D504002285EFB0EFC51C
:10D8A00083D524002285EFB04FC503D6490083A558
:10D8B00009002285EFB0EFBE4A856F40AFC993F5EE
:10D8C000F507C9B7EF426FC701112A84328532C606
:10D8D000EFB06FB4EF903F91835704001787FF1F9D
:10D8E0001307C7F03246231BF100930700F8A30D7E
:10D8F000F1001C471843231AA1008983858BB307C5
:10D90000F740B28548083ECE231C0100230D0100DC
:10D91000EFF01FF205616F408FC4EF426FC000410E
:10D92000014529CC9304C40026853289AE89EFB025
:10D930008FB295452A8A2685035B0401EFB02FAF8D
:10D940002685EFB02FC68D45AA8A2685EFB02FAE6B
:10D950002685EFB02FC55C48420A135A0A01D297B8
:10D960005CC423186401814763983A0146054D81E0
:10D97000330625419337160013F5F70F6F408FBD1F
:10D98000EF422FB989692A8BAE8B328AB68A8144DD
:10D990000144314CFD19EFA0CFF863C9A400EFA0FA
:10D9A0004FFB018D33B5AA006F402FBA3389840332
:10D9B00083270B003E9963170A008347890085047B
:10D9C0003E94D1BF03560A00DE854A8533F6C9006E
:10D9D000EFF0BFF47DD10545C1BFEF420FB6011195
:10D9E0002A847C000355E5003ECAB70707003ECCF9
:10D9F0007C003ECEEF10303D2A8985454808EFB0C7
:10DA0000EFC199454808EFB02FA7AA844A85EF10C7
:10DA1000B03D2380A4009787FF1F938727DD9C4399
:10DA20004166130606F09396870113D78701558F39
:10DA300093D68700F18E558FA207B706FF00F58FAA
:10DA4000D98F11462C00138514003EC4EFB0201F5F
:10DA50005008A382040089452285EFF0BFE609C97A
:10DA6000AA8513058403EFB0EFBB3C4085073CC09B
:10DA700005616F40CFAEEF424FACEFA08FED2A842F
:10DA80000504EFA00FEC3305A402F14791453305DF
:10DA9000F502EF10207B01E565556F404FAC97878D
:10DAA000FF1F23A1A7BCEFA0CFEA2A840504EFA0A3
:10DAB0004FE93305A40289450605EF10A07869DD1A
:10DAC0009787FF1F23A8A7B8EFA0AFE82A84050413
:10DAD000EFA02FE73304A4029787FF1F239E87B68A
:10DAE000EFA02FE72A84EFA0CFE59307140033853A
:10DAF000A7029787FF1F2392A7B697E70000938797
:10DB0000E7CF1787FF1F232DF7B4014579B7EF4201
:10DB10002FA1AA842E8901449789FF1F938909CDDB
:10DB2000130A8006EFA0EFE16345A40001456F40B2
:10DB30006FA23305440383A709024A86A6853E9552
:10DB4000EFF0BFC719E10504F1BF0545CDB7EF42BE
:10DB50004F9CAA8A2E8BB28B368C3A8A8144014420
:10DB60008149978CFF1F938C6CC8130D8006EFA022
:10DB70004FDD63C7A40011E085494E856F40EF9CDF
:10DB80003389A40383A70C025E86D6853E994A8515
:10DB9000EFF0BFC219CDEFA0CFDB0544636B4501A9
:10DBA000D2866286DA8513050903EFF07FDD11C1A5
:10DBB000854985046DBFEF42AF96C16441112A8942
:10DBC00001449789FF1F938969C2130A8006FD14D7
:10DBD00036C632C42EC2EFA0CFD692452246B246F8
:10DBE0006346A400014541016F40CF9633054403CD
:10DBF00083A709023E9509C683473500C18B9DC79F
:10DC000091C68347350093F707028DC363069900D9
:10DC10008357E500639C27010357050001CB63E7A9
:10DC2000E50083478500BA97E3CFF5FA05044DB7C1
:10DC3000EF420F8FC1642A8901449789FF1F93899E
:10DC4000E9BA130A8006FD14EFA0AFCF6344A40025
:10DC50006F404F903305440383A709023E958357D5
:10DC6000E500638897006304990063942701EFF04F
:10DC70007FAB0504D1BFEF424F8989692A8AAE8AFA
:10DC8000328BB68B8144178CFF1F130C2CB6930C70
:10DC90008006314DFD19EFA0CFCA63C4A4006F40C8
:10DCA0008F8A3389940383270C028355CA015A86CD
:10DCB0003E994A85EFF07FB005CD814D05A03384B4
:10DCC000AD038327090303D60B00D68533F6C900BD
:10DCD0003E942285EFF07FC419E5850DEFA06FC457
:10DCE000E3CFADFC31A02285EFF0FFA023040400B8
:10DCF000850455B7EF42EF814169AA8A014A178B23
:10DD0000FF1F130BABAE7D19C14B054CEFA06FC3CA
:10DD10006344AA006F406F8393098006B3073A03F8
:10DD200083290B02BE9983D7E900638C27016384A2
:10DD30002A016398570103A4890311E44E85EFF08B
:10DD4000DFC9050AE1B78357040163997707930494
:10DD5000C4002685EFA03FF085452A8D2685835C8B
:10DD60000401EFA0DFEC2685EFA0FFFF62056185CF
:10DD7000635F05028D452685EFA07FEB89452685EB
:10DD8000EFA0FFEA89452685EFA07FEA8545268535
:10DD9000EFA03FEB83470500094793F7F707639828
:10DDA000E70099452685EFA0DFE9A30285014848F1
:10DDB000337D2D01231894016A9548C40040B5BFF6
:10DDC000EF32BFF737E404008327041D829797875B
:10DDD000FF1F83C7A78E1755FF1F1305A537A30085
:10DDE000F5008327441C82978327841C81461306F1
:10DDF000F00F8145014582976F307FF61777FF1F3F
:10DE00001307C77B18439785FF1F83C5258B97870B
:10DE1000FF1F9387278983468703034697036397EA
:10DE2000D5009787FF1F238BC788828083C5870112
:10DE30000347A7036317B6009787FF1F2380E78870
:10DE4000828003C687016317C7009787FF1F238758
:10DE5000D786828083C68701130750026319D700D3
:10DE6000930760021787FF1F230AF784828083C607
:10DE70008701130660026315D60093077002DDB7B1
:10DE800083C7870155BF9787FF1F9387A781D44B0F
:10DE900009476385E608EF325FEA1779FF1F130928
:10DEA000A97D3E8483470900918B9DCFB7E4040090
:10DEB00083A7041D829783A7441C1775FF1F1305B2
:10DEC000257C829783A7841C81461776FF1F034613
:10DED000267D81450145829721C183470900ED9B3D
:10DEE0001777FF1F230AF7788347040093F7F70F8C
:10DEF00085C791471777FF1F2320F77CEFF05FEC72
:10DF0000EFF0DFEFB7E70400BC4F414691451775CE
:10DF1000FF1F0345A57982976F307FE48280EF323F
:10DF2000DFE18D4741116304F504C5476306F5023F
:10DF300085476310F5029777FF1F2383A778B7E71C
:10DF40000400BC4B930500101775FF1F03450576B1
:10DF5000829741016F30BFE085471777FF1F23018C
:10DF6000F776B7E70400BC4B93050020F1BF977725
:10DF7000FF1F93872773D44B1147638DE600B7E7E4
:10DF8000040083A7071D8297B7E70400BC4B9305E5
:10DF900000045DBF05491777FF1F232F277183C733
:10DFA000070032C62E8493F7F70FC5D7B7E40400F5
:10DFB00083A7041D7D141374F40F8297E37689FC04
:10DFC000B245994703C61500E3F0C7FCFC440906B7
:10DFD0001775FF1F1305056F8297BC48930500084E
:10DFE0001775FF1F0345856C829779BFEF32FFD409
:10DFF0001777FF1F1307076B4047184B1C40977696
:10E00000FF1F23A7F66A6316E4001777FF1F232379
:10E01000F76A130584FEEF907FF3035564FFEF90DA
:10E020003FC6EFA0BFE96F309FD3EF321FD1977784
:10E03000FF1F93872767D84BDC4799C3EFF01FFB7F
:10E0400085471777FF1F2329F7669777FF1F938769
:10E05000E7569C43930500021775FF1F03450565AE
:10E0600083C787031777FF1F230AF764B7E7040006
:10E07000BC4B82976F30BFCE9777FF1F23A6A76256
:10E080008280EF32FFC937E404007C4CA14517754C
:10E09000FF1F0345A56182977C48A1451775FF1FA7
:10E0A0000345C5609774FF1F9384C45F8297DC4467
:10E0B00089E7EFF05FDD6F30FFC903D567FFEF90B1
:10E0C0003FBCAA897DD5D84891476310F7027C4CA4
:10E0D00091451775FF1F0345655D82977C48914503
:10E0E0001775FF1F0345855C829703A9490103D477
:10E0F00009018947B7E904001777FF1F232EF75A54
:10E1000083A7091D21044204829783C78401175500
:10E11000FF1F1305250461191757FF1FA30CF702F2
:10E1200083A7491C418082979777FF1F238A07584E
:10E1300083A7C91C814609469375F40F4A858297C7
:10E1400011E99777FF1F83C7E76789C79740FF1FCC
:10E15000E7800072B7E70400BC4F2146A145177560
:10E16000FF1F0345A5548297B9B7EF321FBD93F740
:10E17000052001112E8481CBEFF03FEB13450420E5
:10E1800005616F30DFBD93F70510A9CB9774FF1FB2
:10E1900093844451DC48EFF07FC61777FF1F1307C5
:10E1A000E741184383C78401034787036316F700D9
:10E1B000DC4499C3EFF09FE385471777FF1F232DBA
:10E1C000F74EB7E70400BC4B930500021775FF1F1D
:10E1D0000345C54D8297134504105DB793F70508B5
:10E1E000ADC79777FF1F83C7F74DE9171946977596
:10E1F000FF1F9385454D1305D10093F4F70F177951
:10E20000FF1F0349294CEFA0902393970401C1837A
:10E210001777FF1F1307874B231DF100231CF10005
:10E220009777FF1F938707483ACE3ACAD843230609
:10E23000010009CBDC439315890154080D46E185A3
:10E24000680082971345040825BF93F72500B1CFD6
:10E250009777FF1F93870745D84B89476306F702D7
:10E260009777FF1F83C7474113F7270011EF918B63
:10E2700099CFB7E70400BC4F1306000A894517750C
:10E28000FF1F0345A542829713452400D5BD97770C
:10E29000FF1F9387A7329C4383C787031777FF1F0E
:10E2A000230EF740EFF0FFDDC5B793F7050291C7E6
:10E2B000EFF03FDD13450402E1B593F7850091C708
:10E2C000EFF0BFD61345840065BD93F7150091C7E5
:10E2D000EFF07FBB1345140065B593F7450091C778
:10E2E000EFF07FBA1345440061BD93F7050485C381
:10E2F0009777FF1F83C7073B81CBEFF07FAC914738
:10E300001777FF1F232AF73A1345040495BD93F7A7
:10E3100005010145E38607E69777FF1F9387873856
:10E32000D84B91476310F7049777FF1F9387C73443
:10E330009C4313D727008583D98F858B91E7B7E757
:10E34000040083A7071D8297B7E70400FC4F91459F
:10E350001775FF1F03458535829785471777FF1F80
:10E36000232CF7341345040121BD9777FF1F238B1E
:10E37000A7448280EF327F9C9777FF1F23AA073242
:10E380009777FF1F23A8073285471774FF1F1304D1
:10E39000E4221777FF1F2321F7321C4083C787032E
:10E3A0001777FF1F230CF730EF90FFDF39C1975726
:10E3B000FF1F23A5A7DA1C4017050000130525DB66
:10E3C00083C787031777FF1F230AF72E1757FF1FEF
:10E3D000A302F7D89777FF1FA386072CB7E704009F
:10E3E00083A7070882979777FF1F2381A72C6F3099
:10E3F0001F97B7C7898E938767ED1757FF1F232F86
:10E40000F7D455BF1777FF1F0347C729795555E341
:10E410009777FF1F9387072903C71700050797768C
:10E42000FF1FA381E62803C717008D463377D70265
:10E430009776FF1FA388E62683C617001777FF1F6E
:10E440001307C717184393F6F60FA9EA8347870304
:10E450001777FF1F2304F72685471777FF1F23032E
:10E46000F7249777FF1F938727219C430145998BBA
:10E47000A9E3EF329F8C37E404007C48C14517754F
:10E48000FF1F0345A52282973C4885451775FF1F4E
:10E490000345C521829701456F307F8C83C71700E4
:10E4A00085466395F600834797035DB78347A703C7
:10E4B00045B782809777FF1F83C7C71EA1CBEF3276
:10E4C000DF8737E404009777FF1F238D071C7C4804
:10E4D00085451775FF1F0345651D82977C4C914547
:10E4E0001775FF1F0345851C82977C48914517755A
:10E4F000FF1F0345A51B82973C48C1451775FF1FA9
:10E500000345C51A829701456F307F857955828012
:10E51000EF32BF822A84035565FFEF906FF697773D
:10E52000FF1F93872718D847BE841DEBEFA05F9885
:10E530009C48232004008DEB9777FF1F23AC8716A0
:10E540009777FF1F23A68716B7E70400BC4B8945C2
:10E550001775FF1F03458515829701456F303F8072
:10E56000630A87001843D1B780C39777FF1F23A39F
:10E570008714D9BF7955DDB7EF322FFC9777FF1F8E
:10E58000938787248843232605002324050051050B
:10E59000EF80D02E6F30AFFCEF322FFA1774FF1FD1
:10E5A000130484221C40411189CF9C472302B500EB
:10E5B0002AC61CC1EFF05FFC1C409C4B99C332453E
:10E5C000829741016F30AFF9EF322FF74111444D7F
:10E5D000328532842EC6EFA00FF92AC42285EFA01F
:10E5E000EFF903A84400630C0800B24583574400C8
:10E5F0001840224683D54500AA8626850298410107
:10E600006F30EFF5EF326FF3404D1DC408C0970532
:10E6100000009385E50213054401EF809018977779
:10E62000FF1F9387671A9C43014589E79777FF1F70
:10E6300023AC87186F30AFF27D55EDBFEF32EFEFAF
:10E64000011168009305F00F02C602C802CA02CC8D
:10E6500002CEEFF07FF405616F306FF09777FF1F08
:10E66000938787169C43D847A1679D076311F702DC
:10E67000EF32AFEC01113285EFA0EFEE230AA100DB
:10E6800081456800EFF05FF105616F304FED8280EA
:10E690009777FF1F938747139C43D847A1679387BA
:10E6A00077036311F702EF324FE901113285EFA0D2
:10E6B0008FEB230AA10081456800EFF0FFED0561B3
:10E6C0006F30EFE982809777FF1F9387E70F9C43B6
:10E6D000D8479547631CF702EF322FE601113285C8
:10E6E0003284EFA04FE8230AA1002285EFA00FE9B2
:10E6F00083574400231BA10081453ECC1C40680089
:10E700003ECEEFF07FE905616F306FE582809307C1
:10E7100085FF89CF8327C5FF91CBDC4B81CBEF32BF
:10E72000CFE1032585FF82976F306FE38280EF3260
:10E73000CFE02A843285EFA00FE3BD4763EBA7004B
:10E7400018449377F5000345B70041995D8DA30503
:10E75000A7006F30CFE0EF324FDE01117C003ECAE0
:10E76000B70707003ECC7C003ECE5C4D8DCF2A849F
:10E7700013858700AE84EF807004A1652A899D050A
:10E780004808EF80FFBD9305803EB345B9024808B5
:10E7900093F5F50FEFA0CFD2014781465008A6852B
:10E7A0002285EF807FDC05616F306FDBEF32EFD8C1
:10E7B000EFF07FFA6F30AFDAEF322FD801117C0023
:10E7C000AE843ECAA165B70707002A843ECC48083C
:10E7D0007C00938575033ECEEF809FB81C444808AB
:10E7E00083C5B700BD89EFA0AFCD50080147814672
:10E7F000A6852285EF805FD705616F304FD6EF3257
:10E80000CFD32A84AE84EFF09FF2A6852285EFF065
:10E81000BFFA6F30CFD4EF324FD2EFF0FFF96F3045
:10E820000FD4EF328FD10329C501411163040902CE
:10E830002A843285B284EFA00FD32AC62685EFA0A2
:10E84000EFD3832749002A8691C7DC4781C7B245A9
:10E850002285829741016F308FD0EF320FCE444D29
:10E8600081CC2A843285EFA06FD1DC40AA8589C78C
:10E870009C4799C3228582976F306FCEEF324FCA83
:10E88000032AC501411163030A062E89AA8495450E
:10E8900032853284EF80DFAC85452285EFA0CFBD85
:10E8A000AA89CA852285EFA0EFC283274A009DC7A7
:10E8B000DC438DC72285EFA0AFBA83274A00104002
:10E8C00083564400DC437115A307A100B2961307D9
:10E8D000F1004E86CA852685829701C523800900EE
:10E8E00031A08345F1002285EFA00FB941016F30BF
:10E8F0006FC6EF328FC465711C083EC2B707800136
:10E900003EC41C0832893EC62A84AE84EFF07FF1F3
:10E910004A85EFA0AFC68357A10089CFAA855000D2
:10E920002285EFF0BFF5014781465000A68522857C
:10E93000EF809FC359616F308FC2EF326FBE657138
:10E940001C088329C5013EC2B70780013EC41C08CC
:10E950002A84AE8432893EC6EFF03FF06384090218
:10E960004A85EFA0AFC18357A100AA8581CF50008F
:10E970002285EFF0BFF0014781465000A685228531
:10E98000EF809FBE59616F30EFBCEF320FBB6571F6
:10E990001C083EC2B70780013EC42A841C08328589
:10E9A0003EC6AE84EFA08FBD8357A10089CFAA8554
:10E9B00050002285EFF09FEC014781465000A6856C
:10E9C0002285EF807FBA59616F306FB9EF32EFB6B1
:10E9D000444D91E88347450093B71700B307F040D3
:10E9E0003E856F30CFB71845FD577DDB9707000098
:10E9F000938707032A845CCB97050000938565D134
:10EA000013858400EF80E05980C0034744008147AC
:10EA100061FB1777FF1F232B97DAD9B7EF324FB07F
:10EA20008329C5014111032985008147638B0908AA
:10EA30000324090191452A8A2285EF807F9285452A
:10EA40002285EFA06FA38945AA8A2285EFA0CFA2D5
:10EA5000AA84EF809F9683A749002A8B9DC79C4379
:10EA60008DC72285EFA0CF9F83A74900A306A100F1
:10EA70001040835644009C431307D100B296D685BC
:10EA80001306E1005285829709CD83570B0023803E
:10EA9000F400A183A380F40023800A00A3060100F0
:10EAA00029A88357E10022852380F4008345D10003
:10EAB000A183A380F400EFA02F9C8347D100B3373C
:10EAC000F0000347B900920701453D9BD98FA3058C
:10EAD000F90041016F300FA8EF322FA641111DE957
:10EAE0009777FF1F938787CE804305C8044013099B
:10EAF00084009DC55C4099C79C4B89C726852EC65E
:10EB00008297B2459307803EB385F5024A85EF8030
:10EB1000605521A0404DAA8479F841016F302FA49F
:10EB20004A85EF80A0555C40EDDBDC4BFDD72685A8
:10EB30008297E5B7EF326FA02A843285EFA0AFA2AB
:10EB4000AA852285EFF05FF96F306FA1EF32EF9E5B
:10EB50002A84AE84EFF01FFEA6852285EFF0BFBFAA
:10EB60006F30EF9F08413355B50005898280EF3241
:10EB7000CF9C1774FF1F130464C71C5C011123177B
:10EB800001008D83858BA303F1008327040B2318D9
:10EB900001002319010003D7C7013ECA3C0023141A
:10EBA000E1007D572315E1000357C4023ECC02CE9D
:10EBB0002316E100EF802FE38357E101231EA1001C
:10EBC00093F707E093E71710231FF1009777FF1FD4
:10EBD00083C767C485C305470145638AE700834748
:10EBE000840393E727001777FF1F230DF7C2056102
:10EBF0006F30EF96814717D700001307271C854613
:10EC00001306710085454808EF70E04B6DF18347AE
:10EC10008403F59B1777FF1F2306F7C085471777F7
:10EC2000FF1F230AF7BEE1B7EF322F8E977DFF1F3C
:10EC3000938DCDBB03A6CD0639712A8981478144C6
:10EC4000930600023357F600058B01C7850493F441
:10EC5000F40F8507E398D7FE83A70D0B2317010256
:10EC60002318010203D7C7013EDA3C102314E10246
:10EC70007D572315E10203D7CD023EDC23190102A3
:10EC80002316E10202DEEF800FD68357E103231E35
:10EC9000A102014593F707E093E71710231FF10244
:10ECA0009777FF1F83C727B7A9EF9777FF1F83C702
:10ECB00077B73EC69779FF1F938949B30144014D49
:10ECC0009D4A054B954B177CFF1F130C6CB9977C25
:10ECD000FF1F938C6CB803DAC90563090A00EA8543
:10ECE000631459036685EFF0FFE71DC1050DA147C9
:10ECF0008909E312FDFE2DE09777FF1F23A007B6D9
:10ED0000014521616F302F846285EFF0BFE579DD29
:10ED10003247B3878400E3F0E7FE9C00130614003B
:10ED200006043E9413178A0093578A00D98FC207AE
:10ED3000C183A30EF4FCA183230FF4FC03A70D07EA
:10ED4000B317AB01D98F1777FF1F2329F7B06304DF
:10ED50007601328461BF15449777FF1F83C787AB65
:10ED6000138717009776FF1F2386E6AA93161400D1
:10ED7000230EF10017D700001307470481478506CB
:10ED80007008CA854818EF700034E34705F68347DA
:10ED9000C10105451777FF1FA30EF7A69777FF1F41
:10EDA000238B27A7B9BFEF22BFF70111AA892E84B1
:10EDB000EFD0EF9C2A899774FF1F938424A3639953
:10EDC000090A9C5C414793F707036393E70A1777A7
:10EDD000FF1F034797A4894763ECE70883A7040B49
:10EDE000231701002318010003D7C7013ECA3C00C6
:10EDF0002314E1007D572315E10003D7C4023ECC64
:10EE0000231901002316E10002CEEF80CFBD231E9F
:10EE1000A100EFC06FCD8357C101230FA100914620
:10EE200013D78700A207D98F2312F1009777FF1F0E
:10EE300083D7679F13D78700A207D98F2313F100C9
:10EE400017D70000130707F781475000954548087A
:10EE5000EF70602705889317240003C484036D981E
:10EE60005D8C9777FF1F238F879A05616F209FEE38
:10EE7000EF70B0781775FF1F1305459BEF800020DA
:10EE800083A7040B9775FF1F83D5059903D5C70189
:10EE9000EF10E0279777FF1F83C7C79893F6070205
:10EEA000014789E61777FF1F035707979776FF1FDC
:10EEB000239CE6961777FF1F13070792184309CB89
:10EEC000C18B99C789451775FF1F0355E5940297B4
:10EED0009777FF1F23A207949777FF1F238D079231
:10EEE0009777FF1F23AA07969777FF1F23A80796F8
:10EEF0009777FF1F23A6079683D7840393F7270CE2
:10EF000093E717001777FF1F231EF79083572903F6
:10EF1000A18B99C3EF70E03F11C49777FF1F23A91E
:10EF2000078EA1B78D471777FF1F2323F78EEF902A
:10EF30002FA59305803EB305B5021775FF1F130576
:10EF4000E58EEF80201215B79777FF1F9387078A0A
:10EF5000D85325C791C99777FF1F238E078A9777C4
:10EF6000FF1F23AD078E8280EF223FDD83C7F702AC
:10EF700041112EC685071777FF1FA300F78A9777E1
:10EF8000FF1F2394A78A9D471777FF1F2322F78827
:10EF9000EF900F9E2A84EF90AF9DB24501E5EF9070
:10EFA0002F9DAA85B305B4401775FF1F130505886B
:10EFB000EF80400B41016F209FDA82809777FF1F1F
:10EFC0009387C782D85331C7EF223FD703C7F702D1
:10EFD00005079776FF1FA382E68411CD8C5F0D474E
:10EFE0000145898185899776FF1F23A3E682EFF08B
:10EFF0009FDB6F20DFD685479305C0441775FF1F41
:10F000001305C5821777FF1F2324F780EF80800543
:10F01000CDB78280EF227FD21767FF1F0347A77FFC
:10F020008547631EF7009767FF1F9387277C83C779
:10F03000870393C787001767FF1F2305F77E1765B0
:10F04000FF1F1305A57EEF806003EF807FEF9947D8
:10F050001767FF1F232EF77A9767FF1FA38F077A83
:10F060009767FF1F2389077AEF90AF8F93074006BA
:10F070003305F5029767FF1F23A2A77A6F203FCEC3
:10F080009767FF1F83C7077AC18B99C7EF22FFCA13
:10F09000EFF0FFAD6F20BFCC695582809767FF1FEF
:10F0A0009387C774DC5381CBEF223FC98545EFF0CE
:10F0B0009FCF6F20DFCA82801767FF1F1307077378
:10F0C00001468146BA852148631E06019DCA2390E8
:10F0D000A60083C7850393E717001767FF1F230365
:10F0E000F77405A08357C705631DF502F8598547D6
:10F0F000B397C70093C7F7FFF98F1767FF1F232147
:10F10000F7769C5D9183858B85C79767FF1F83C7C3
:10F11000877099EFEF227FC21D45EFF0FFB06F209F
:10F120001FC481E699E39306C7050506090769BF71
:10F130008280EF221FBE8605AA84B309B500976AB4
:10F14000FF1F938A6A71054B976BFF1F938B0B719F
:10F15000214C639434039767FF1F938727699C5F53
:10F160009183858B89CB9767FF1F83C7C76A81E728
:10F170002145EFF07FAB6F205FBD03DA0400630B26
:10F180000A041769FF1F130969660144CA8C835773
:10F19000C905639D4703A2855685EFF0BF9C11E525
:10F1A000A2855E85EFF01F9C05C903A74C07B31726
:10F1B0008B00D98F1767FF1F2324F76A83C78C033F
:10F1C00093E717001767FF1F230EF764050409096B
:10F1D000E31F84FB8904B5BF231E0904C5BF17675D
:10F1E000FF1F034747638547631AF700EF22FFB409
:10F1F000EFF05FE2EFF0BF976F207FB6828081472C
:10F2000085451306000293861700B397F500E98F32
:10F2100013F7F60F89E7B687E397C6FE01473A85ED
:10F220008280FD4785457D56B396F500138717000C
:10F23000E98E1377F70F89E6FD17E397C7FE0147BD
:10F240003A85828089E901473A85828001473A857B
:10F2500041016F20DFB0EF225FAE41112AC62E853B
:10F260002EC4EFF0DFF9A2457D158547B397A700BF
:10F27000E39EF5FC32469377360099C3719A1106E6
:10F280009767FF1F9387475694433E871768FF1F72
:10F290001308C85489EA832708009107F19B9766F1
:10F2A000FF1F23A3F654032588001843B307A700C4
:10F2B000B3F7B702B387F540FD15FD8D83274800EE
:10F2C000AA95B306B600E3F3F6F8E371D5F82E97E6
:10F2D0009767FF1F23A8D7503DDB3A858145EF2074
:10F2E000DFA82A87ADB718419767FF1F9387074F9D
:10F2F00023A4070098C35841D8C39767FF1F23A5CD
:10F30000074E8280EF22DFA1AA8401441769FF1F04
:10F310001309C94D9309400EEF807FD56345A400C2
:10F3200001456F203FA3330534038327090B3E9526
:10F330008357C501E38797FE0504F9BFEF227F9D40
:10F340009769FF1F9389894A3E84BA8483470600E0
:10F3500003A7090041119D83058B3D8F83C744019D
:10F36000AE8A2A89F99BD98F238AF4001C44B6857A
:10F37000231204001CC02285328A36C6EF90DF8F2C
:10F38000B246D2853686EF90900BDC4883A5090003
:10F390000840858B56869D8DEFD03FCC61E91840A3
:10F3A0007D558347570003476700A207D98FC207DF
:10F3B000C1872394F4006358F00A83C7440193F78C
:10F3C0000703B5CBD0489377160003A609001D8E1E
:10F3D0009767FF1F938747789C43ADEB814641A019
:10F3E00003A70B0093172A00BA971840944383474A
:10F3F00057008345670033F65601A207CD8F63118E
:10F40000F602834737000346470003472700A20759
:10F41000D18F4207D98FBD82B3F76701638AF604A3
:10F42000050AEF80DFC3420593170A014181C183BA
:10F43000E3E8A7FA41BFA16A370B0200014A976BC4
:10F44000FF1F938B6B48FD1A7D1BE1BF83C74401EF
:10F4500013070003854693F70703E391E7F8A285B6
:10F460004A85EFD0FFCF41016F203F8E6155E5BF48
:10F470007955D5BFEF22DF8A9764FF1F9384441F1D
:10F480009C40D9EF9767FF1F9387C7349C436399CC
:10F49000070CEF80DFBE930780023305F502894534
:10F4A000EFF05FDA41C99767FF1F23A7A73EEF8000
:10F4B0001FBC9307400E3305F5029145EFF09FD82E
:10F4C00035C99767FF1F23ABA73CEF805FB201CD23
:10F4D000EF80FFB191450E05EFF0DFD621CD9767A4
:10F4E000FF1F23AFA73AEF801FCB11CDEF80BFCA1C
:10F4F000D9473305F5028945EFF0DFD405CD97678D
:10F50000FF1F23A9A738EF809FB591450A05EFF0AB
:10F510007FD30DC19767FF1F23A8A73A014521A8F4
:10F52000EF803FC2930780063305F5029145EFF067
:10F530007FD101E565556F20FF819767FF1F23A7E6
:10F54000A72C0144130A80061769FF1F1309092A13
:10F55000B14AEF801FBF6364A4029C40E38407F2BA
:10F56000EF803FBE9307A0043305F5028945EFF015
:10F570007FCD69D19767FF1F23ACA73419BFEF80F8
:10F580005FBB89450605EFF0FFCB4DD5B3094403BA
:10F59000032709024E9708CBEF80BFB83305550308
:10F5A0009145EFF03FCA59D583270902050413742A
:10F5B000F40FCE9788DB71BF9767FF1F93870723F0
:10F5C000884705898280C167FD176319F500976731
:10F5D000FF1F9387A72103A5070B8280EF22EFF57A
:10F5E000EFF05FD26F20AFF7814709C58347E50190
:10F5F000B337F0001767FF1F1307471F184709832A
:10F60000058B19C393E727003E858280EF22EFF236
:10F610002A84EFF07FFD8347E401AA85130594084F
:10F6200099E3130504039766FF1F9386261C9442F3
:10F63000130615021307840213059504EFD0CFC0FB
:10F640006F20EFF1EF22CFED9764FF1F9384041A30
:10F6500098442A892E840983058B9C4019C763141A
:10F66000F5006380050E014401A2E3FEA7FE1387A7
:10F67000A702E36AA7FE850763FCA70883A9440BDA
:10F68000EF80FF961316350081454E85EF20EFED94
:10F690009767FF1F23AC27159767FF1F23AA07143F
:10F6A00049CC9C4493E747001767FF1F2324F714B6
:10F6B0009767FF1F2388071A630F040C9767FF1FC4
:10F6C00023A6271301440549EF807F926341A40AD2
:10F6D000EF80FF9493050006B3C5A502B7F7360087
:10F6E000938707E81765FF1F130505184169014453
:10F6F0009309400E7D19B385F502EF70B016EF80C7
:10F700001F97634FA4080145EF3040700544A9A836
:10F710006398A7029DE583A9440BEF805F8D1316C4
:10F72000350081454E85EF204FE49767FF1F23AFDB
:10F73000270B9767FF1F23AD070A9C44ED9BADB7CE
:10F7400085C51767FF1F0347E7119307F005E3FC23
:10F75000E7F021F8EF60F03C6DD19C4493E707029D
:10F760001767FF1F2328F70822856F20AFDE83A7C6
:10F77000440B131534003E958357050081CB834716
:10F78000250099C721468145EF202FDE05042DBFB6
:10F7900023012501E5BF9767FF1F23AB07040DBFBA
:10F7A0003305340383A7040B3E958357C501638457
:10F7B0002701EFF0BFE5050499B7EF220FD8EF80DE
:10F7C0001F86130400063345A4029764FF1F938429
:10F7D000E40183C784073E951375F50F9767FF1FF4
:10F7E0002382A7089307F00563E7A7020545EF30DA
:10F7F000E061EF80DF823345A402B7F536009385E0
:10F8000005E8B305B5021765FF1F1305E505EF70A1
:10F8100070056F20CFD49C4405458983858B81CBAF
:10F82000EF904F8888408145EFF0DFE1DDB7EF30A2
:10F83000E05DC5B7EF22CFCE130495082A891306E1
:10F840009005A28513050503EF90603F1306900510
:10F8500081452285EF206FD14A85EF30C054814425
:10F86000176AFF1F130A8AF8930A8002EF803F810C
:10F8700063C4A4006F200FCE338454038327CA0AC5
:10F880003E94035704008357C9016317F702834767
:10F8900044009DC3930964014546CE851305540079
:10F8A000EF90E039454681454E85EF200FCC22850B
:10F8B00023020400EF30005785044DBFEF22EFC74D
:10F8C0009767FF1F9387C7DA9C432A8491C70DC5AA
:10F8D0000355C501EFE00FC29767FF1F9387C72746
:10F8E0009C4389CBEFB0DFD085476315F5002285B7
:10F8F000EF50C05D6F20AFC641657D15E1BFEF22BF
:10F90000CFC31764FF1F130464EE444093871400B1
:10F910001767FF1F232EF7ECEF30605E1C448983CE
:10F92000858B9DE75840B7E7B0009387075063F198
:10F93000E7020145EFF01F9D01CD0545EF809FF6E1
:10F94000084085450505EFF0FFCF0145EFF01FF7B3
:10F9500026856F20CFC0EF22AFBCA1642A89014465
:10F960009769FF1F938949F6FD14338AA500EF803C
:10F970000FEF6344A4006F20EFBD03A709009317A6
:10F980002400BA979843658F42074183634C27014F
:10F99000635A470123800700A380070023810700E3
:10F9A000A38107000504E1B7EF222FB68359450074
:10F9B000C547411163F537310441C1E53385340151
:10F9C000834785FF034795FF0348B5FFA207D98FFB
:10F9D0000347A5FFC207220733670701D98F0347F3
:10F9E000C5FF0348D5FF2207336707010348E5FF3A
:10F9F0000345F5FF420722083365A800498FB98FF8
:10FA00001767FF1F130707EA1768FF1F130888EB24
:10FA10003A85832807006384172B1107E31B07FF30
:10FA20001767FF1F130707EA1843131827004295AB
:10FA30001CC10507A1473367F7029767FF1F23A380
:10FA4000E7E893F735001397470083474601C16BFA
:10FA5000368993F7F7FCD98F32842E8A230AF60071
:10FA6000814A176CFF1F130C6CD8FD1B976CFF1F8E
:10FA7000938C0CC0176DFF1F130D8DE5EF802FDFEA
:10FA800063C7AA00E154268541016F20CFAB13085C
:10FA9000400EB3870A0303280C0BB30DF800638EE6
:10FAA0000D2083D7CD01638A772183A70C00014BFA
:10FAB000639707169767FF1F9387C7D19C4363908F
:10FAC000071683C7040003C70D0493F7F707631BEA
:10FAD000F71ACA872287CE86268693859D061385C8
:10FAE0001D04EFF0BF85631F051883D7CD010327E1
:10FAF00009002320B4012312F400FD572313F4005E
:10FB00008347170093F6F7078347D40093F707F866
:10FB1000D58FA306F40093F7F707B337F000B307C8
:10FB2000F0402307F400834717009D839396370026
:10FB300083474401DD9BD58F230AF40083473700B8
:10FB400083464700A207D58F83462700C206D58F7C
:10FB50001CC88347770003478700A207D98F231566
:10FB6000F4000D476304EA00BD5491DF938707104A
:10FB7000C207C1831307B00FBD54E376F7F0EF80DF
:10FB80000FC98144E31105F09766FF1F83C606D4B1
:10FB9000938716001767FF1F230AF7D21767FF1F07
:10FBA000130787D2231BD4009397260014430357CF
:10FBB0008400E175BE96A1671386F7FFB377C7008F
:10FBC00098426D8FD98F9CC21848F18F3E07D98F0C
:10FBD0009CC2EF80CFC89767FF1F83C727CF33F53D
:10FBE000A7029767FF1F2383A7CE71BD9307A004C9
:10FBF000B308FB0283270D00BE9803D7080083D704
:10FC0000CD01631DF70083C7040003C7880093F785
:10FC1000F707630BF70083C7FD019DEB050BEF8032
:10FC20004FD2E345ABFC71BD9385980113859800D5
:10FC3000CA872287CE86268646C6EFF02FF0B248C6
:10FC400079F98347440193E74700230AF40071BD23
:10FC500083C7040003C7980293F7F707E310F7FC84
:10FC6000CA872287CE8626869385A8031385A80295
:10FC7000EFF0CFEC45F58347440193E72700230AD3
:10FC8000F400C1B783C7FD018DCB83C7040003C750
:10FC90009D0993F7F7076312F702CA872287CE867A
:10FCA000268693852D0C1385AD09EFF02FE911E51C
:10FCB0008347440193E7270049BF850AC1B3FD5438
:10FCC000D9B3EF220F85797183544500AA8B2E8416
:10FCD000B28AEF80CFBB590563499504B7E40400AD
:10FCE00003A90407EF80AFBA590542054181029983
:10FCF0002A8905CD2AC623180100EF804FB959057E
:10FD00002319A1006146814528089769FF1F93893F
:10FD1000E9AD4ACAEF206F852302810203A489005E
:10FD2000058819E4BC544A85829745616F20EF81AC
:10FD300074003008D6855E85EFF01FC765F5680052
:10FD4000EF807FF1176AFF1F130A0AE183270A0079
:10FD5000AA84035B010189CB89476397FA00835525
:10FD600001025E85EF50203003552102EF704FC82D
:10FD700019E503552102EF708FD43334A000931797
:10FD800064000344C1022C0868001374F4FB5D8C0A
:10FD900023068102EF60B056E9576314F5028356DB
:10FDA000E1029767FF1F938727B29C4313972600B2
:10FDB0006176BA979843718F98C39767FF1F23871F
:10FDC000D7B0831721026345F00085476396FA0098
:10FDD000B25793F7070C95E7D247C2040347C10215
:10FDE000C180BE9426C62318610113770703C1475B
:10FDF000631DF70083475102054793F7F7076390A8
:10FE0000E704B7E70400BC5739BF92570544A18304
:10FE100093F7F707E377F4FE15C78347C10213078B
:10FE2000000293F707036397E700EFB06FFC854785
:10FE3000E319F5FC8347C10293F7070389CFEFB0BD
:10FE4000AFCA21A8EFB08FD7E30985FCEFB04FFA16
:10FE5000E31985FAD9B7EFB0EFD8AA850146054571
:10FE6000EF707FF82A8451DD8347C102414793F741
:10FE700007036384E70232478347170093F707F8C5
:10FE8000A300F7003247925783461700A18393F7E8
:10FE9000F707FD17D58FA300F70003560101B24500
:10FEA000130BC4005A85EF80DFDFE24A130690058A
:10FEB0008347C10283C4EA01918BB384C4021385D2
:10FEC0001404569595C35444B3879A0083C7070416
:10FED00003C70600137707F82380E60058448346DB
:10FEE0000700D58F2300F700B25703A6090081460B
:10FEF000858B1D8EDA85EFD0EF9B15E9B25783A570
:10FF00000900484413869406858B56969D8DEFD044
:10FF1000CF9411ED83270A0099EFB25705479183DB
:10FF20008D8B6387E7049DCF09476389E7042285AA
:10FF3000EF80DFF8F9B5EFB0AFEB85476309F50067
:10FF40008347C102414793F70703E398E7FC8355D2
:10FF500021025A85EF40907C69D183172102E35E2C
:10FF6000F0FAF1B7EFB08FC57D151335150061D1EB
:10FF7000014681452285EF70FFEF55BFEFB04FE797
:10FF8000E5B7EF129FDB9764FF1F9384A487268554
:10FF9000EF809FEB2A8419E16F107FDC1305C4000A
:10FFA00005468145EFF0FFD12285EF803FF1C5B7CF
:10FFB000EF12BFD84111AE842A849307950313072B
:10FFC00015019306F10005466C0026852306010005
:10FFD000EFD0CFBE1DEDA68541462285EF8030468D
:10FFE0008347F1009305140226852308F400EFD01F
:10FFF0006FC805E19767FF1F938707B69C4389EF9A
:020000040001F9
:100000001306940497C500009385C5DB2685EFD0C1
:100010008FD441016F10BFD41306940297C500001E
:100020009385C5DA2685EFD00FD379D9DDB7EF12E6
:100030003FCF9767FF1F938727898043AE84B2899C
:10004000368AAA8AEF80AF81131625008145228562
:10005000EF10BFD19767FF1F238A07869757FF1FAF
:100060009387C77803A4070B13F714003E89230F67
:10007000E400CE8525C713059408EFF07FF301C592
:1000800055556F103FCD8947A30FF4009767FF1FA9
:10009000938787AC9C4303278900858093B717001B
:1000A00086072300F402231E54019757FF1F23AF36
:1000B000477385889377B7FF99C0936747001757B1
:1000C000FF1F2329F7722285930700061757FF1F8A
:1000D000230AF778EFF08FD3014565B713050403C2
:1000E000EFF01FED45D569BFEF123FC5FD57231057
:1000F000F500231105002312050023130500130644
:10010000200481452105EF105FC66F105FC5EF1217
:100110003FC14111AA8401441759FF1F1309497BAC
:100120009309A0042EC6EF80CF81B2456344A4009A
:1001300061550DA033053403832709003E9583578D
:100140002500639CB7008357050063989700EFF084
:10015000BFF9014541016F10FFBF0504E1B7EF1280
:100160003FBC9757FF1F9387E7669C434111AA84C2
:100170002E84B28903592500C1C39757FF1F83D727
:10018000A769639B2707EF700F862A8903D5240090
:1001900093051002B305B40285472302F10093577B
:1001A0008900A302F10093578500A303F10083D7D0
:1001B00044002304A100254613D787002305F1003E
:1001C00083D76400A304E1004E8513D78700A305FD
:1001D000E1002306F1001387950093879501A1059F
:1001E000B386B400A6974C00269723032101EFD0D5
:1001F000EF9C41016F101FB6EF60FFFE51BFEF1281
:100200003FB24111AA8401441759FF1F1309496CD9
:100210009309A0043AC636C432C22EC0EF707FF2F2
:1002200082451246A24632476344A400615599A014
:10023000B307340303250900AA9703D8070003D5A1
:10024000C4016310A80495E91DEE91CA03C6E40138
:10025000930510023306B60225063E9690C201456C
:1002600011CB83C6E40113061002B386C602E5066D
:10027000B6971CC341016F10FFAD03D52700E305FE
:10028000B5FC050441BF83C5E40113051002B38525
:10029000A502BE9583C585002300B6007DB7EF1289
:1002A0003FA85C4141112A8403DA2700C167FD178A
:1002B000AE843289630CFA002685EF807F9A8D47E1
:1002C00063EDA7007D5541016F10DFA82E85EF80FB
:1002D0003F999D47E3E2A7FEF5B75C40268583D5AD
:1002E0004700EF809F90835584002685EF80FF8F25
:1002F0008D452685EF803F8EAA89EFF04FE093571A
:1003000005012380F90093578500A380F90023811C
:10031000A9005840C167FD178345A7006314FA0080
:1003200093E505082685EF801F8F9757FF1F93875A
:10033000674A9C430840D9CF8347B400858BD9CB0B
:1003400078003400130671008145EFF05FEB1DC9A2
:100350008347B400184093069005F99BA305F40069
:100360008347E701B387D702B306F70083C60604C5
:10037000A303D1009386170493879706BA96BA977A
:1003800036C43EC61754FF1F130444461C440C4099
:1003900026858983858B9D8D834771009E05DD8D24
:1003A00093F5F50FEF803F871C4410402245898369
:1003B000858BCA861D8EA685EFC0DFCFE31505F0BD
:1003C0001C440C40324689838840858B9D8DEFC04C
:1003D000DFC8D5BD8347B40013079005F99BA3057B
:1003E000F4008347E501B387E7023307F5000347CD
:1003F0000704A303E10013871704938797062A973E
:100400003E953AC42AC6BDBFEF129F91032A45000C
:100410009307F00FAA840347AA00AE893284368975
:100420006316F700EFB06FAB2305AA00938AC900EB
:100430000146D6852685EFF09FE62A8A21E51757E3
:10044000FF1F130767711843DC4039C383C6A70039
:100450000547638FE60283D547005685EF40102C91
:1004600005C9DC40839747006354F00201CC1C406F
:1004700089C74A868145014582975C4081C7CA8504
:10048000014582974E85EF807FA352856F109F8C28
:10049000DC4003D54700EF60BFD501E9DC4003D560
:1004A0004700EF60DFE181471DCD19C41C4089C7BB
:1004B0004A868145014582974E85EF807F9FAA85B8
:1004C0001755FF1F13050534EF80DF9511C45C40FD
:1004D00081C7CA85014582971755FF1F1305C5318E
:1004E000EF60F0368547D84085460346A700E30B0A
:1004F000D6F8031747006353E000C9F74A86A28580
:100500004E85EF703F97BDBFEF129F81AA840144D3
:100510001759FF1F1309C93B9309A004130A950833
:10052000EF703FC26344A400014535A03305340396
:10053000832709003E958357250099E30504CDB72D
:100540000357050083D7C401E31AF7FE5286854599
:10055000EFF0FFC065D56F10EFFFEF126FFCAA84BC
:1005600001441759FF1F1309A9369309A004EF701E
:100570005FBD6344A4006F10EFFD33053403832790
:1005800009003E958357250081CF83570500639965
:10059000970093059502130610022105EF80206A4B
:1005A0000504F1B7EF126FF90347E5012A84834789
:1005B000F5016307B70089E781452E856F102FFA93
:1005C000230FB400054781C9E398E7FE8947A30FCD
:1005D000F4008545DDB7638BE7020947E39FE7FC3D
:1005E0002285EFF02FA59757FF1F9387A71E9C43E7
:1005F00099E79757FF1F9387A7079C4389C7035520
:10060000C401EFF09FF5A30F0400E1B755D6C9BFB1
:10061000EF120FF1EFA0FFEE85476312F508EF80B0
:10062000EFCC1754FF1F130424531C4081CBEFA0C1
:100630003FFC89476304F5001C4082979757FF1FD2
:10064000938747199C43B9CF82979757FF1F93878A
:1006500027029C4391C382971754FF1F1304041968
:100660008327040B83D4C701EF60FFB78327040BF4
:10067000AA85144003C6E7011C448983858B99C36E
:100680001366260026854169EF40C03D8144D94963
:100690007D19EF705FB063CAA4006F10AFEBEF80FD
:1006A0000FCA41B7EF705F884DB7B3873403032794
:1006B000840ABA9703D527006308250103C64701BA
:1006C00083D50700EF40A03B8504E1B7EF124FE56B
:1006D00001449754FF1F938464111309400EFD5980
:1006E000EF70FF98634FA40401449754FF1F938455
:1006F000E40F13098002FD59EF707F98634CA40446
:1007000001449754FF1F9384640E5949FD59EF70BB
:100710009FA8634AA40497F5FFFF9385450A1755E0
:10072000FF1F13056514EF60D00797050000938540
:1007300085851755FF1F1305250CEF6050056F10B9
:100740006FE13307240383A7040B0504BA97239EA4
:10075000370179B73307240383A7C40A0504BA977E
:100760002390370151BF3307240383A7840A05046C
:10077000BA972391370161BFD4410387350085477C
:100780003356F5026377E600A54899E72380060013
:100790008280B387E702EDB73358F502038735004F
:1007A0003375F502B3D7E7021307000363DA0801D4
:1007B00003C6050013077003118A19E213077005B9
:1007C00085064297A38FE6FEC9B718451C4163769C
:1007D000F7005C41BA972380B7001C4585071CC50C
:1007E0008280EF128FD54111AA872E85B285368679
:1007F00036C6829763480500B246158D3335A00092
:100800003305A04041016F108FD5EF126FD10569FC
:1008100041112A8A2320060001448149975AFF1F6B
:10082000938A8A0D056B7D1932C62EC4EF703F8501
:10083000AA84EF70DF832695A24532466346A40062
:100840004E8541016F100FD103A70A0093171400C2
:10085000BA9703D707003377670101E71CC2050485
:10086000E1B703D707009356D700858AE39946FF7F
:1008700033772701E315B7FEBE89D5B7EF12EFCB6B
:1008800001112EC6B2843689EFB02FEE2A8461554D
:1008900001C8B24589E9232E040023200402014542
:1008A00005616F10CFCBA1463008CA852685EFF0D1
:1008B0005FF37DF5835781010357A101231EF400E7
:1008C0008357C1012310E4022311F4028357E1018D
:1008D000D207D1832312F4028357E1011397370122
:1008E00063560700FD57231FF4005DBF231F04005C
:1008F00045BFEF12EFC21754FF1F130424EF8327E5
:10090000040B03D7C701C167FD17630EF710975794
:10091000FF1F9387A7249C4381C70545EF4060775D
:10092000C1690149930A400EFD19175BFF1F130BA4
:10093000AB22EF70CFF3634BA90E1757FF1F03478E
:1009400067F29307F00563E4E702EF704FED93055C
:100950000006B3C5A502B7F73600938707E8175519
:10096000FF1F130565F0B385F502EF60A06F8145A9
:100970001705000013058520EF60DFF8EFB0EFDE0C
:1009800001CD0357C50109CB0357E50111C78347C3
:10099000050299C3EF60A06BEFB06FDE31C517574A
:1009A000FF1F0347E7F89757FF1F938767F80DCF9F
:1009B00003C717002304E50003C72700A304E500CD
:1009C00003C737002305E50003C74700A305E5007B
:1009D00003C757002306E50003C7670083C77700F6
:1009E000A306E5002307F5001C4493E717001757FB
:1009F000FF1F2321F7E05C4085E7EF708FEF0DC10B
:100A0000EF702FEF44402A89EF70AFEE33F5A40268
:100A10005C40FD17CA97898F1757FF1F232AF7DC01
:100A20000145EF70DF9F01456F10CFB2B30459034A
:100A30008327040BBE9483D7C40163883703138ACA
:100A40000403D2855285EFF0AFD605E183C7F401E8
:100A500099CF938594082E85EFF08FD509C9130699
:100A6000900581455285EF104FB00509D9B5832710
:100A70000B00268593B7170086072380F402EFE06A
:100A8000FFB8E5B7854763F8A7009307F5FFBE9564
:100A90003305A040E98D2E8582809841C167BA97C1
:100AA00013D707016304A7009CC182804207998F76
:100AB000E5BFEF128FA841112EC63284B684EFB085
:100AC0000FCCE15701C9B24591E99757FF1F238128
:100AD00007E681473E8541016F106FA89D46175676
:100AE000FF1F1306F6E4A6852285EFF09FCFAA87A5
:100AF00075F105479756FF1F238CE6E2E1BFEF1221
:100B00002FA2411191E99757FF1F23A307CE01445C
:100B1000228541016F100FA4B68532858D46700085
:100B2000EFF03FCC2A846DF58347D1000347E10005
:100B30001759FF1F130989CBA2074207D98F034713
:100B4000C100D98F1757FF1F2324F7CAEF706FDA40
:100B500061D1EF700FDA83244900AA89EF706FD951
:100B600033F5A40283274900FD17CE97898F1757C5
:100B7000FF1F232FF7C669BFEF122F9C1C45AA84C5
:100B800091CFD84B01CF83D7470089CBEF601F921D
:100B9000AA8509C588446105EF60C04C9757FF1FBF
:100BA000938747C39C43014489EF6F104F9B9C4838
:100BB00013171400BA9703D5070019C1EFE0CFCF80
:100BC0000504EF70CFC7E344A4FEC5B7EF12EF965C
:100BD000011185E9EF605FDA01449757FF1F23A3F6
:100BE00007CA9757FF1F23A107CA9757FF1F23AFB5
:100BF00007C89757FF1F23AD07C8228505616F10EF
:100C00000F96B6873285C9467000BE85EFF07FBD6E
:100C10002A8465F541469305E1001755FF1F13052A
:100C200065C6EF80C0010355C100EF608FD7F1B7F3
:100C30008DE19757FF1F23AB07BA9757FF1F938785
:100C4000E7BA9C470145ED9B1757FF1F2324F7BACE
:100C50008280EF128F8E4111B68532859546300025
:100C6000EFF03FB815EDA2471757FF1F2320F7B845
:100C70009757FF1F938787B79447B24713F7B6FF7D
:100C800013F6170019C213E74600858393F7F70799
:100C90009756FF1F23A0E6B61757FF1F2304F7BC84
:100CA00041016F10CF8BEF12AF8703841500DC4139
:100CB0002A89AE8485070387F7FF19C36340800C38
:100CC0008387240091C7635580007D14620461848A
:100CD0009C40370700FF0907F98F37070010090705
:100CE0006392E70A6355800079146204618483C7C4
:100CF0000400858B95E39379F40F4E8A93178A014C
:100D0000E187634AF008A287635304008147338474
:100D1000F9407D14620461848385240081C54A857D
:100D2000EFF0BFAA9C40370700FF0907F98F37078C
:100D300000100907639AE706930500034A85EFF060
:100D4000DFA883C7040093058005918B99E3930581
:100D500080074A85EFF07FA783C70400858B81CB8E
:100D60001374F40F93178401E1876347F004C040C4
:100D700005048305F4FFA1E96F00DFFD7D14620423
:100D800061840DBF370700080907E392E7F6E350D7
:100D900080F67D1499BF930500024A857D1AEFF015
:100DA000DFA2137AFA0F99BF370700080907E39506
:100DB000E7FA9305000371BF930500034A85EFF03E
:100DC000DFA07D1471BF4A85EFF03FA055B7EF0259
:100DD000DFF6EF70CFAA2A84EF706FA922958945BC
:100DE0000605EFE02FC6E55711C59757FF1F23A54E
:100DF000A7B081473E856F009FF693070002630608
:100E0000F5005D1513355500828005458280EF029F
:100E10003FF14111AA892A89130419008304F4FFC0
:100E200032C62EC42685EFF05FFDA245324659E159
:100E30009307D0026392F408830404000548130466
:100E400029009377F6FEC9E793070003639FF40E2A
:100E5000830704001307800593F7F7FD6399E706FE
:100E60008304140041460904B70600806314080097
:100E700093C6F6FFB3FEC6028147254F654EFD5F60
:100E800033D3C602138704FD6368EF06BA8463D5C3
:100E9000C408630DF5017D55636AF3006394670030
:100EA00063C69E000545B307F602A69705048304B2
:100EB000F4FFC9BF22898DB79307B0020148E392BE
:100EC000F4F8830404002A88130429009DBF01CA92
:100ED0008947E31BF6F893070003E397F4F88307C9
:100EE00004001307200493F7F7FD639BE7048304D2
:100EF0001400094609048DBF13E704021307F7F92C
:100F0000636CEE009388F4FB1307700363741E0197
:100F100013077005998CA5BF7D576300E502630434
:100F20000800B307F04091C519C19309F4FF23A04D
:100F300035013E8541016F00FFE1B687FDF5D5BF64
:100F40009304000315F2214605B719FE294629BF6F
:100F5000EF021FDD011161540DC53284AE89414697
:100F600081453689EFF0BFEA93140501C180639E85
:100F700009002685EF30102B014401C58145EF2083
:100F80005016228505616F00FFDC2285CD4670007A
:100F9000CA85EFF01F852A846DF52685EF309028ED
:100FA00009E90356C1008345E1012685EF20500B76
:100FB00001C941469305E1001105EF705048D1B7D2
:100FC0005D54C1B7EF02DFD50111E15401CDB28408
:100FD000AE89414681453689EFF07FE32A846397E5
:100FE00009008144268505616F00DFD62685D1463C
:100FF0007000CA85EFF0EFFEAA846DF58357C1003B
:10100000EDD3EF700F8E4205931704014181C18328
:1010100063F9A702EFB08FB64204E1474180330481
:10102000F40241460C082A9413054400EF70304145
:101030008357E1002311F4008357C1002310F4000B
:1010400055B7E55445B7EF02BFCD7971E15415C5E9
:101050003284AE8941468145B684EFF05FDB1319D7
:10106000050113590901639E09004A85EF40106587
:10107000814401C58145EFB02FB1268545616F00E0
:101080007FCDA6859306300270002285EFF06FF5C4
:10109000AA8465F54A85EF4070622A8411E54A8585
:1010A000EFB04F8C2A8431C58357C100231124012E
:1010B000930964002310F4008347E1009305F100D5
:1010C00041462302F4004E85EF7070371309740116
:1010D00041469305F1014A85EF707036930554003F
:1010E0004E85EFC04FBF930564014A85EFC0AFBE88
:1010F00069B7DD5459B7EF02BFC2797111E5E15408
:10110000268545616F001FC5B284AE894146814581
:101110003689EFF0DFCF131A0501135A0A01528501
:10112000EFE06FCA2A846398090071D98145EFB056
:101130002FB48144F1B72685930610027000CA854A
:10114000EFF02FEAAA844DFD31C8B2479305D100D4
:101150004146858B230FF400B247130504038583B2
:1011600093F7F707A30FF400EF70702D4146930536
:10117000D10113059408EF70902C59B7330469031B
:1011800083A70A0B3E948357C40163833703050981
:10119000EF60FFEDE344A9FEDD549DB7C16901494D
:1011A000974AFF1F938A8A64130B400EFD19CDB72F
:1011B000231E440159BF49CDEF029FB64111B289A8
:1011C000AE8441468145368AEFF07FC4931A05010B
:1011D00093DA0A010149174BFF1F130B2B61EF60D4
:1011E0001FE1634AA9000145ADCC81441749FF1FA7
:1011F0001309C95F81A883274B0B131439003E9450
:1012000083570400638857050509D1BF8327490B1D
:10121000139434003E948357040085E7231054014F
:1012200091467000D2854E85EFF0AFDB1DE9B247E5
:1012300013978700E1832183858B58C02301F40035
:101240000DA08504EF60BFDAE3C2A4FC5D5511A8D0
:1012500061558280F1F4214681452285EF00FFB07F
:10126000014541016F001FAF1971D2C4130AC106B5
:1012700086CEA2CCA6CACAC8CEC6D6C2B6D6BAD860
:10128000BEDAC2DCC6DE52C463810524FD151C1023
:101290002ACC2ECA02CE3EC89304B0021549A949F1
:1012A00083050600130416009DE1F2465247E2470B
:1012B00063FBE620B697238007007245F64066443C
:1012C000D6444649B649264A964A09618280930720
:1012D00050026386F5004808EFF02FCFF5A883573A
:1012E000C10023070100014593F7C70F2316F10042
:1012F000814501480147014681469308D002130306
:101300000003130E300205048307F4FF99C7638CB2
:10131000970463C3F404638BC70501CA0346C10085
:10132000858A799AD18E2306D10063090800834605
:10133000C100098BF59A558F2306E10019C12307D7
:10134000B100138707FD1377F70FA54663E2E606A2
:101350008146A545294535A0E38717FBE39F67FA3A
:101360000546FD564DB70545854571BF05487D5776
:1013700059BFB386A60205048307F4FFBA96E206B6
:10138000E18613F7F70F130607FD1376F60F63E5F3
:10139000C500138707FDF1BF1306F7F91376F60FA3
:1013A000636EC902138797FAE30537FDA306D100E0
:1013B000130790066385E704634BF7061307800560
:1013C0006384E70A6345F702E38107EE13075002DF
:1013D00093055002E381E7F02286D9B51307F7FBA6
:1013E0001377F70FE364E9FC138797FC75BF1307C6
:1013F00030066386E70A13074006E39FE7FC0325F0
:101400000A00A947A307F100930A4A0063580500A0
:101410009307D0023305A0402307F1006C00EFF0E2
:10142000AFB56C004808EFF01F88568A75B71307F0
:101430003007638EE7066341F7021307F006638EF9
:10144000E70413070007E399E7F80347C1001367B0
:1014500027002306E10009A813075007638BE70262
:1014600013078007E39AE7F6938787FA414793B714
:101470001700A307E100139727008347C100ED9BE6
:10148000D98F2306F100930A4A006C0003250A0055
:1014900079B7A947A307F100FDB7A147E5BF8305C9
:1014A0000A004808930A4A00EFF02FB2BDBF832715
:1014B0000A006C0048083EC8EFF0EFFE1C10930ACB
:1014C0004A003EC89DB7BA97FDB30145C5BBEF02C0
:1014D000DF862A88368583464800BA870347580046
:1014E000A206D98E328717B600001306669089E5EA
:1014F00017B6000013068690BE85EFF0FFD66F008A
:101500001F869747FF1F938727429C4381CFEF0297
:10151000DF82D843B2862E861847AA853E85029779
:101520006F00FF8361558280EF023F818357050082
:1015300039712A84231EF100834745009305650015
:1015400041461305F101230FF100EF70406F930541
:10155000740141461305F102EF70606E835624005A
:1015600017B600001306C691E5450A85EFF0DFCFF8
:101570006C08130630020A85EFF0BFF821616F0096
:101580000FFEEF028FFB39712A8493050503414654
:101590001305D101EF70A06A930594084146130525
:1015A000D102EF70C0698347E4010347F401835619
:1015B000C401858B0607D98F17B600001306068D68
:1015C000E5450A85230EF100EFF01FCA6C081306EB
:1015D00010020A85EFF0FFF221616F004FF8EF0271
:1015E0002FF437040001B70400FF0111814A1749A5
:1015F000FF1F1309A91F7D149389F4FF17BA000078
:10160000130A4A8DEF60BF9E63C5AA0005616F0093
:101610006FF48327490B13973A003E9783473700AF
:1016200095CF5C43A30107005286B3F6870082473B
:10163000E5454800E58FD58F3EC083462700B3F7C8
:101640003701858AE206D58F835607003EC0EFF04A
:10165000BFC111468A854800EFF0BFEA850A5DB731
:10166000EF02AFED01468145EFF0BFE96F002FEFCC
:1016700083576500638E071A1D71A2CCA6CACAC81B
:1016800086CECEC6D2C4D6C2DAC05EDE801013F7D4
:1016900017003289AA8431CBF99B2313F500EF6040
:1016A0001F9906053D0541990A8BC16A3301A14086
:1016B0008A8B8149014AFD1AEF607F97634CAA0C1F
:1016C0007947930604FB17A600001306A67FCA8578
:1016D0002685EFF0DFDF638F090C13961900DE8596
:1016E000130504FBEFF0FFE15A8183D7640013F781
:1016F000270021CBF59B2393F400EF605F94060550
:101700003D0541998A8A3301A1400A8B8149014AEA
:10171000EF60FF926345AA0A6547930604FB17A68C
:1017200000001306A67ACA852685EFF05FDA638784
:10173000090A13961900DA85130504FBEFF07FDC24
:10174000568183D7640013F7470005CBED9B2393A5
:10175000F4006547930604FB17A6000013064677BE
:10176000CA852685EFF0BFD69C4481C703D74700C2
:101770003DEB130504FBEFF0BFEE130104FAF64056
:101780006644D6444649B649264A964A064BF25B19
:1017900025618280DC4413171A00BA9703D707002B
:1017A0006308570193971900DE972390E700850996
:1017B000050A19B7130504FBEFF09FEA35B79C48FB
:1017C00013171A00BA9703D7070019C79397190080
:1017D000DA972390E7008509050A1DBF130504FB6E
:1017E000EFF01FE8B1BF2314E4FA03D767008326A4
:1017F000C4FA2146520751832315E4FA370700F053
:10180000758F9447930584FA130504FB9206918221
:10181000558F2326E4FA83C7770013F70701834720
:10182000F4FABD9BD98FA307F4FAEFF09FCDB1B7BF
:101830008280EF020FCE1744FF1F130424FB0444E1
:10184000797193F7F4FB1747FF1F2325F7FA93F7F6
:101850000404A1C78588A1E097A90000938989673E
:10186000EF60EFF863DBA4028327440B1399340085
:101870003E998356090091CE4E86E5454808EFF023
:10188000BF9E4808EFF0DFDD214681454A85EF0025
:10189000CFCD8504F1B7EFF09FD41C4413F7F7F7D1
:1018A0009746FF1F23A8E6F493F707086397071EE0
:1018B0001C4413F7F7EF9746FF1F23ADE6F213F72B
:1018C00007106318071E18449377F7DF9746FF1F2A
:1018D00023A2F6F29376072095C6058B630A0720AC
:1018E00018408983858B3ACA0347840715464C08FC
:1018F0000607D98F17A500001305855A230CF100A0
:10190000EFF03FC01C4413F7F7BF9746FF1F23A318
:10191000E6EE93F707408DC3835744000D464C080D
:10192000231AF1008357640017A50000130585579B
:10193000230BF100EFF0FFBC1844FD749387F47F94
:10194000F98F9746FF1F23A7F6EA9317470163DF36
:101950000700EFA08FE119C98356C5016391061AEC
:1019600017A5000013058554EFF09FCF1C447D7729
:101970007D177D8F9746FF1F23AEE6E6139737014D
:10198000635A0702858B6388071CEFA04FDF1DC1D8
:1019900018458347E5001D463ACA0357C5004C0861
:1019A00017A5000013050551231CE100230DF100CC
:1019B000EFF03FB51844F977FD17F98F9746FF1FF1
:1019C00023AAF6E29317270163D90700814517057B
:1019D0000000130525CAEF50FFF21844E177FD1708
:1019E000F98F9746FF1F23A7F6E09317070163D3EC
:1019F0000702EFA0BF982A84814417A900001309A9
:101A0000E94BEF600FEE939704014205C1834181DA
:101A100063EAA71445616F004FB383A70A009314CC
:101A20001900BE9483D7040033F767011DCF1396C6
:101A3000170133F77701B3F637016352060417A68F
:101A400000001306E64309E717A600001306064444
:101A5000E5454808EFF05F814808EFF07FC083D785
:101A60000400B3F747012390F4000509EF602FE16C
:101A7000AA84EF60CFDF2695E341A9FA15BD36852C
:101A800019C7EF40A04361DDEFF01FAAC9BFEFD037
:101A90009FB371D5EFF0FFAED9B785697D7A014963
:101AA000974AFF1F938A4AE5056B896BFD197D1ADA
:101AB00075BF858B9DC7EF500FF3231AA1004146D8
:101AC0009745FF1F938505DC13056101EF70201713
:101AD00049464C0817A500001305053CEFF07FA20E
:101AE000DDB317A500001305253BEFF07FB7E1BB81
:101AF00017A500001305C53AEFF09FB621B50357AF
:101B0000E501C17785073E978357A101FD1413377F
:101B100017003207E58FD98F231DF100231AD1005A
:101B200083560502035725022146231BD100231C9F
:101B3000E100035745028566FD16758FFD76F58F2A
:101B4000D98F4C0817A5000013054536231DF10059
:101B5000EFF03F9B21BD17A500001305A535EFF061
:101B60003FB089BD5C4813F7E7FF58C8858B89CF24
:101B7000A6864A86C9450A85EFF00FEF8357040011
:101B800099E70A85EFF0DFAD850461049DBD231A56
:101B9000F100835724009305440041462808231B85
:101BA000F100EF70C00951464C080A85EFF07F95AF
:101BB000E1BFEF028F9885473395A7009747FF1F36
:101BC0009387C7C29C47411181455D8D9747FF1F91
:101BD00023A2A7C29377057085E393576500858B91
:101BE000A1CBC167938707887D8D05EDEF606FD12D
:101BF0009305803EB305B5021745FF1F130505D0B9
:101C00002EC6EF50A03BB24519C16349B50085C54A
:101C10001745FF1F130585CEEF50C04441016F00EB
:101C20000F94EF600FCE2A84EF60AFCEE360A4FC88
:101C3000EF602FCE75BF0145EFF0BFBFC5B7EF0214
:101C4000CF8F7971AA8601441749FF1F130909BA7A
:101C500036C6EF60CFB9B246635CA4028327490B56
:101C600093143400BE9483D704006396D70285C6CC
:101C700017A6000013060626E5454808EFF0CFDE5C
:101C80004808EFF0FF9D214681452685EF00EF8D46
:101C900045616F00CF8C050465BF19C22320060083
:101CA000814701C59306D00389E53E85828085057D
:101CB0000505838705000307050099CF6394E700B6
:101CC000E397D7FE8147D5B79306D0038547E30E48
:101CD000D7FC93371700D1BF9307F002E316F7FE46
:101CE000854761D6050508C2C9B799C123A005007B
:101CF00081470DC11308D0031306F0023307F50026
:101D00008306070081CA638706016397C60099C1ED
:101D1000050798C13E8582808507CDB731C9EFF2AE
:101D20005EFF41112E8A6C002A89368BB28A97A4F5
:101D300000009384E40DEFF05FFB2A8C0144A68938
:101D4000B14B88406286CA85EF70E01801ED0E0441
:101D50004E945C403245DA865686D28582974101A0
:101D60006FF0BEFE0504A104E31D74FD6155C5BFFF
:101D70007D55828099E561558280615505616FF0DE
:101D80007EFDEFF2FEF92E8A2A8401118145B2848C
:101D900052854146BA893689EFF06F879315050160
:101DA000C1811376F50FA1812285EF507FB12A847E
:101DB00069D552854C08EFF05FF3524A2A8BE30E47
:101DC0000AFA2A8697A500009385C50F5285EF7001
:101DD0008010AA8A0DED7D5AEF606FA563C5AA0039
:101DE00099E8014561BF5C4413971A00850ABA97C8
:101DF00023904701D5B74C442EC6EF604FA3B245A0
:101E0000131615004E850299E34DA0FC85BF5A8636
:101E100097A500009385850B5285EF70C00B0DE1EF
:101E2000032A0401EF60AFA1131615008145528506
:101E3000EFF0BEF3DDD40C482EC6EF604FA0C1B763
:101E40005A8697A500009385A5085285EF70A008D3
:101E500041E11C44A5CF81ECD443370700E0758FE6
:101E60009447D8C33707001F758F98C701BFA14695
:101E70003008CE854A85EFE0DF96E31105F018447F
:101E8000835781017D762312F7008357A101939632
:101E9000470183576700D182F18FD58FF2467D7657
:101EA0007D16F182858AB206F18FD58F2313F70054
:101EB0008347E1018356C1012305F7008347B7003B
:101EC0002314D700FD8BA305F7004DBD7D557DB5CF
:101ED0005A8697A50000938525F35285EF60B07F61
:101EE000E31D05E81C4CE38A07E89C43E38707E809
:101EF000CE864A86A6852285829749B5EFF2FEE313
:101F00003687B2862E86AA850545EFF0BFE66FF0CC
:101F10001EE5EFF29EE23687B2862E86AA8501453F
:101F2000EFF05FE56FF0BEE3EFF29EDF411199C184
:101F300023A005009747FF1F9387079E8043814496
:101F40001DC82E89AA8931141DC40C4070004E850D
:101F5000EFF0BFD419CD81E8A284630C0900B24729
:101F60002320F90039A08C4008400146EFF0FFD251
:101F700065F5404869F8268541016FF0BEDD1841DE
:101F800011CBEFF29EDBAE873E85B2853686029797
:101F90006FF0FEDC35558280EFF23EDA8357C500E4
:101FA00013D70501C205B387E7021841C18148492B
:101FB000BA95BE95EFF0BFFC6FF07EDA584111CBB9
:101FC000EFF2BED7AE873E85B285368602976FF0B8
:101FD0001ED935558280184509CBEFF21ED6AE8743
:101FE0003E85B28502976FF09ED7355582805C455D
:101FF00099C7EFF29ED42E8582976FF05ED6355545
:102000008280EFF2FED183290500035AC5002A849D
:102010004849AE848145EFF09FFD2A890DE193D5B3
:102020000401B38545030356C4004848CE95EFF03C
:102030009FFA2A8909E548488545EFF05FFB4A8504
:102040006FF05ED1EFF2DECD2A890441035BC5005B
:10205000484979712E848145B28A368AEFF03FF97A
:1020600041E193590401B3896903420441802694F4
:10207000A29903440901330480403374440111CC14
:1020800003254901A2865686CE85EFF03FF3AA8448
:1020900031E1330A8A40A299A29A8144630C0A0270
:1020A0005286D685080803244901EF6050398346DB
:1020B00009011C089305F00F33864641338547011B
:1020C00036C6EFF09ECAB2461008CE852285EFF0E4
:1020D000FFEEAA84032549018545EFF05FF12685CF
:1020E00045616FF03EC7EFF25EC52E864C41A146BA
:1020F0002A84EFF03FF5AA8403450401A145EFE0EF
:102100007F985C403385A74048C026856FF03EC568
:10211000814797A600009386A6CC6393C700828070
:102120003387F500034707008507398D13574500AE
:102130003697034707001205398D1375F50F1357AE
:1021400045003697034707001205398D1375F50FC3
:10215000E9B7EFF29EBE2A84AA851D461305F00F4B
:10216000EFF01FFB834774003385A7403335A00091
:102170006FF0FEBEEFF27EBC4111A1463000EFF0E1
:10218000BFE109ED03578100C167FD1705456317DE
:10219000F7002800EFF0FFFB3335A00041016FF09E
:1021A0001EBCEFF2FEB7AE848C414111A1462A89D4
:1021B00003440501EFF05FDEAA8939E9A1452285D4
:1021C000EFE05F8C9C400357C9002A8AAA97939638
:1021D00007019CC0C182098F639CE602C16513D7C9
:1021E0000701B385B74011E78355E900FD15C20526
:1021F000BE958CC0A1460A864A85EFF0FFD9AA8910
:1022000001E90A85EFF0FFF401C9832749009CC06A
:102210004E8541016FF01EB40357C900835721005A
:1022200080403307474163DBE70033FA4703631716
:102230000A004177798C3E9480C0D9BF03450901DB
:10224000A145417AEFE01F84098CAA8A80C0337AC5
:102250004401417B63648A0081495DBFA14630002F
:10226000A2854A85EFF05FD3AA895DF12800EFF0DF
:102270005FEE11E98357A1000357C100337A6A0169
:1022800080C0BA973E9A33045441E9B7EFF2FEAAF0
:102290002A84AA851D461305F00FEFF07FE7A303FC
:1022A000A4006FF0DEABEFF2DEA62A840345050141
:1022B0005D71A145EFE00FFD5C402A8B0355E40002
:1022C0004179B3F727016C003EC6EFE00FFD83555F
:1022D000C400B247A1463008BE95B385654122854A
:1022E0002EC8EFF07FCBAA84634B05002808EFF0DF
:1022F0005FE611C9B2452285EFF0BFD0AA842685DA
:1023000061616FF09EA4C2470357A101417C338BEA
:102310006741B3F72701BA973EC810100C08228511
:10232000C24BEFF01FE8AA8479F90810EFF07FE2C2
:102330002DE95C403ECA30104C0822855249EFF02E
:102340005FE6AA844DFD035781028357010263169D
:10235000F7002810EFF0FFDF09C55840D247E31C13
:10236000F7FC63902B058357410285CF83572102E9
:10237000B3FA8B010810BE9A1C442311F102EFF04E
:10238000FFF083490401035A4102B309304193F934
:102390000902631B0A000C102285EFF0DFD4AA8427
:1023A00039FDE31C7BF7B9B74E8963733A01528953
:1023B000CA861018D6852285EFF01FBEAA8421F1A7
:1023C000630909000C44CA8610182285EFF09FC7E4
:1023D000AA8403450401CA85EFE0CFEA1C443E9578
:1023E00008C4E39E04F0330A2A41CA9A5DB7EFF2AB
:1023F0003E93411191E5FD54268541016FF09E9574
:10240000C44983D725014CC904C12316F50003C76D
:1024100005012A842317E50003C51501931607015A
:10242000130700022308A400C182E366A7FCE1D7DA
:10243000B3E4F402E9F08547E3FFD7FAA145EFE002
:102440006FE4AA89014A01498357C4009315090121
:102450002285BE95B38535412EC2EFF0BFD119ED6F
:102460000355E4004C00050AEFE02FE39245420AD1
:102470002285135A0A01EFF0FFCF09E905098357B6
:10248000E400420913590901E360F9FC8357E400B1
:1024900063944701D1548DB7639427039245A146B5
:1024A0003000B38535412285EFF01FAF35E12800BC
:1024B000EFF03FCA11C50355E4004C00EFE0EFDD3B
:1024C0009247C17A3387374158C04177F98F1CC48E
:1024D0004C401C4463EEF500A14630002285EFF02D
:1024E000BFAB1DE52800EFF0DFC6032A44001DC185
:1024F0005C400355E4004179B3F727014C003EC22C
:10250000EFE0AFD992452285EFF0DFC6635C0502AC
:10251000AA84DDB512450359A100035BC10033F560
:10252000AA002A9903450401DA85EFE0AFD54A9560
:1025300008C46314450163130B04330A3A41232290
:10254000440179B709C58547A308F40075B54C4027
:102550002285EFF01FAB4DFD48408357C40086092C
:102560003375A9003E953305354148C033752501C3
:1025700008C42285EFF03FD379D559BF4D5549BFE7
:1025800083471501C9CFEFF2CEF82A840345050130
:1025900041112E8AA145BA893689328BEFE08FCE60
:1025A0008357C4000605898F7D5563E727075C4084
:1025B00081443EC230004C002285924AEFF07FBE3B
:1025C00021ED835B810063994B012800EFF07FB818
:1025D00001E58504C204C18058409247630BF702AD
:1025E000E3FA99FC8356C10061559DC663E6340346
:1025F000C175B3FABA006373D900CA868355A100C6
:102600005A862285D695EFF03F9919E50355C1000A
:1026100021A06155E3884BFD41016FF00EF3495550
:102620008280EFF28EF10147EFF09FF56FF02EF30D
:10263000EFF2AEF03284B2862E8683554500084113
:10264000EFF03FFE635385002A8422856FF02EF160
:10265000EFF2AEEB834715013971C954BDC7034B87
:1026600005012EC62A84A1455A853689328AEFE0B3
:102670006FC10D473307E5028357C400AA8DFD548F
:10268000998F63E427056304090063000A045C4032
:102690003ECA30084C082285524DEFF09FB0AA89FF
:1026A00045ED8357810132476397E7002808EFF033
:1026B0005FAA630605105840D247E31CF7FC81442B
:1026C000631B090019A0814499E7268521616FF0F9
:1026D0008EE7E35CA0FE5A85CA85EFE0AFBA014BF6
:1026E00011C5330BB501420B135B0B01014D7D5C32
:1026F000C17B930C44008357E4006380A70D1C4406
:1027000044403307FB0063EBE40432472311F1023A
:102710000810FD572310E102231221032303F102C5
:10272000EFF0DFB6630909000C44CA8652862285A1
:10273000EFF05F91AA8903450401CA85EFE08FB4E9
:102740001C443E9508C4639909000C102285EFF0E3
:102750009F99AA89CA8435D9CE8485BF03450401CF
:10276000A145EFE02FB2B387A4002311F1028357F4
:10277000C400B3F4740123108103BE94898C44C057
:10278000081023120102EFF07FB00C102285EFF049
:102790009F95AA840355E400E685EFE00FB05C4006
:1027A000B3F777011CC4E39204F22285EFF0BFAFC8
:1027B000AA84E31C05F0050D3DBFC15439B783570A
:1027C000C101E30209F0E39827F1C177034C04014A
:1027D000B377FD00035DA101330C8041137C0C0233
:1027E0003E9DD28ACA8CE28B63F38C01E68BDE8637
:1027F0001010EA852285EFF02FFAAA84E31B05EC7E
:102800005E860C105685EF602041AA84E31505EC26
:10281000B38C7C415E9DDE9AE3970CFC7DB5EFF2B4
:10282000CED181460146EFF0BFE26FF04ED3638C0C
:10283000050EEFF20ECE5D71054D19C213BD1600E7
:1028400003590502B68B328B050942091359090158
:102850002E8A2A84CA89216C930A8500E15C93043C
:10286000F9FFC204C180638F84059306A004500061
:10287000A6855685EFF0FFDA6357050063139501CF
:10288000A6892689E9BF9C083E95230A05FA4C00D3
:102890005285EFF00ED875F563040D0883570402D6
:1028A000639597089387F4FF2310F4028946130673
:1028B0000402A1655685EFF0BFD963580506616132
:1028C0006FF0AEC80145E31C0DFE0549B1675D55CB
:1028D000E387F9FE9165CE9593048400C205DE86F8
:1028E0005A86C1812685EFF0BFD6630D0900528557
:1028F000EF60405DAA865286CE852685EFF05FD5D3
:10290000E34F05FA8357040263FF370323103403B0
:10291000894613060402A1652685EFF07FD325A022
:10292000A689014965B77D558280A6855685EFF059
:102930001FEFE34605F89165FD15CA95C205C181F3
:102940005685EFF0DFEDE35CA0F601458DBFEFF2B9
:102950004EBC03540502916A1D71050442042A8984
:10296000AE894180A16B130A8500FD1A130B050285
:102970009304F4FFC204C180639D7405916B2164CC
:10298000130A8900850B170C0000130CACCA83577F
:10299000090293041400C204C18085076383F40E06
:1029A0005E949306A0045008A68552854204EFF079
:1029B0005FC74180AA8A854613067100A2855285A9
:1029C000EFF03FC62A8B634750076347A006268473
:1029D0007DBF56949306A0045008A68552854204F4
:1029E000EFF03FC441802A8C854613067100A28512
:1029F0005285EFF01FC3634C8003E351A0F8835767
:102A00000902E39D97F69387F4FF2310F9028946A4
:102A10005A86A1655285EFF0BFC3A6855285EFF0B7
:102A20001FE0A2855285EFF09FDF268491B7E3581F
:102A3000A0FCA9B7634BA000A6855285EFF03FDE4E
:102A4000A2855285EFF0BFDD59B79C10BE9A238A4C
:102A50000AFA639109022C004808EFF0EFCC25D95F
:102A60001C45224552C62318810074006286DA850F
:102A70008297B1BF0146CE854808EFF00FA261FDF5
:102A8000B9B7014525616FF04EACEFF20EAB973749
:102A9000FF1F938767E88043814409C42A89311462
:102AA000814401E426856FF08EAB631809005C4415
:102AB00081EF404865D83114EDB708400146CA851A
:102AC000EFF0AF9D6DF5F5B78297E5F4AA84D5B721
:102AD000EFF2AEA69737FF1F938787E48043AA845F
:102AE00009EC2685EFF07FFAAA840144EF502FD03D
:102AF000636CA40026856FF08EA65C402285A685B7
:102B00009C4382970040E9BF05041374F40FF9BF9A
:102B1000EFF2AEA20145EFF0BFFB6FF04EA4973786
:102B2000FF1F9387E7DF23A0070023A2070082800F
:102B3000EFF2AEA09737FF1F938707DE23A00700B1
:102B400023A20700EFF0BFFD6FF06EA1EFF2EE9E43
:102B50004111130985002A84EF50CFE5AA854A85E3
:102B6000EFF0FF88AA8419ED89461306E100A165FC
:102B70004A85EFF01FABE177634405008357E1001E
:102B80002310F402268541016FF06E9D9737FF1FD9
:102B9000938707D990430147B28691EE05E3DC4362
:102BA00010C11737FF1F232DA7D685EF9737FF1FBB
:102BB00023AAA7D6828036879442C5B7144385E2FC
:102BC000DC432320050091EB9737FF1F23ACA7D4EC
:102BD0009737FF1F23A6A7D4828088C3C1BF14C123
:102BE00008C38280EFF26E951734FF1F130484CE62
:102BF0002285EFF0BFF5AA8405E5179900001309B7
